:020000040100F9
:10000000585A0020E5000001ED000001EF0000015A
:1000100000000000000000000000000000000000E0
:10002000000000000000000000000000F1000001DE
:100030000000000000000000F3000001F5000001D6
:10004000F7000001F7000001F7000001F7000001D0
:10005000F7000001F7000001F7000001F7000001C0
:10006000F7000001F7000001F7000001F7000001B0
:10007000F7000001F7000001F7000001F7000001A0
:10008000F7000001F7000001F7000001F700000190
:10009000F7000001F7000001F7000001F700000180
:1000A000F7000001F7000001F7000001F700000170
:1000B000F7000001F7000001F7000001F700000160
:1000C0000348854600F02EF90048004799210001B9
:1000D000585A002040BA7047C0BA70470138FDD165
:1000E000704700000448804704480047FEE7FEE7E9
:1000F000FEE7FEE7FEE7FEE769120001C10000012E
:1001000030B50B46014600202022012409E00D46AF
:10011000D5409D4205D31D469540491B2546954037
:1001200040191546521E002DF1DC30BD03460B432D
:100130009B0703D009E008C9121F08C0042AFAD29D
:1001400003E00B780370401C491C521EF9D2704723
:10015000D2B201E00270401C491EFBD2704700225F
:10016000F6E710B513460A4604461946FFF7F0FFB6
:10017000204610BD421C0178401C0029FBD1801A8A
:10018000704710B5002200E0521C835C8C5CA342D7
:1001900001D1002BF8D1D8B2E1B2401A10BDC9B2DA
:1001A00003E003788B4203D0401C521EF9D200209A
:1001B000704730B504460020034600E05B1C9342C4
:1001C00003D2E05CCD5C401BF8D030BD03460A781A
:1001D0000270401C491C002AF9D11846704730B5FE
:1001E00005460020034600E05B1C934205D2EC5C10
:1001F000C85C201A01D1002CF6D130BDF7B582B011
:100200000F460026029C01F04FF900900068019013
:100210002578641C002D05D000F02CF80068405DA6
:10022000C007F5D12B2D02D02D2D1CD0641E0098B7
:100230000021016039462046049A00F01FF801466B
:10024000002F04D03868A04201D10298386000988D
:10025000006802280BD00098019A0260700506D54C
:10026000484205B0F0BD012080020643DFE70846A2
:10027000F7E700000048704764310001F7B582B02D
:10028000029C00272078641C15460197302802D074
:10029000002D15D015E020780127641C782804D0A3
:1002A000582802D0002D09D00BE0002D01D0102DD0
:1002B00007D1002710252078641C02E0082500E003
:1002C0000A250026009610E00099012769430818C6
:1002D000020C294680B2714300908E183804864281
:1002E00001D3012001902078641C294600F02CF8ED
:1002F0000028E9DA0398002805D0002F01D0641EF9
:1003000000E0029C04600198002806D001F0CCF8BF
:1003100002210160C81E05B0F0BD009930040843F9
:10032000F9E70000064C0125064E05E0E36807CC1E
:100330002B430C3C98471034B442F7D3FFF7C4FE6C
:1003400098340001B83400013A2800D23038202314
:1003500002469A43412A01D310463738884201D3D6
:100360000020C04370470000F0B58DB006460F4630
:100370002C22444902A8FFF7D9FE02A801F06CFD27
:10038000002804D140A001F0CFFE0DB0F0BD022E38
:100390000FDB01A9786802F045FB002805D1019820
:1003A00001280DD0019802280AD045A001F0BCFE1A
:1003B000EBE70398012801D1022000E00120019021
:1003C00001990398884204D14CA0019901F0DEFD07
:1003D000DBE70198012801D104A800E008A8044641
:1003E0000198012801D14C4800E04C480090216858
:1003F0000098814207D16068002804D00721890352
:100400006068884206D96368226845A0019901F0B6
:10041000BDFDBAE750A001F087FE6168206801F0D9
:100420002DFD0546A168A94209D02B46A26858486F
:10043000019901F0ABFD57A001F076FEA5E76368D6
:10044000E26861A0019901F0A1FD0198039002A862
:1004500001F00CFC002803D06BA001F065FE94E7CE
:100460006EA001F061FEC82001F0F4FA00BFBFF3F6
:100470004F8F71487149C860BFF34F8F00BF00BFF5
:10048000FEE700000040000161707073773A20625F
:100490006F6F7473657474696E67207265636F72D1
:1004A0006420696E76616C69642C20726566757370
:1004B0006520746F207377697463680D0A0000000B
:1004C00075736167653A206170707377205B317C6A
:1004D000325D20286E6F20617267203D207377693E
:1004E00074636820746F20746865206F7468657227
:1004F0002062616E6B290D0A00000000617070734C
:10050000773A20616C7265616479206F6E2041508A
:1005100050256C750D0A00000080000100400201AA
:1005200061707073773A2062616E6B256C75207212
:1005300065636F726420696E76616C6964202861FE
:100540006464723D30782530386C582073697A6560
:100550003D256C75290D0A0061707073773A20761D
:100560006572696679696E67207461726765742067
:10057000696D616765206372632028666577207303
:1005800065636F6E6473292E2E2E0D0A0000000025
:10059000043400012020202020202072756E20428B
:1005A0004C45204F544120746F2077726974652048
:1005B000612076616C696420696D61676520666998
:1005C0007273740D0A00000061707073773A2062D4
:1005D000616E6B256C7520696D616765206F6B209E
:1005E000287665722030782530386C582C20256CA0
:1005F000752042292C20737769746368696E672EB1
:100600002E2E0D0A0000000061707073773A20668C
:100610006C617368206661696C0D0A0061707073AB
:10062000773A20646F6E652C207265736574746907
:100630006E672E2E2E0D0A000400FA0500ED00E074
:1006400030B58BB004460D462C2204496846FFF7AE
:100650006DFD684601F04AFB0BB030BD0040000163
:1006600070B58CB006460C46032E0ADA53A001F092
:100670005BFD5AA001F058FD5E4801F055FD0CB03D
:1006800070BD6946A06802F0CDF9002803D05AA0D9
:1006900001F04AFDF3E72C225C4901A8FFF746FD73
:1006A00001A801F0D9FB002806D12C2101A8FFF7F1
:1006B00056FD57A001F038FD63A16068FFF761FDAA
:1006C00000280CD10098012806D00098022803D0F9
:1006D0005FA001F029FDD2E70098029058E0606821
:1006E0000078622850D160684078312803D0606873
:1006F0004078322848D160684078312801D103A879
:1007000000E007A805466168881C59A1FFF739FD7C
:1007100000280ED158490098884207D057490098C0
:10072000884203D056A001F0FFFCA8E7009828609B
:100730002EE06168881C61A1FFF723FD00280BD122
:10074000072189030098884203D95EA001F0ECFCE0
:1007500095E7009868601BE06168881C62A1FFF75C
:1007600010FD002802D10098A86011E06168881C83
:100770005EA1FFF706FD002802D10098E86007E0BF
:100780005BA001F0D1FC7AE759A001F0CDFC76E73F
:1007900061685DA0009A01F0F9FB01A801F066FA1A
:1007A000002803D061A001F0BFFC68E764A001F05D
:1007B000BBFC01A801F09AFA00BF60E7757361679E
:1007C000653A206273736574203C6669656C643EAB
:1007D000203C76616C3E0D0A000000002020666916
:1007E000656C643A20616374697665203C317C32C3
:1007F0003E0D0A004C34000162737365743A206246
:1008000061642076616C75650D0A0000004000018E
:1008100062737365743A206578697374696E6720D2
:100820007265636F726420696E76616C69642C20F6
:1008300072656275696C642066726F6D2073637295
:10084000617463680D0A0000616374697665000075
:1008500062737365743A20616374697665206D759F
:1008600073742062652031206F7220320D0A0000FF
:100870006164647200000000008000010040020119
:1008800062737365743A2061646472206D75737469
:100890002062652043414949435F415050315F42E6
:1008A000415345206F722043414949435F415050B5
:1008B000325F424153450D0A0000000073697A65BA
:1008C0000000000062737365743A2073697A6520D2
:1008D00065786365656473207468652062616E6B1A
:1008E0002073697A650D0A00637263007665720091
:1008F00062737365743A20756E6B6E6F776E2066E7
:1009000069656C640D0A000062737365743A202592
:1009100073203D2030782530386C582C2077726950
:1009200074696E672E2E2E0D0A00000062737365C7
:10093000743A20666C617368206661696C0D0A0008
:1009400062737365743A206F6B20287665726966EE
:10095000696564290D0A0000F8B5164C164920682F
:10096000884208D12821204601F088FAA16A8842ED
:1009700001D1012000E00020064665680FA112A009
:1009800001F004FB002E03D117A001F0CDFB0225DE
:10099000294620A001F0FAFA01F088F87D21C9006B
:1009A0000090FFF7ADFB074639461FA001F0EEFAB5
:1009B000F8BD00000040000111C011CA56312E30B0
:1009C000312E303300000000626F6F746C6F616411
:1009D00065723A2025732C20646F776E6C6F6164AA
:1009E000206D6F64650D0A00626F6F7473657474B7
:1009F000696E673A20494E56414C4944202D204F9C
:100A00005441207461726765747320415050310DF8
:100A10000A0000006375722062616E6B3A204150DB
:100A200050256C750D0A0000757074696D653A206B
:100A3000256C7520730D0A0070B506460D46022E12
:100A40001EDB002415E00C226243194B995868689C
:100A5000FFF797FB00280BD10C206043144BC01804
:100A600042680C206043195812A001F08FFA70BD43
:100A7000641C092CE7D312A0696801F087FAF6E735
:100A800018A001F051FB00240BE00C206043084B40
:100A9000C01842680C206043195806A001F076FA8D
:100AA000641C092CF1D312A001F03EFB00BFDEE76D
:100AB000442D00012020252D38732025730D0A00B8
:100AC000756E6B6E6F776E20636F6D6D616E643ADD
:100AD0002025732028747279202768656C70272977
:100AE0000D0A0000636F6D6D616E64733A0D0A004C
:100AF0006B6579733A20544142203D20636F6D70DD
:100B00006C6574650D0A000070B504460D46034817
:100B100001F00AFB01200249087070BD6831000134
:100B20000C40002008A001F0FFFAC82000F092FF5E
:100B300000BFBFF34F8F08480849C860BFF34F8F0D
:100B400000BF00BFFEE70000726573657474696ED4
:100B5000672E2E2E0D0A00000400FA0500ED00E0BD
:100B600070B504460D4605A001F0DEFA0BA001F0B9
:100B7000DBFA17A001F0D8FA70BD0000757361723E
:100B800074313A2054583D5042362052583D50421C
:100B9000372028414634290D0A000000626175643F
:100BA0003A203436303830302C203820646174617B
:100BB00020626974732C206E6F2070617269747981
:100BC0002C20312073746F70206269740D0A00004C
:100BD000666C6F7720636F6E74726F6C3A206E6F05
:100BE0006E653B2074783A20706F6C6C65643B20B6
:100BF00072783A20444D412072696E672028334B49
:100C0000422C20706F6C6C6564290D0A0000000096
:100C100070B504460D4605A107A001F0B7F91148CB
:100C2000016811A001F0B2F970BD000056312E30FC
:100C3000312E303300000000626F6F746C6F61649E
:100C400065722076657273696F6E3A20257320286D
:100C5000646F776E6C6F6164206D6F6465290D0A37
:100C6000000000000040002053797374656D436FED
:100C70007265436C6F636B203D20256C7520487A4C
:100C80000D0A00000168254A114001600021016041
:100C900041608160C1602249884208D120490839F9
:100CA00049680F2211431E4A083A516035E01C4939
:100CB0001431884208D11A4908394968F022114391
:100CC000174A083A516028E015492831884209D16D
:100CD0001349083949680F2212021143104A083A91
:100CE00051601AE00E493C31884209D10C4908395B
:100CF00049680F2212031143094A083A51600CE077
:100D000007495031884208D10549083949680F22FE
:100D100012041143024A083A51607047FEFF000076
:100D200008000240002904D0026801231A4302602F
:100D300003E00268014B1A4002607047FEFF0000AA
:100D40000146486880B2704710B5002202680D4B1A
:100D50001A400C6A8B6823430C6923434C69234374
:100D60008C692343CC6923434C6A23438C6A234315
:100D70001A430260CB6843600B6883604B68C360B2
:100D800010BD00000F80FFFF10B5002B01D01061D7
:100D900001E00024146110BD70B503460A4600212D
:100DA0000024002076E001268E40156835402C4650
:100DB000002C6ED05568022D02D05568122D20D11E
:100DC00008250D40002D0ED0586A4D07EE0E0F2558
:100DD000B5400646AE4330464E07F60E5569B5405F
:100DE000284358620DE0186A4D07EE0E0F25B540F6
:100DF0000646AE4330464E07F60E5569B5402843C9
:100E000018625568012D08D05568112D05D0556818
:100E1000022D02D05568122D0BD1586801258D4046
:100E20000646AE4330461579ED06ED0F8D4028435A
:100E3000586018684E000325B5400646AE4330465C
:100E40001579AD07AD0F4E00B54028431860D8683E
:100E50004E000325B5400646AE4330464E00956829
:100E6000B5402843D860986801258D400646AE43BA
:100E70003046D5688D4028439860D86A4E000125D9
:100E8000B5400646AE4330464E001569B54028438E
:100E9000D862491C1568CD40002D84D170BD00007A
:100EA000054901600F2141610021416081600121FC
:100EB000C160002101617047FF3F00000246002031
:100EC00013690B40002B01D0012000E00020704787
:100ED000F7B5D4B004460E4600205390052052903A
:100EE0000025002700BFEFF310800090FF2145315F
:100EF00001A8FFF734F901F0B9FD05462448854201
:100F000018D101200003844202D1002053902AE02E
:100F100001204003844202D14011539023E003207A
:100F20000003844203D10120400253901BE05298F9
:100F300057B0F0BD1748854213D101200003844209
:100F400001D153900FE001204003844201D153901E
:100F500009E003200003844201D1539003E052983A
:100F6000E6E75298E4E705AF0137FF2241320A492C
:100F700001A8FFF7DBF8012000F0A9FA3146569AE4
:100F80005398B8475290009800F0A1FA5298CFE7D2
:100F9000C4401300856013006A2B000170B504463D
:100FA000002500BF00BFEFF310800546012000F0D0
:100FB00091FA00BF01200006241A2046054909685D
:100FC0008847064600BF284600F084FA00BF304636
:100FD00070BD00005040002010B508480849086066
:100FE000943008490860FF382D3807490860C92245
:100FF000920006490938FFF799F810BDCD4F00203F
:10100000504000205440002058400020BC2D0001DA
:10101000F8B504460D461646002700BF00BFEFF3A3
:1010200010800746012000F055FA00BF012000069D
:10103000241A324629462046054B1B6898470090E3
:1010400000BF384600F046FA00BF0098F8BD000027
:1010500054400020002905D0054A52690243044B40
:101060005A6104E0024A52698243014B5A61704757
:1010700000100240002905D0054A92690243044B42
:101080009A6104E0024A92698243014B9A61704777
:101090000010024010B500210022214B5B6804249F
:1010A00023401946002902D0042906D102E01D4B35
:1010B000036005E01C4B036002E01A4B036000BFB5
:1010C00000BF174B5B683024234019460909174BB2
:1010D0005A5C0368D3404360114B5B6807242402C9
:1010E00023401946090A124B5A5C4368D340836077
:1010F0000B4B5B68E40023401946C90A0C4B5A5C51
:101100004368D340C360064BDB6A10242340002BA6
:1011100002D0084B036102E07D23DB03036110BDB5
:10112000001002400090D0030048E801B82D0001F3
:10113000B02D000100093D00F1B58AB000200990F2
:101140007D20C00008900125AD02002700200790F7
:101150007F20069040240026002005900390200167
:101160000290002001903E490A98884206D83D48E6
:101170000068610288433B49086006E0394800681E
:101180000121C9030843374908607D21C9000A9835
:10119000FEF7B6FF7D21C9000090FEF7B1FF4501C3
:1011A00000BF304800687F21090288430190200277
:1011B000019908432B4908600520FEF78FFF10E0D6
:1011C0000120FEF78BFF2748406B022108400028D2
:1011D00000D007E00598411C05910899884200D984
:1011E00000E0EDE700BF1F48C06B86B2AE4201D9F8
:1011F000771B00E0AF1B0298874203D2E0B2039056
:10120000B8B20290AE4201D3069400E0079406996A
:1012100007984018C005000E04900498A04200D121
:1012200003E0049C09988742BBD800BF0D480068C2
:101230007F21090288430190039800020199084325
:10124000084908600846406840084000486000BF00
:1012500004484068042108400028F9D10BB0F0BDD3
:101260000090D0030010024010B53E48C069012133
:10127000090708433B49C861812000063A490863D1
:101280003A4848613A4808623A48006803218903AD
:101290008843384908603421374800F073F83648ED
:1012A0000069401C002803D033480069002817D18A
:1012B0002C4840680121090408432A49486008462F
:1012C000406807210902884326494860084640686B
:1012D00009150843234948602848FFF72DFF3FE0E0
:1012E000214880694409640123480078C006C00E83
:1012F00004431D4884611B4800680121C9038843D9
:1013000018490860084600687F210902884304469E
:1013100019480069000220431249086008464068E5
:101320000121090408430F49486008464068072125
:10133000090288430B49486008464068091508437C
:10134000084948600846006A0D4908400549086296
:101350000846006A0849C968090208430149086249
:1013600010BD000000100240007000400F08000097
:101370001800020000100140604000200090D003DF
:10138000FF00F8FF70B504460D462A4621460120AD
:101390000003FFF79DFD70BD002905D08289012360
:1013A0005B031A43828103E08289024B1A408281E7
:1013B00070470000FFDF0000002A03D0838A0B4340
:1013C000838202E0838A8B43838270470246002037
:1013D00001235B02994200D100BF13880B40002B10
:1013E00001D0012000E0002070470000F0B589B076
:1013F00005460E4600240020089000BF00BF0027CD
:10140000B089002800D000BF2F462C8A2048044015
:10141000F08804432C82AC891E480440B08831898E
:101420000843718908430443AC81AC8A1A480440DC
:10143000B0890443AC8201A8FFF72CFE174887420D
:1014400002D10498089001E0039808903268910056
:101450001923089A5A431046FEF752FE079064215A
:101460000798FEF74DFE04012109642041430798C7
:10147000411A069106990901084632306421FEF7A7
:101480003FFE0007000F04432C8109B0F0BD0000AF
:10149000FFCF0000F3E90000FFFC0000003801402E
:1014A000CA05D20D82807047004870475C4000201A
:1014B00002E008C8121F08C1002AFAD1704770471D
:1014C000002001E001C1121F002AFBD1704780F308
:1014D0001088704780F3108870470000002007498B
:1014E000087007490860074908600749086007490C
:1014F00008600749087007490870704710400020CD
:1015000024400020284000202C40002034400020AF
:101510004440002045400020002002490870024954
:10152000088070474C40002048400020F7B584B048
:101530000746494906980860002686E0BC5D474892
:101540000078002804D0012810D0022874D13AE095
:10155000CA2C0AD142480470012042490880052063
:101560004149088001203D4908706BE03D480188F1
:101570000088401C3B4A108039484454104600887B
:1015800005281FD13649C978354A1279120211430C
:101590000846FF21E131884205D900212F4A117008
:1015A000304A11800DE0C11D2F4A11801146098873
:1015B0002C4A1288914201D1002100E00221274AE1
:1015C000117000BF3EE0274801880088401C254A72
:1015D00010802348445410460088234909888842D3
:1015E00028D11F48C0781E490979090208430546D9
:1015F000281D81B21A48401C00F0B0FE0390681DFF
:101600001749095CA81D164A105C000201430291AB
:1016100002990398884207D11046817840782B467A
:10162000521D019000F034F800200C4908700D495B
:10163000088000BF06E0FFE700200849087009495C
:10164000088000BF00BF701C86B20598864200DA91
:1016500074E707B0F0BD0000404000204C4000207F
:10166000444D0020484000204A40002031B5064A41
:1016700001216846FFF75AFF044804780020034917
:101680000870204638BD00003D290001464000207A
:10169000F8B504460D4616461F46102C06D0112CF0
:1016A0000AD0122C0ED0132C24D111E03A46314628
:1016B000284600F099FE1EE03A463146284600F0E2
:1016C0004BFF18E03A463146284601F019F812E07F
:1016D000FFF704FF0948002213210368284601F0A0
:1016E000EFF8074800680749884202D101200649FF
:1016F000087000E000BF00BFF8BD000024400020DB
:10170000404000203D2900014640002010B511480E
:10171000007800281CD000F0C9F90F490968441A64
:101720000E480078002803D0FF202D30844203D2D9
:101730007D20000184420AD300BFBFF34F8F0848C9
:101740000849C860BFF34F8F00BF00BFFEE700BF6E
:1017500010BD00003A4000203C40002039400020ED
:101760000400FA0500ED00E0F8B507460D463846DE
:10177000FEF700FD84B20BA000F0D6FC002604E0CA
:101780000BA000F0D1FC701C86B2AE42F8DB05A0C5
:1017900000F0CAFC002C03D02146384600F04EFA77
:1017A0002046F8BD0D63616969632D3E00000000AD
:1017B0002000000008B5002400253A4800F0B4FCE1
:1017C00000BFFFF7A3FF3848007800280ED000F0D4
:1017D0006DF9401B3549884208D90020324908700C
:1017E000FFF79AFE32A000F09FFC0024684600F04C
:1017F000F9F9002800D1E4E72B480078002810D040
:1018000000F054F9054668460078FFF72FFF0028DE
:1018100006D00020244908702FA000F085FC002489
:10182000CFE7684600780A280BD004DC082816D0D9
:10183000092823D11CE00D2802D07F281ED10FE0FB
:1018400000BF30A000F070FC00202F49085508466A
:1018500000F036FB00241EA000F066FC20E000BF74
:10186000002C04D0601E84B228A000F05DFC17E0BC
:101870002146254800F04CF8044611E068460078FF
:1018800020280CD34F2C0AD2684602782046611CCF
:101890008CB21D490A540121684600F0CFF900BFFF
:1018A00000BF8EE7A03200010C400020B80B000002
:1018B0000D0A5B6F74615D2062696E617279206DE3
:1018C0006F6465204F4646202869646C65290D0ABF
:1018D00063616969632D3E000D0A5B6F74615D2071
:1018E00062696E617279206D6F6465204F46462093
:1018F0002861626F7274290D0A63616969632D3E04
:10190000000000000D0A0000F44C00200820080030
:10191000F0B597B007460C460025002002902246FD
:1019200020213846FEF73BFC002802D0204617B0A5
:10193000F0BD0020385500262AE00C2070434149B4
:1019400008580190224639460198FEF748FC0028C5
:101950001DD10298002808D103A80199FEF736FC92
:1019600003A8FEF707FC85B20EE001E0681E85B211
:10197000A54206DD2A4603A80199FEF730FC00289F
:10198000F4D1002003A948550298401C0290761C0F
:10199000092ED2D30298002801D12046C7E7029829
:1019A000012819D109E003A90819012100F046F91D
:1019B00003A8005D3855601C84B24F2C01D2AC42A4
:1019C000F1DB4F2C06D220203855601C84B21EA0BB
:1019D00000F0AAFB2046AAE7A5420FDD09E003A913
:1019E0000819012100F02AF903A8005D3855601C90
:1019F00084B24F2C23D2AC42F1DB20E013A000F0E4
:101A000093FB002612E00C2070430E490858019009
:101A1000224639460198FEF7E2FB002805D10198DD
:101A200000F082FB0AA000F07FFB761C092EEAD3AF
:101A300006A000F079FB21463846FFF795FE2046C8
:101A400075E70000442D0001200000000D0A000091
:101A50002020000000B5024600F028F8034600BF31
:101A600000F024F8C01A9042FAD300BD00B587B048
:101A700001210820FFF7FEFA01A8FFF711FA202044
:101A80000190002002900220039001A90648FFF770
:101A900083F920210448FFF711FA012801D107B08A
:101AA00000BD0020FBE70000000C01400748006972
:101AB000012109040840002804D005480068401CA2
:101AC00003490860024800687047000000E000E039
:101AD0000840002000B595B001210820FFF7CAFAA0
:101AE00001218803FFF7C6FA0FA8FFF7D9F94020B4
:101AF0000F9002201090042014900FA93148FFF796
:101B00004BF980200F90042014900FA92D48FFF767
:101B100043F9E120C0020B9000216846018641860E
:101B2000818601870C21C1860BA92748FFF75EFC3F
:101B300001210846FFF78EFA00212448FFF7F2F84A
:101B40002248FFF79FF80123204A20491C3903202F
:101B5000FFF71AF91C48001D00901D480190002055
:101B600002900320800203900020049080200590C2
:101B70000020069007902020089000020990002085
:101B80000A9069461148FFF7DFF8002011490880E4
:101B900001210E48FFF7C6F8012240210A48FFF74D
:101BA0000BFC01210848FFF7F7FB0B480B49486184
:101BB000002088610520086100200949086015B0EF
:101BC00000BD0000000C0140003801401C00024034
:101BD0009440002004400020FFF9000000E000E0F5
:101BE0000840002070B5044600F01CF805460B487C
:101BF0000088A84201D1002070BD09480749098822
:101C0000405C20700321890204480088401CFEF7D4
:101C100077FA024801800120EEE70000044000202E
:101C20009440002010B50448FFF78AF80321890288
:101C3000081A80B210BD00001C00024070B50546B5
:101C40000E4600240CE0295D0748FFF729FC00BF81
:101C500080210548FFF7BAFB0028F9D0601C84B248
:101C6000B442F0DB70BD00000038014010B50446FE
:101C700000F02EF810482060204600F021F8A06205
:101C80000E48FFF78BF9002801D0012010BD2C224F
:101C900021460A48FFF7BCF9002801D00120F5E7EA
:101CA0002C2206492046FEF784FA002801D00120A4
:101CB000ECE70020EAE7000011C011CA0040000173
:101CC00010B504462821204600F0D8F810BD0000C9
:101CD00010B505480078002804D1FFF77DF90120F0
:101CE0000149087010BD00004D40002070B5044649
:101CF000204600F0B1F8002801D015A000E016A0A1
:101D000005462A461A491BA000F040F920A0216888
:101D100000F03CF925A0616800F038F929A023699A
:101D2000E268A16800F032F932A0616900F02EF992
:101D300036A0236AE269A16900F028F92DA0616A42
:101D400000F024F93DA0A16A00F020F970BD000068
:101D500076616C6964000000494E56414C4944204C
:101D600028626164206D616769632F637263290073
:101D700000400001626F6F7473657474696E672050
:101D8000402030782530386C583A2025730D0A00F1
:101D900020206D61676963202020202020203D20C5
:101DA00030782530386C580D0A000000202061631F
:101DB000746976655F62616E6B203D20256C750DE0
:101DC0000A000000202062616E6B313A2061646479
:101DD000723D30782530386C582073697A653D251E
:101DE0006C75206372633D30782530386C580D0A6D
:101DF0000000000020202020202020202076657276
:101E00003D30782530386C580D0A00002020626182
:101E10006E6B323A20616464723D30782530386CE4
:101E2000582073697A653D256C75206372633D3077
:101E3000782530386C580D0A0000000020206372AD
:101E4000633332202020202020203D203078253090
:101E5000386C580D0A00000010B504460649206889
:101E6000884207D12046FFF72BFFA16A884201D1A3
:101E7000012010BD0020FCE711C011CA30B5024698
:101E80000B460021C94312E01078521C4140002447
:101E90000BE04808CD07ED0F002D01D0074D00E005
:101EA000002568400146601CC4B2082CF1DB1846CE
:101EB0005B1E0028E8D1C84330BD00002083B8ED88
:101EC000F0B589B0074600263C4621E000E0641CDE
:101ED00020782028FBD020780928F8D02078002806
:101EE00000D11AE03046761C800001A90C5000E0B9
:101EF000641C2078002805D02078202802D0207883
:101F00000928F5D12078002802D000202070641C18
:101F10002078002801D0082ED8DB00BF002E02D187
:101F2000002009B0F0BD002513E00C226A430D4BE0
:101F300099580198FEF725F9002809D10C2068432B
:101F40000849401801A98268304690470020E8E718
:101F50006D1C092DE9D304A0019900F017F80120A8
:101F6000DFE70000442D0001756E6B6E6F776E2009
:101F7000636F6D6D616E643A2025732028747279E9
:101F8000202768656C7027290D0A00000FB4F0B592
:101F900089B0644C0FA80890B0E00E9800780790C4
:101FA0000E98401C0E900798252803D007982070A3
:101FB000641CA3E000200690202605900E9800786F
:101FC0002D2804D1012006900E98401C0E900E98EA
:101FD0000078302803D130260E98401C0E900BE07C
:101FE0000E9800780E99491C0E91014630390A224C
:101FF00005985043081805900E980078302803DBA8
:102000000E9800783928EBDD0E9800786C2802D104
:102010000E98401C0E900E980578002D02D00E9858
:10202000401C0E90642D21D006DC252D58D0582D53
:1020300045D0632D58D112E0732D04D0752D2CD0CE
:10204000782D51D13AE020200090089802C80890DD
:102050002046069B059A00F02BFD04464CE00898AC
:102060000178001D08902170641C45E0089880C824
:102070000890FB0F002F01DA784200E038460A2270
:1020800002A9019000F03BFD009602A92046069BA4
:10209000059A00F00DFD04462EE0089901C90023C1
:1020A0000A22089102A900F02AFD009602A9204602
:1020B000069B059A00F0FCFC04461DE000BF089951
:1020C00001C900231022089102A900F018FD009612
:1020D00002A92046069B059A00F0EAFC04460BE0A4
:1020E00025202070641C07E025202070641C002D32
:1020F00001D02570641C00BF00BF00BF0E9800789F
:10210000002804D007485430844200D245E700201C
:1021100008902070034800F007F809B0F0BC08BC34
:1021200004B01847944C002070B504462046FEF7D2
:1021300021F885B229462046FFF780FD70BD0000DA
:1021400001460A684B68094882420DD3084882421A
:102150000AD808460830834206D3072080030818AF
:10216000834201D2012070470020FCE7014000209B
:1021700000C0002004460120C00720430549086331
:10218000206880F3088800BF62B66068804700BF9F
:10219000FEE70000007000401CB5344C344801904C
:1021A000002700263349206888421CD12821204678
:1021B000FFF764FEA16A884215D16168022902D145
:1021C0002146183101E02146083108460127284AF6
:1021D0000168914206D3412292040168914201D2E2
:1021E0000168019100BFFFF775FC23A000F031FCEE
:1021F000FFF73CFC002803D001262FA000F029FCAB
:10220000002E1BD1FFF752FC05460FE06846FFF792
:10221000E9FC002809D0684600780D2803D06846FC
:1022200000780A2801D1012607E000BFFFF73EFC35
:10223000401B7D2109018842E8D300BF002E0AD14E
:10224000002F08D10A48FFF77BFF002803D10126A1
:1022500025A000F0FEFB002E04D030A000F0F9FB1A
:10226000FFF7A8FA0198FFF785FF00000040000182
:102270000080000111C011CA0D0A5B626F6F745DAE
:102280002043414949432D424F4F542056312E306F
:10229000312E3033202D20456E746572207769749D
:1022A00068696E2032733A20646F776E6C6F616478
:1022B000206D6F64650D0A005B626F6F745D207343
:1022C000747261702070696E204849474820283335
:1022D0005633293A20646F776E6C6F6164206D6F9E
:1022E00064650D0A000000005B626F6F745D206E14
:1022F0006F2076616C69642061707020696D616720
:10230000652C20666F7263656420646F776E6C6FF6
:102310006164206D6F64650D0A0000005B626F6F81
:10232000745D20444F574E4C4F4144204D4F44451F
:1023300020286F74612F636C69206F766572205559
:102340004152542C202768656C702720666F7220DC
:10235000636F6D6D616E6473290D0A0030B50246BE
:102360000F4817E01578521C2C02604000230EE045
:102370000124E4030440002C04D04400094D6C40C7
:10238000A4B201E04404240C20465C1CE3B2082BF8
:10239000EED300BF0B464C1EA1B2002BE2D130BDE4
:1023A000FFFF00002110000010B5044611E00C49A9
:1023B00009680C4A12688818FEF7F0FD002801D061
:1023C000052010BD07480068012109034018054990
:1023D000086004480068A042E9D30020F1E700004B
:1023E000144000202C400020F7B586B00C4615465E
:1023F0000C2D09D0102D07D00023012210210698A2
:1024000000F05EFA09B0F0BD204600F04DFA064635
:10241000201D00F049FA05902046083000F044FAEB
:102420000490102D04D120460C3000F03DFA00E05D
:102430000020039036480078002807D03548022253
:1024400010210368069800F03BFADBE7324F33496E
:102450003868884208D128213846FFF70FFDB96A4D
:10246000884201D1012000E000200190019800285D
:1024700004D07868012801D1294800E02948029059
:10248000042E03D307208003864206D900230322AB
:102490001021069800F014FAB4E7234800780028C9
:1024A00004D1FEF799FD01201F4908700120184949
:1024B00008701E49029808601D4806601D4905986D
:1024C00008601D49049808600020124908601B49F3
:1024D00008601B4908601B4908600398C007C00FCB
:1024E000002806D0184800681849884201D1012008
:1024F00000E00020164908700020164908700023EB
:102500001A461021069800F0DBF900BF7AE70000B8
:1025100010400020244000200040000111C011CADA
:1025200000400201008000013840002014400020DB
:10253000184000201C40002020400020284000209F
:102540002C40002034400020404000203D29000164
:102550004440002045400020F7B582B06148007833
:10256000002807D1002302221121029800F0A8F9C7
:1025700005B0F0BD0498042807D25B480122112160
:102580000368029800F09CF9F2E7039800F08CF9D8
:1025900001900398061D0498041F00945249019865
:1025A0000968884212D051480078002803D050486A
:1025B0000078002809D14C480222112103680298B2
:1025C00000F07EF901204A490870D1E746480068CA
:1025D000001948490968884207D943480322112154
:1025E0000368029800F06CF9C2E73F4800680019E0
:1025F0003D49086008460068FFF7D6FE0546002DF5
:1026000021D13D48006800281DD00AE031783A48C1
:1026100002680068401C384B186038488154761CAA
:10262000641E35480068042801D2002CEED13248DF
:102630000068042807D10421304800F019F9054644
:1026400000202D490860002D0BD1042C09D3A708C8
:10265000BF003946304600F00BF90546F619E41B79
:1026600000BF002D08D1002C06D022463146234859
:10267000FDF75CFD20480460002D09D01A482A4669
:1026800011210368029800F01BF9FEF727FF6FE79E
:1026900000201749087015480078002819D0124802
:1026A00001680098081A000B00030F490968090B1C
:1026B0000903884205D10C4800680E490968884220
:1026C00006D10948002211210368029800F0F8F8A9
:1026D0004EE70548002211210368029800F0F0F847
:1026E00000BF45E710400020244000204440002067
:1026F0004540002018400020344000203040002099
:10270000F7B50E4650480078002806D10023022273
:102710001221009800F0D4F8FEBD0298042807D0DA
:102720004A48012212210368009800F0C9F8F3E733
:10273000304600F0B9F80546444800684449096845
:10274000884207D04148022212210368009800F015
:10275000B7F8E1E73F480068002820D008E0FF21F3
:102760003C4802680068401C3A4B18603A48815463
:10277000384800680428F2D30421374800F078F87C
:10278000002809D03148052212210368009800F082
:1027900097F8FEF7A3FEBFE700202E4908602C48FB
:1027A00001682E480068FFF769FB0446AC4203D17C
:1027B0002B480068844209D024480422122103686F
:1027C000009800F07DF8FEF789FEA5E72348006831
:1027D000001D00F069F8074620480068083087426D
:1027E00006D31E4800681A4909684018B84209D83B
:1027F0001648062212210368009800F061F8FEF7DF
:102800006DFE89E700F0A8F8002809D00F480522DE
:1028100012210368009800F053F8FEF75FFE7BE793
:102820000020104908700A4800221221036800980D
:1028300000F046F8FFF73AF90B49086001200B4910
:10284000087000BF68E7000010400020244000200E
:102850001840002034400020304000201440002068
:102860001C400020394000203C4000203A4000201D
:1028700070B505460C460A4909680A4A1268881864
:1028800022462946FEF7C4FB002801D0052070BD72
:10289000044800680019034908600020F7E70000B9
:1028A0001440002028400020014608784A7812028F
:1028B00010438A7812041043CA78120610437047F6
:1028C000FFB587B005460E461C4668460675099951
:1028D000417584752004010E6846C1752002010E01
:1028E00068460176200E694648761348006800283D
:1028F0001FD0CA21684601711F21417185710621CF
:10290000C17100210172062205A90930FDF70EFCF4
:102910000A2101A80130FFF721FD07466846C77369
:10292000391201740D2101A8034A126890470BB0B7
:10293000F0BD00BFFBE700004040002070B504463A
:102940000D4629462046FFF779F901200149087014
:1029500070BD00003940002010B58CB02C222A49EF
:1029600001A8FDF7E3FB29490198884206D12821F7
:102970002548FFF783FA0B99884203D02C2101A840
:10298000FDF7EDFB2148019021480068214988426C
:1029900001D1012000E0022002901D4800681D497D
:1029A000884201D103A800E007A80446184800683F
:1029B000206019480068606018480068A0601848E6
:1029C0000068E060282101A8FFF758FA0B900E4834
:1029D000FEF7E4FA002802D005200CB010BD2C222E
:1029E00001A90948FEF714FB002801D00520F4E7EF
:1029F0002C22054901A8FDF7DCFB002801D00520A9
:102A0000EBE70020E9E700000040000111C011CA17
:102A10001440002000800001184000201C400020CD
:102A200020400020F8B504460D460020009000220A
:102A300069462046FDF7E2FB06460098A04203D017
:102A400000980078002801D00120F8BD2E600020F9
:102A5000FBE710B5044604E02046641C0121FFF7A3
:102A6000EDF820780028F7D110BD000070B5D2B085
:102A70000024002500BFEFF310800646FF214531FA
:102A800001A8FDF76CFB01AC01349822074901A8AD
:102A9000FDF74CFB0120FEF71AFDA0470546304626
:102AA000FEF715FD284652B070BD0000AA2C0001AB
:102AB000F8B504460D4616461F462846FDF75AFB54
:102AC0000090002F08D102E006982070641C304668
:102AD000761E00998842F7DC03E0287820706D1C90
:102AE000641C28780028F8D102E020202070641CA3
:102AF0003046761E00998842F7DC2046F8BDFFB5C7
:102B000083B007460C46002500BF38460599FDF7FF
:102B1000F7FA0E460A2E02D23046303001E0304637
:102B20003730C2B22846691CCDB269460A543846CD
:102B30000599FDF7E5FA0746002FE6D1069800282B
:102B400005D02D222846691CCDB269460A5406E0FC
:102B5000681EC0B205466946085C2070641C002DE2
:102B6000F6D10020207007B0F0BD40BA7047C0BA5F
:102B700070470138FDD170470000F7B50325AD0659
:102B8000286A82B016460C46400840002862286A2F
:102B9000022108432862286A8007FCD46620686006
:102BA00001272F61A86AC005FCD5992068602F61B4
:102BB000A86AC005FCD5FF209130FFF7DAFFFF239C
:102BC0000133AB626846EF60352169602F61A96A05
:102BD000C905FCD5AB62A969EF60C9B205226A607C
:102BE0002F61AA6AD205FCD5AB62AA690902D2B2EA
:102BF00011430180C80702D0032005B0F0BDAB62CD
:102C00006869FF210831884368616869C91E084303
:102C1000686102980002483068600820A860EE6091
:102C20002F61A86AC005FCD5FF200130A8620023EF
:102C3000F61CB0080ED0B208114800689900605424
:102C4000060A09194E70060C000E8E705B1CC870C7
:102C50009A42F1D8FF200130A8626869FF2108314B
:102C600088436861686938436861286A8008800021
:102C70002862286A38432862002005B0F0BD800031
:102C8000000C032080064169FF2208329143416114
:102C9000426901210A434261026A9208920002627B
:102CA000026A0A430262704700000020032189067D
:102CB000096A490849000322920611621146096A0D
:102CC0000222114303229206116200BF03218906EA
:102CD000096A022211400229F8D0D101032292068A
:102CE00091620321D1609F2151600121116100BFD8
:102CF00003218906896AFF22013211409142F7D1EE
:102D0000032292069162114688694969FF220832BE
:102D100091430322920651611146496901221143F0
:102D20000322920651611146096A890889001162DD
:102D30001146096A0122114303229206116270476B
:102D4000000000007C33000148330001390A000113
:102D50002C3300011C330001110C00014033000131
:102D6000483200015909000184330001F0320001AA
:102D700041060001BC330001D831000161060001A9
:102D8000FC330001C433000169030001EC3200018F
:102D900010320001090B0001B43300018032000140
:102DA000250B0001343300018C330001610B00015D
:102DB0000000000001020304000001020138FDD1FF
:102DC00070470000F0B40324A406236A5B085B008C
:102DD0002362236A02252B432362236A9B07FCD4C8
:102DE000FF230133A3626569DE1DB5436561656933
:102DF0001E1D3543656100026B3060600820A060D5
:102E0000E26001262661A06AC005FCD5A36200230A
:102E1000D21C90080ED095080F4800689A0088547C
:102E2000070A52185770070C000E97705B1CD07081
:102E30009D42F1D86069FF21083188436061606973
:102E400030436061206A800880002062206A30433D
:102E50002062F0BC002070478000000CF8B50646E8
:102E600001200025C004864201D90520F8BD0324B5
:102E7000A406206A400840002062206A022108431C
:102E80002062206A8007FCD4FF270137A76200F088
:102E9000BBF8002801D0032515E006206060012161
:102EA0002161A06AC005FCD5A762300220306060B5
:102EB0002161A06AC005FCD5A7620C4800F0C8F8E3
:102EC000002800D102256069FF2108318843606134
:102ED0006069012108436061206A800880002062E7
:102EE000206A084320622846F8BD0000E6960100EB
:102EF000F7B506460120C00482B01546864202D9C5
:102F0000052005B0F0BD03208006016A490849008C
:102F10000162016A022211430162016A8907FCD43D
:102F2000FF2101318162F2B28C1AA54200D8ACB205
:102F30000398009000F068F8002840D10621480668
:102F4000416001210161816AC905FCD5FF21013180
:102F50000320800681624169FF220832914341616A
:102F60004169042211434161310232314160C46040
:102F70000022002C16D9009887183B78F87819465B
:102F80007B7800061B021943BB781B0419430143DD
:102F90000802F978000A0906084319490860121D59
:102FA000A242E8D30121032080060161816AC9059C
:102FB000FCD5FF2101318162124800F049F8A54299
:102FC00009D00398361900192D1BFF2401340390F2
:102FD000A542ADD8ABE7032080064169FF22083245
:102FE000914341614169012211434161016A8908AC
:102FF00089000162016A11430162002005B0F0BD41
:103000008000000C1A06000038B401250320800659
:103010006A46C560352141600561816AC905FCD5F4
:10302000FF24013484628169C560CBB2052141600F
:103030000561816AC905FCD5846280691902C0B244
:10304000014388B21180C00700D0012038BC70470E
:10305000F8B400210125032292066B46D560352481
:1030600054601561946AE405FCD5FF270137976227
:103070009469D560E4B2052656601561966AF60536
:10308000FCD5976296692402F6B234431C80E307AC
:1030900022D0814202D9F8BC002070470322920658
:1030A0006B46D560352454601561491C946AE4056B
:1030B000FCD597629469D560E4B205265660156127
:1030C000966AF605FCD5976292692402D2B214433F
:1030D000A2B21C80D207DCD1F8BC012070470000EE
:1030E000004040404040404040404141414141401B
:1030F00040404040404040404040404040404040D0
:10310000400502020202020202020202020202025E
:103110000220202020202020202020020202020263
:1031200002029090909090901010101010101010BB
:1031300010101010101010101010101002020202C7
:10314000020288888888888808080808080808080B
:103150000808080808080808080808080202020207
:1031600040000000E13000015B6F74615D20626926
:103170006E617279206D6F6465204F4E202D207333
:10318000656E642030784341204F5441206672615F
:103190006D6573206E6F770D0A28626C655F7072C3
:1031A0006F746F636F6C2E6D642073656374696FE9
:1031B0006E20362E363B204F54415F41424F5254D1
:1031C000206F722033732069646C652065786974A0
:1031D00073290D0A000000006273736574203C6659
:1031E00069656C643E203C76616C3E3A207772697A
:1031F000746520626F6F7473657474696E6720669E
:1032000069656C6420286361726566756C212900AC
:103210006F74613A205541525420656E7465727323
:10322000204F54412062696E617279206672616D2F
:1032300065206D6F646520287365652068656C7016
:10324000206F74612900000073686F7720626F6FD0
:103250007420696E666F202B206375722062616E28
:103260006B20284F5441207772697465732074680D
:1032700065204F544845522062616E6B2900000062
:1032800072657365743A2073797374656D20726525
:1032900073657420287265626F6F742900000000E6
:1032A0000D0A434C492072656164792028626F6F72
:1032B000746C6F6164657220646F776E6C6F6164AB
:1032C000206D6F6465292E2054797065202768650C
:1032D0006C702720666F7220636F6D6D616E647312
:1032E0002E0D0A63616969632D3E00006F746100F1
:1032F000627364756D703A2073686F7720626F6FC8
:103300007473657474696E67207265636F7264208C
:103310002B2063726320636865636B0073686F774B
:1033200020626F6F746C6F61646572207665727372
:10333000696F6E0075617274696E666F00000000DF
:10334000646576696E666F0068656C70205B636D9E
:10335000645D3A206C69737420636F6D6D616E6497
:1033600073202F2073686F77206F6E6520636F6DF9
:103370006D616E6427732068656C700068656C70A1
:1033800000000000627364756D70000075617274F6
:10339000696E666F3A2073686F77205553415254B7
:1033A000312070696E732F626175642F666F726D64
:1033B0006174000072657365740000006273736568
:1033C000740000006170707377205B317C325D3A6D
:1033D0002073776974636820626F6F742062616E16
:1033E0006B2028637263207665726966696564295B
:1033F000202B207265626F6F740000006170707323
:103400007700000061707073773A2062616E6B25FF
:103410006C7520696D61676520637263206D6973E7
:103420006D6174636820287265636F726420307800
:103430002530386C582C2061637475616C203078AD
:103440002530386C58290D0A00000000202020206B
:1034500020202020206231616464727C62326164C9
:1034600064727C623173697A657C623273697A65F1
:103470007C62316372637C62326372637C62317638
:1034800065727C6232766572203C6865787C646522
:10349000633E0D0A00000000B83400010040002027
:1034A00060000000B01400011835000160400020E9
:1034B000F8190000C01400010090D00300000000C3
:1034C00000000000000000000000000000000000FC
:1034D00000000000000000000000000000000000EC
:1034E00000000000000000000000000000000000DC
:1034F00000000000000000000000000000000000CC
:1035000000000000000000000000000000000000BB
:083510000000000000000000B3
:1040000011C011CA010000000080000124DB000083
:104010006EDA83231C000100000000000000000095
:0C40200000000000000000001AC4DC25B5
:10800000E8BD002069810001718100015DB10001BE
:108010000000000000000000000000000000000060
:10802000000000000000000000000000C5B50001D5
:10803000000000000000000027810001C9B5000118
:108040007B8100017B8100017B8100017B8100013C
:108050007B8100017B8100017B8100017B8100012C
:108060007B8100017B8100017B8100017B8100011C
:108070007B8100017B8100017B8100017B8100010C
:108080007B8100017B8100017B8100017B810001FC
:108090007B8100017B8100017B8100017B810001EC
:1080A0007B8100017B8100017B8100017B810001DC
:1080B000D1B700017B8100017B8100017B81000140
:1080C0000348854601F076F80048004785FE000128
:1080D000E8BD002040BA7047C0BA70470138FDD1F2
:1080E0007047000040BA7047C0BA7047704670478A
:1080F000084B19680868203080F30988022080F353
:108100001488BFF36F8F3FBCAE4608BC04BC62B698
:1081100018470000C4470020EFF3108072B6704784
:1081200080F310887047EFF309800E4B1A682038EF
:108130001060F0C044464D4656465F46F0C008B554
:1081400072B60BF09DFA62B60CBC1168086810306C
:10815000F0C8A046A946B246BB4680F3098820383D
:10816000F0C81847C4470020044880470448004727
:10817000FEE7FEE7FEE7FEE7FEE7FEE721B60001C9
:10818000C180000130B50B460146002020220124A9
:1081900009E00D46D5409D4205D31D469540491B3B
:1081A0002546954040191546521E002DF1DC30BD84
:1081B00070B500242546002801DA01244042002938
:1081C00001DA01254942FFF7DDFFAC4200D0404211
:1081D000002C00D0494270BDF0B51FB40646002007
:1081E00082B005464024019100901BE0019922468F
:1081F0000F46304600F02DFE049A059B801A9941E7
:1082000010D310461946224600F013FE361A8F414D
:108210000197224601200021009F00F00AFE381835
:108220004D4100902046641E0028DFDC019B009831
:108230002946324607B0F0BD01464139192900D818
:10824000203070470549064A08685043054A80189F
:108250000860400870470149086070471C480020CA
:108260006D4EC6413930000003460B439B0703D0D7
:1082700009E008C9121F08C0042AFAD203E00B78EB
:108280000370401C491C521EF9D27047D2B201E063
:108290000270401C491EFBD270470022F6E710B561
:1082A00013460A4604461946FFF7F0FF204610BD64
:1082B000421C0178401C0029FBD1801A704710B580
:1082C000002200E0521C835C8C5CA34201D1002B95
:1082D000F8D1D8B2E1B2401A10BDC9B203E00378B8
:1082E0008B4203D0401C521EF9D20020704730B59B
:1082F00004460020034600E05B1C934203D2E05C8E
:10830000CD5C401BF8D030BD03460A780270401C9B
:10831000491C002AF9D11846704730B5054600209F
:10832000034600E05B1C934205D2EC5CC85C201A5B
:1083300001D1002CF6D130BD0FB400B58DB009903D
:108340000B9010A900200091C0430A9000200C90CF
:1083500006480690064807906A4609A80F9900F05B
:10836000B1FD0DB008BC04B018470000E58E000157
:10837000058F0001FFB5087889B01546FF2805D0A4
:10838000491C2D2804D00022002407E000240BE023
:108390000122F9E70A235C430419491C0878FF28E5
:1083A000F8D1002A00D06442002004902A780146C7
:1083B0002D2A01D02B2A0FD16D1C2D2A02D000228C
:1083C000049209E00122FBE700260A2233466D1CD5
:1083D00000F0F2FC381871412F78FF2FF4D10C9A7D
:1083E000A218069202460A4304D0FF23069A91334C
:1083F000DA4205DA002109980A4606C00DB0F0BD40
:108400000024B74AB54D2646079200F011FC0290B1
:1084100006980391002801DA474200E00746390533
:108420000020AF4A001C51410191009012E0F80772
:1084300007D022462B463046079900F0D9FA064667
:10844000079122462B461046194600F0D1FA044601
:108450000D467F10002FEAD10698019B0028009A54
:108460000399029806DA00F02BFB3246079B00F0D6
:1084700027FB05E000F0BCFA3246079B00F0B8FA93
:10848000049A002A02D00122D2075140099A03C25D
:10849000B4E7FFB591B0002009900025ED432E20F0
:1084A0009E685C681F460190B9696D1C12988847E8
:1084B0000090396A88470028F6D10098401C0AD0FD
:1084C0000D20C0018443002E12DD00982B2809D016
:1084D0002D280DD103E00020C04315B0F0BD0120D0
:1084E00080020443B9696D1C12988847761E00907B
:1084F00003A9600501D52D2000E02B206A461073EA
:10850000491C0CA80F9102900AE0B9696D1C1298E1
:10851000884700900120400204431398761E0560AE
:10852000002E02DD00983028EFD001990098884293
:1085300046D18020044308E00998401E099001209C
:10854000400204431399681C0860B9696D1C761ECB
:108550001298884700903028EED031E00199884287
:1085600005D1200603D480200443761E1EE0009827
:1085700003F03CFB002826D001204002044307A959
:108580000F980331761E88420BD200980F9930382D
:1085900008700F98401C0F90200607D50998401EC0
:1085A00003E0200602D40998401C0990A00502D5DA
:1085B0001399681C0860B9696D1C1298884700906F
:1085C000002ECBDC59E0002E57DD0098652801D045
:1085D000452852D1A00550D5032000028443B96933
:1085E0006D1C761E129888470090002E0CDD2B28FB
:1085F00004D02D2808D1FF2001300443B9696D1C37
:1086000012988847761E0090E00501D52D2100E0E4
:108610002B21029801700298401C0290019025E0E5
:108620000120400204430EA902980131761E8842BF
:108630000ED20098029930380006000E087003D15F
:108640000299019881420AD90298401C029006E0E2
:10865000E00501D5234801E0224840420990B9696C
:108660006D1C12988847009013980560002E04DD59
:10867000009803F0BBFA0028D2D1F9691298884714
:108680000F99FF200870029903AA087000200A9031
:108690000B900CA90AA8099BFFF76CFEA00502D459
:1086A0000120C04319E72420044209D0E00713D178
:1086B00038680B9A0A99031D3B60006806C00BE0FE
:1086C0000B990A9800F05CFB0146E00704D138687A
:1086D000021D3A60006801602846FEE60000144072
:1086E0000000F03FF1D8FFFFF7B582B00F4600263B
:1086F000029C03F067F90090006801902578641CE3
:10870000002D05D000F0CAFB0068405DC007F5D120
:108710002B2D02D02D2D1CD0641E0098002101604D
:1087200039462046049A00F0FFFB0146002F04D092
:108730003868A04201D10298386000980068022889
:108740000BD00098019A0260700506D5484205B02A
:10875000F0BD012080020643DFE70846F7E7F8B5E1
:1087600002464A40D40F42004B0052085B089A422E
:1087700002D20246084611464A0023D0C30D4A00E1
:10878000DDB2120EAD1A202D35DA49020126490A52
:10879000F6058A19002C00D0524220214F1B1146A9
:1087A000B9402A411018C20D9A4221D0002C17D08E
:1087B000012D08DCDA05801AD20F8019D207DBB24E
:1087C00000F060FCF8BDDA05801A012340001B06AA
:1087D000C01880185A428018CA0F1043490007E099
:1087E0004908C2071143DA05801A80194008801829
:1087F00000F040FCF8BD61000122511A001BF7E7B0
:108800000122D2075140AAE70122D2075040A6E731
:10881000024670B54A40D30FDB0740002DD04A0016
:108820002AD0010E140E000212020919400A520A3F
:108830008418E50104465443000A120A2E045043EA
:10884000A4194219200CC543AA18120C0125AD0326
:10885000521C521912047F39240400D0521C1043B8
:1088600001D44000491EC2B20C06C0092018401CA9
:108870004008802A02D003E0002070BD400840007C
:10888000002900DA0020184370BD0000F0B507464B
:108890000846584087B0C00F049048000E46590063
:1088A00040084908BC1A884105D2384631461E4660
:1088B00017460B4602465800400810434CD0300D76
:1088C000039040055900400D490D0590401A029053
:1088D000402872DA18030121000B090508430190B2
:1088E00004980092002805D0019952420020884146
:1088F00000920190029840210A1A0199009800F014
:1089000098FA05460C466B4607CB00F0B3FAC0193F
:108910007141039A0E0D0023D71756401A467A402C
:10892000164344D0049A002A2DD0029A012A039AB1
:1089300015DC1205C01A914101263605001C714153
:10894000D20F059ED2070093019202962A46234633
:1089500000F0DEFB07B0F0BD38463146FAE71605F9
:10896000224A0F46B218C01AB74101210905001C5E
:108970004F4100187F41114618187941E20F10430A
:108980006D19644113E0E2076D0815436408C207DE
:108990001443039A01261205C01A91413605001CA2
:1089A0007141CE07400830434908C01851412A465A
:1089B000234600F0A0FBCDE7FFE70498012240002A
:1089C000C117121A00238B4104983146C417381A74
:1089D000A141EEE730B40124E407634030BC55E721
:1089E00030B40124E407614030BC4FE70000E0FFF1
:1089F000F0B51FB488B00B99099800244840099934
:108A0000C00F490049080991C0070B99009049001F
:108A100049080B9109990898A64608431CD00B9960
:108A20000A98084318D0099801244000420D4800D4
:108A3000410D099824050003000B204309900B9871
:108A40000003000B20430B9050181C4940180022D3
:108A500001901446104605E0002001460DB0F0BD1F
:108A6000032801DA034600E003239C46C11A0AAE3C
:108A70000AE05F0008ADED5B4F00F75B7D43002728
:108A8000AA187C41491C5B1E6145F2DD410004AB24
:108A90005A522104120C0A43240C401C0828DFDB24
:108AA000019802900099704601910090059B049AEC
:108AB0000799069800F02CFBD0E700000DFCFFFFA3
:108AC000F0B50C465C4085B0E40FE40703944C001D
:108AD000002664085900944649080246029622433B
:108AE00021D062460A431ED06200570D4A000E0391
:108AF0002303550D012402462C492405781B1B0B2A
:108B0000360B401823432643614600901C46501AFA
:108B1000B44103D30098401C009002E092180098E2
:108B20005B41002803DA0020014605B0F0BD0020BB
:108B3000012109050746864611E064461D46141BBF
:108B4000B54106D36546521BB341744607430C43F7
:108B5000A646CD0740084908284392185B410546C0
:108B60000D43EAD11046184313D0604619465040D1
:108B70007140084306D06046101AB34106D2012264
:108B8000002306E000220123DB0702E00122D2439A
:108B90005310009874460105381C6141029C039DE6
:108BA0000019694100F0A7FABFE70000FD030000CB
:108BB00070B54B005B0803430BD04B005C0D0026E7
:108BC00033466542B341D417AD1AA34102DB0020FE
:108BD000014670BD12053018514170BD10B500221C
:108BE0009623114600F04EFA10BD00000EB5C217D4
:108BF000C10F5040CA0740180021054B0293019253
:108C000000910A460B4600F083FA03B000BD000055
:108C1000330400000EB505490291002100910A4677
:108C20000B46019100F074FA03B000BD330400005C
:108C30000EB5054A0292002200921346019200F0FE
:108C400067FA03B000BD000033040000C20F41000A
:108C500040020123400ADB05D207090EC0187F2914
:108C600001DA00207047962903DC9623591AC84080
:108C700001E096398840002AF4D040427047000055
:108C800070B5CD0F4A0009030123090B1B051943D9
:108C90000B4BED070024520D9A4201DA002070BD03
:108CA000074B34339A4203DC9A1A00F0D2F802E000
:108CB0000449511888402C43F1D0404270BD000057
:108CC000FF030000CDFBFFFF4A0009030123090B4E
:108CD0001B0519430A4B10B5520D9A4202DA0020C7
:108CE000014610BD064B34339A4203DC9A1A00F059
:108CF000B0F810BD034BD21800F09BF810BD000077
:108D0000FF030000CDFBFFFFC20FD2074000400869
:108D10000BD0C10D0723DB01C91840020905400A29
:108D20001143C208400711437047002001467047B5
:108D300010B5002904DB0124E40740428C412146A0
:108D4000002B04DB1C460123DB075242A3418B426C
:108D500000D1824210BD000010B5002904DB0124BF
:108D6000E40740428C412146002B04DB1C460123D2
:108D7000DB075242A341994200D1904210BD00004E
:108D8000CB0FDB07490010B5490802460A4307D05C
:108D90000A0D07240903E401090B121B002A01DC58
:108DA000002010BDC900440F0C43C100E018D205DB
:108DB000801800F05FF910BDF0B51FB486B0002038
:108DC0000090019002900698069980B2049007984E
:108DD000090C02040014114307900027089D09980C
:108DE00006913E463C4603900398A9B20204000C4B
:108DF000039004982D0C154348430021224600F0AF
:108E000018F8C719714110340E46402CECDB384677
:108E1000029A00F00EF8009A019B801800905941C8
:108E200002980191103002904028CCDB00980BB0E2
:108E3000F0BD10B5202A04DB0146203A9140002005
:108E400010BD914020239C1A0346E34019439040F3
:108E500010BD10B5202A04DB0846203AD04000217E
:108E600010BD0B46D340D0402024A21A91400843A5
:108E7000194610BD10B5202A06DBCB170846203A4C
:108E80001041C1170B4306E00B461341D04020248C
:108E9000A21A91400843194610BD000000487047CF
:108EA000844F010110B50446FFF7F8FF0068005D2C
:108EB000C007C00F10BD0000026813785118016090
:108EC0001846704710B5D1600449516104491162D8
:108ED00000211161114600F08FF910BDB98E00011B
:108EE000A58E00014268002A08D001680B78491C51
:108EF000002B03D0521E06C0184670470121C160E6
:108F0000881E70474268002A0BD0C3680168002B96
:108F100007D183688B4204D0491E521C06C0002032
:108F200070470020C0437047F7B582B0029C00270D
:108F30002078641C15460197302802D0002D15D0EA
:108F400015E020780127641C782804D0582802D026
:108F5000002D09D00BE0002D01D0102D07D10027E6
:108F600010252078641C02E0082500E00A25002670
:108F7000009610E00099012769430818020C294661
:108F800080B2714300908E183804864201D30120CC
:108F900001902078641C294600F01EF90028E9DAC7
:108FA0000398002805D0002F01D0641E00E0029C29
:108FB00004600198002806D002F004FD022101603F
:108FC000C81E05B0F0BD009930040843F9E7000061
:108FD0000FB400B589B00CA900910B990023CB60A8
:108FE000204B214A06930792042201921F4A0292C3
:108FF0001F4A089202466B460020FFF74AFA09B062
:1090000008BC04B0184770B586B006460020C043BF
:109010000190002015460C460091029104903246C2
:10902000694604A8FFF7D4FF024604982118002DD2
:1090300005D0002801D0084600E0204628600498AA
:1090400000280DD0002A02DD0098884208D0081BB5
:109050000190009432466946029404A8FFF7B8FFD5
:1090600006B070BDE58E0001058F0001FFFFFF7F98
:10907000A58E0001002904DA401C490001D14008F6
:109080004000704770B40024050C05D11024000482
:1090900002D1002921D01124050E01D1000208348B
:1090A000050F01D10001241D850F01D18000A41CF2
:1090B000002801DB4000641C002908D020252E1B5D
:1090C0000D46F540A14000D0012129430843010687
:1090D0001B1B000ADB1D02D5002070BC7047DB059E
:1090E000181880180029F8DA401C4900F5D170BC26
:1090F00040084000704710B5002B08DA0024401CDF
:10910000614192185B411A4301D14008400010BDF3
:10911000F0B51FB482B005460C0003D0084602F03B
:1091200039FC02E002F036FC203002460090214675
:109130002846FFF77EFE049B059A04460F46184317
:109140001143084314D0184610431BD00098402107
:109150000A1A18460599FFF77CFE05460E46009A46
:1091600005990498FFF765FE084305D0012004E047
:109170002046394607B0F0BD0020C11705430E4315
:109180002C43374300990E986305401A7905E40A89
:1091900000220C43FD0A0A3002D500200146E9E70F
:1091A0000105101969410C9C0D9D00196941FFF7DB
:1091B000A2FFDFE7064C0125064E05E0E36807CC79
:1091C0002B430C3C98471034B442F7D3FEF77CFF96
:1091D000EC5401010C5501013A2800D2303820230B
:1091E00002469A43412A01D310463738884201D3B8
:1091F0000020C04370470000F3B58DB000200A90F6
:1092000001200B90002608460C300C46099062693C
:10921000012109989047051E2ED0252D2DD0216AB9
:109220008847002818D06269012109989047216A6F
:1092300088470028F7D1411E62690998904700E0ED
:10924000761CA1690D988847216A88470028F7D1C4
:10925000E1690D988847DAE7A1690D9888470746C4
:10926000A84201D1761CD2E7E1690D9888477F1C9E
:1092700002D10A98002877D049E1002762693D466B
:109280003946099890472A280CD16269012109982A
:109290009047012506E00A214F433F18303FEBD4A9
:1092A0001020054362690121099890470146303931
:1092B0000A2903D29B498F42DEDCECE7E90600D4A1
:1092C000994F6C280AD04C2810D0682824D06A28DE
:1092D0002ED074280CD07A280AD00DE062690121C2
:1092E000099890476C2823D004211CE020200543D6
:1092F0006269012109989047A760656065284FD091
:1093000026DC582839D01ADC452849D012DC25281B
:1093100034D04128B0D143E06269012109989047D7
:10932000682802D008210D43E6E70120C002DEE7ED
:109330000220DCE7462833D047282CD130E05B28D8
:1093400070D061282CD063286CD0642823D161E0D0
:109350006F284FD009DC662822D0672820D06928E2
:1093600026D06E2817D12EE0CDE070284DD073287E
:109370006FD075284ED078280DD154E0A1690D9892
:1093800088470546252800D16CE7E1690D98884794
:109390006D1C00D16DE7BAE00A224CE00A2252E0CF
:1093A000012023466A46C0430D99FFF772F8A3E0F7
:1093B0002846402108436060A807234601D50022C3
:1093C00039E000223FE0E80700D020E72068011DD7
:1093D00021600068290501D5067018E7290701D525
:1093E000068014E7A90703D5F117066041600EE770
:1093F00006600CE72846402108436060A807234622
:1094000001D5082217E008221DE0484928460840F7
:10941000606016E02846402108436060A8072346A4
:10942000BCD5B9E715E02846402108436060A8078D
:1094300007D5234610220120C0430D99C046C046DF
:109440005AE0234610220120C0430D99C046C04671
:1094500052E000210C910B460091632802D05B285A
:1094600007D043E0E80601D40120A060012000906D
:109470003CE062690121099890475E2805D10120EE
:109480000C9001466269099890472169002906D12C
:109490000B4601AA8F00491CD3510829FADB00288A
:1094A00035D0216900290ED1C117C90E09184A11FA
:1094B000930001AA9A1849094901411A0120136829
:1094C00088400343136062690121099890475D2831
:1094D000E5D10C98002808D0002001AB81005A5833
:1094E000401CD2435A500828F8DB01AB0120224629
:1094F000C0430D99C046C04600280ADA401C06D178
:109500000B98002803D00020C0430FB0F0BD0A988C
:10951000FBE7E90702D10A99491C0A913618002095
:109520000B9074E6CCCCCC0CFFFFFF7FF1F7FFFF74
:1095300070B58C180578401C6B075B0F01D1037860
:10954000401C2A1106D10278401C03E006780E70F8
:10955000401C491C5B1EF9D12B0705D40023521E69
:109560000DD40B70491CFAE70378401CCB1A921CEF
:1095700003E01D780D70491C5B1C521EF9D5A142F9
:10958000D8D3002070BD000003B40148019001BD94
:10959000232A000003B40148019001BD6D5600006C
:1095A00003B40148019001BD6560000003B40148A7
:1095B000019001BDAF7F000003B40148019001BDDF
:1095C000B551000003B40148019001BDD37E0000F5
:1095D00003B40148019001BD697E000003B4014855
:1095E000019001BDC37F000003B40148019001BD9B
:1095F000E954000003B40148019001BD99570000EF
:1096000003B40148019001BDED57000003B40148C7
:10961000019001BD1D7C000003B40148019001BD13
:109620000D2A000003B40148019001BDAB520000B7
:1096300003B40148019001BDF58F000003B4014857
:10964000019001BDE1FE000003B40148019001BD9D
:10965000250E010003B40148019001BDB143000093
:1096600003B40148019001BD85290000C943416050
:1096700070470268702392B29A430A4302607047AF
:1096800070B5044602F08CF8002818D080690028D4
:1096900015D0FFF7A3FA05462046FFF79FFA2946A3
:1096A000FFF7B2F8FFF730FB064A074BFFF708FA5F
:1096B0000022064BFFF7EAF8FFF762FB70BD044D8E
:1096C000EAE700001F85EB51B81E01400000394059
:1096D00000803B4470B50D460646002402F060F859
:1096E000002816D0C169002913D0026A002A10D0C0
:1096F0008BB290B289B292B2102D0CD0202D0AD02C
:10970000302D17D0402D15D0502D13D0602D11D0F5
:1097100022E0002070BD891AB01AAF229200504397
:10972000FEF746FD044696340FD47D20C0008442E7
:1097300011DC11E0191AAF22301A12015043FEF762
:1097400037FD4B21C900441801D5002404E0E12075
:109750000001844200DD0446204670BD70B5104C07
:10976000A0421BD185140121284601F0A7FE00214B
:10977000284601F0A3FE0121284601F093FE094886
:1097800060610020206060601F21A16006492161A6
:10979000A06160622062A0620448E06170BD0000C8
:1097A00000080240080A02000000FC0F2E6D0000B5
:1097B0000029016802D00122114301E04908490053
:1097C0000160704704220029816902D01143816140
:1097D00070479143816108480649C16207490163A6
:1097E00007494163074981630749C163084907483D
:1097F000086070472200780000080240E700E1009E
:109800009F00BF04190C051670206E286E2B0000F7
:109810004008024002220029016801D0114300E003
:10982000914301607047C06880B270470246526839
:1098300000200A4200D0012070470000044A9068CE
:10984000C90640094001C90E0143916070470000FC
:109850000008024070B5054649480C464EC88CB019
:1098600003960293019200914EC8079606930592C3
:109870000491426801688068099208910A90414AFF
:1098800000996846914217D1282104F079FB0A9982
:10989000884211D1022D1ADB0020646802460B9029
:1098A0000BA92046FEF720FF05460B98A04209D0E1
:1098B0000078002806D101E033A004E0012D0AD091
:1098C000022D08D03EA004F059FC0CB070BD0198E8
:1098D000012809D001250198A84207D1294647A0AF
:1098E00004F0E6FB0CB070BD0225F4E7012D6C46D8
:1098F00014D01834012D13D047482268824206D173
:109900006068002803D00721890388420AD92946C4
:1099100042A0636804F0CCFB0CB070BD0834E9E7EA
:109920004C48EAE74CA004F029FC6168206804F088
:1099300027FBA268824206D003462946544804F019
:10994000B7FB54A0BFE729465FA06368E26804F054
:10995000AFFB6846019503F0B5FE002801D06AA070
:10996000B1E76EA004F00AFCC82009F07FFDBFF348
:109970004F8F72497048C860BFF34F8FFEE70000F9
:109980000040000111C011CA61707073773A206203
:109990006F6F7473657474696E67207265636F723C
:1099A0006420696E76616C69642C207265667573DB
:1099B0006520746F207377697463680D0A00000076
:1099C00075736167653A206170707377205B317CD5
:1099D000325D20286E6F20617267203D20737769A9
:1099E00074636820746F20746865206F7468657292
:1099F0002062616E6B290D0A0000000061707073B7
:109A0000773A20616C7265616479206F6E204150F5
:109A100050256C750D0A00000040020161707073E2
:109A2000773A2062616E6B256C75207265636F7288
:109A30006420696E76616C69642028616464723D9B
:109A400030782530386C582073697A653D256C75FF
:109A5000290D0A000080000161707073773A20764A
:109A60006572696679696E672074617267657420D2
:109A7000696D61676520637263202866657720736E
:109A800065636F6E6473292E2E2E0D0A0000000090
:109A9000585401012020202020202072756E204281
:109AA0004C45204F544120746F20777269746520B3
:109AB000612076616C696420696D61676520666903
:109AC0007273740D0A00000061707073773A20623F
:109AD000616E6B256C7520696D616765206F6B2009
:109AE000287665722030782530386C582C20256C0B
:109AF000752042292C20737769746368696E672E1C
:109B00002E2E0D0A0000000061707073773A2066F7
:109B10006C617368206661696C0D0A006170707316
:109B2000773A20646F6E652C207265736574746972
:109B30006E672E2E2E0D0A000400FA0500ED00E0DF
:109B400010B50B488CB01EC803940293019200918B
:109B50001EC80794069305920491426801688068C4
:109B60000A9009920891684603F0DAFD0CB010BD26
:109B700000400001F0B58DB00E46032807DA54A06E
:109B800004F0FCFA5AA004F0F9FA5F480FE0002450
:109B9000B76822460BA938460B94FEF7A5FD05468B
:109BA0000B98B84202D00078002804D057A004F0E7
:109BB000E5FA0DB0F0BD5A4B87CB039702920191A5
:109BC000009087CB07970692059104909A68596890
:109BD00018680A920991534A009908906846914280
:109BE00005D1282104F0CCF90A9988420DD00094BF
:109BF00001940294039404940594069407940894A1
:109C0000099449A00A9404F0B9FA55A17068FEF7C6
:109C100056FB002804D070680178622908D02BE038
:109C2000012D03D0022D01D04FA0C0E701953AE0ED
:109C30004178312902D0322902D01DE002AC00E087
:109C400006AC51A1801CFEF73AFB002816D07068C4
:109C50004FA1801CFEF733FB002819D070684EA17D
:109C6000801CFEF72CFB00281AD070684BA1801CCA
:109C7000FEF725FB002815D049A098E74E488542FD
:109C800004D04E48854201D04DA090E725600AE0FF
:109C900007208003854201D958A088E7656002E06B
:109CA000A56000E0E5602A465DA0716804F000FA56
:109CB000684603F007FD002801D062A077E766A0A0
:109CC00004F05CFA684603F02BFD0DB0F0BD000017
:109CD00075736167653A206273736574203C6669C9
:109CE000656C643E203C76616C3E0D0A000000000D
:109CF00020206669656C643A20616374697665202A
:109D00003C317C323E0D0A00A05401016273736540
:109D1000743A206261642076616C75650D0A0000FA
:109D20000040000111C011CA62737365743A206566
:109D300078697374696E67207265636F72642069F5
:109D40006E76616C69642C2072656275696C642042
:109D500066726F6D20736372617463680D0A000030
:109D6000616374697665000062737365743A20619B
:109D70006374697665206D75737420626520312087
:109D80006F7220320D0A00006164647200000000EE
:109D900073697A6500000000637263007665720083
:109DA00062737365743A20756E6B6E6F776E2066A2
:109DB00069656C640D0A000000800001004002012A
:109DC00062737365743A2061646472206D75737494
:109DD0002062652043414949435F415050315F4211
:109DE000415345206F722043414949435F415050E0
:109DF000325F424153450D0A0000000062737365F3
:109E0000743A2073697A65206578636565647320A8
:109E10007468652062616E6B2073697A650D0A0053
:109E200062737365743A202573203D2030782530A5
:109E3000386C582C2077726974696E672E2E2E0D3F
:109E40000A00000062737365743A20666C6173687F
:109E5000206661696C0D0A0062737365743A206F45
:109E60006B20287665726966696564290D0A0000B1
:109E700000B583B0002103200B4601220191009020
:109E8000920203A1034809F059FF03B000BD00008E
:109E9000434C49009DA2000110B5022805DB48682B
:109EA0000DA1FEF70CFA002805D00D480078002817
:109EB00004D00CA103E007F0E3FA10BD0BA110A041
:109EC00004F0F6F8124C13A0218904F0F1F81CA05C
:109ED000E16804F0EDF810BD6A736F6E00000000D9
:109EE000A847002076616C696400000064656661C3
:109EF000756C7420286E6F74207361766564290018
:109F0000706172616D733A2025730D0A00000000C4
:109F1000C46A002020206C6564203D202575202027
:109F2000286C65643120626C696E6B2068616C66B8
:109F300020706572696F642C206D73290D0A000012
:109F4000202070776D203D20256C752020287077AB
:109F50006D20647574792C202525290D0A000000D8
:109F6000F3B595B015980D46032807DA6F4804F04D
:109F700005F96FA004F002F979A023E07FA16868D9
:109F8000FEF79DF9002810D00020AE680246009030
:109F900069463046FEF7A8FB04460098B04202D05E
:109FA000007800287BD077A00CE000240226B000C7
:109FB00014902858FEF77CF90746E019801C5028B9
:109FC00004D975A004F0DAF817B0F0BD002C03D066
:109FD000202069460855641C14983A46295868465A
:109FE0000019FEF741F91598E419761C8642DEDB6C
:109FF000002069460855451E6E462C4605F0E8FDD2
:10A00000304603F013FF060023D003F0F4FE0028CF
:10A010001FD069A1304603F0B7FE074603F0E2FE09
:10A02000002800D07D6965A1304603F0ADFE0746EB
:10A0300003F0D8FE002800D07C69002D13DA002C34
:10A0400022DA5FA004F09AF8304603F073FE17B0EE
:10A05000F0BD65A004F092F8002EF8D0304603F071
:10A0600069FE17B0F0BD294666483239814209D3EE
:10A07000654A322165A004F01BF8304603F05AFE11
:10A0800017B0F0BD002C0BDB642C09DD642164A04B
:10A0900004F00EF8304603F04DFE17B0F0BD14E0AA
:10A0A000304603F047FE002D01DB62480581002C9D
:10A0B00001DB6048C46007F037FA002801D05EA0D9
:10A0C00080E707F0DDF917B0F0BD3BA16868FEF747
:10A0D000F6F8002807D039A16868FEF7F0F80028E4
:10A0E0000DD05CA06EE7204646493238884203D343
:10A0F000454A322145A015E04E48048109E0642C10
:10A1000005D9642146A003F0D3FF17B0F0BD49483C
:10A11000C46007F009FA002801D055A052E7224692
:10A1200059A0696803F0C4FF17B0F0BD14540101D1
:10A1300020206C6564203D206C65643120626C6970
:10A140006E6B2068616C6620706572696F64203583
:10A15000302E2E3130303030206D730D0A0000006B
:10A16000202070776D203D2070776D2064757479A4
:10A1700020302E2E31303020250D0A006A736F6E8C
:10A18000000000006170707365743A2062616420A1
:10A1900076616C75650D0A00617070736574206A74
:10A1A000736F6E3A206C696E6520746F6F206C6FF0
:10A1B0006E670D0A000000006C65640070776D002A
:10A1C000617070736574206A736F6E3A206E6F20D1
:10A1D0006B6E6F776E206B657920286C65642C2020
:10A1E00070776D290D0A0000617070736574206AC4
:10A1F000736F6E3A207061727365206661696C0DD1
:10A200000A000000DF260000102700006C656420B3
:10A2100072616E67652025752E2E25750D0A00006A
:10A2200070776D2072616E676520302E2E25750D5A
:10A230000A000000C46A0020617070736574206AAF
:10A24000736F6E3A20666C617368206661696C0D8D
:10A250000A000000756E6B6E6F776E207061726120
:10A260006D20286C65642C2070776D290D0A000024
:10A270006170707365743A20666C61736820666102
:10A28000696C0D0A000000002573203D20256C75C7
:10A290002C2073617665640D0A000000002498B0DC
:10A2A000F9A527461594661E28461294FEF700F875
:10A2B00081B2284603F07CFC03F0E8F8FE48002554
:10A2C000807800283BD003F0E1F86421684603F071
:10A2D00059FB002816D06846007802F09DFE002841
:10A2E0000ED0F5490020887003F040FCF3A5284605
:10A2F000FDF7DEFF81B2284603F05AFC03F046FC6E
:10A30000002518E0643502F0D7FDF648854212D3E7
:10A31000E9490020887002F0CFFD02F0C1FD03F092
:10A3200025FCF1A00190FDF7C3FF81B2019803F075
:10A330003FFC03F02BFCE04880780028C3D10021CB
:10A34000C943684603F01EFB0028B5D015980028C5
:10A3500005D000211591694609788142ACD0129848
:10A3600001281FD0022826D0684600781B287DD0FF
:10A3700009287CD00D287BD00A287AD0082879D0EB
:10A380007F2877D0014620395F2995D23F2C72D2A1
:10A39000E0490855641CA4B20121684603F008FC9A
:10A3A000274689E7684600785B2802D00020129093
:10A3B00082E70220FBE700201290684600784128DF
:10A3C00016D04228EDD1002EEBDB761E57D4BA48CA
:10A3D0004078801BC01DC117490F0918C908C90062
:10A3E000401A8101CC4809184038FDF78DFF49E03B
:10A3F000B148711C02789142D3DA4078761C801BF8
:10A40000C01DC117490F0918C908C900401A8101A8
:10A41000C14809184038FDF777FFBE480290FDF7A4
:10A4200047FF85B2BDA42046FDF742FF81B220461A
:10A4300003F0BEFB0024002F0BD9BBA00190FDF759
:10A4400037FF81B2019803F0B3FB641CA4B2BC4295
:10A45000F3D3B2A42046FDF72BFF81B2204603F0D0
:10A46000A7FB002D34D02946029805E036E038E0FD
:10A47000E2E0E3E081E18EE103F09AFB28E0A54908
:10A4800000200870A3480290FDF712FF85B2A3A434
:10A490002046FDF70DFF81B2204603F089FB002422
:10A4A000002F0BD9A0A00190FDF702FF81B2019807
:10A4B00003F07EFB641CA4B2BC42F3D397A42046F5
:10A4C000FDF7F6FE81B2204603F072FB002DCAD1E3
:10A4D0002F469048FDF7ECFE84B2EDE60120129085
:10A4E000EAE603F043FB8B4800252F46019003F07A
:10A4F00076FD1390224620210198FDF7EEFE0028FC
:10A5000060D1019908551399149000295AD91498CB
:10A5100003F068FD224616900199FDF7FEFE002823
:10A5200019D1002F0AD102A81699FDF7EDFE02A855
:10A53000FDF7BEFE85B20DE06D1EADB2A54206D997
:10A540002A4602A81699FDF7E8FE0028F4D100215A
:10A5500002A841557F1C14981399401C14908842FE
:10A56000D5D3002F64D0012F1AD0A5422BD902AF2A
:10A570003F2C5DD2AC425BD23819012103F018FBAD
:10A580000198395D0155641CA4B2F1E73819012125
:10A5900003F00EFB0198395D0155641CA4B200E084
:10A5A00002AF3F2C44D2AC42F0D301992020085591
:10A5B000641C5DA5A4B22846FDF77AFE81B2284648
:10A5C00003F0F6FA34E059A52846FDF771FE81B292
:10A5D000284603F0EDFA1398002500281CD92846D8
:10A5E00003F000FD074622460199FDF796FE00287C
:10A5F0000ED13846FDF75CFE81B2384603F0D8FA3A
:10A600004BA73846FDF754FE81B2384603F0D0FA26
:10A6100013986D1C8542E2D344A52846FDF748FEF9
:10A6200081B2284603F0C4FA2146019803F056FD92
:10A63000274603F0ABFA3FE60A2000E00D20159014
:10A6400003F094FA39A52846FDF732FE81B2284678
:10A6500003F0AEFA2F49002008550D46287800284F
:10A6600077D0154C207800280AD06078C01D4007AC
:10A67000C10D294808182946FDF721FE002868D099
:10A6800060788101244856E00D0A434C49207265E8
:10A690006164792E2054797065202768656C702775
:10A6A00020666F7220636F6D6D616E64732E0D0A8C
:10A6B00063616969632D3E00504700200D0A5B6F9E
:10A6C00074615D2061626F727465642C20626163E5
:10A6D0006B20746F20434C490D0A63616969632DD7
:10A6E0003E000000102700000D0A5B6F74615D20C2
:10A6F00069646C652074696D656F75742C20626186
:10A70000636B20746F20434C490D0A636169696370
:10A710002D3E0000E05C0020205D00200D6361699B
:10A7200069632D3E00000000200000000D0A0000BB
:10A73000202000000DE008182946FDF7E5FD6078AF
:10A74000401C4007400F60702078082801D2401C50
:10A750002070002003F00CFD134803F04FFC13A4FD
:10A760002046FDF7A5FD81B2204603F021FA03F053
:10A770000DFA00242746661E9EE5002CFCD0641EC0
:10A780000CA5A4B22846FDF793FD81B2284603F03C
:10A790000FFA274690E508A52846FDF789FD81B206
:10A7A000284603F005FA87E5E05C002063616969EB
:10A7B000632D3E00082008000700000010B50C467D
:10A7C000022812DB0EA16068FDF779FD002809D090
:10A7D0000CA16068FDF773FD002804D00AA003F007
:10A7E000CDFC10BD012001F0D9FF01F0D1FF002800
:10A7F00001D003A100E003A10AA003F059FC10BDA1
:10A800006F6E00006F66660075736167653A20625F
:10A810006C656C6F67205B6F6E7C6F66665D0D0AA2
:10A8200000000000626C65206C6F673A2025730D94
:10A830000A000000F8B502F043FA074602F03CFABD
:10A840000546254A25A128A003F032FC02F066FA4D
:10A8500001462CA003F02CFC2F48874203D12FA0E7
:10A8600003F08CFC15E000F09BFF044602F088FA30
:10A8700006460A213846FDF79BFC0A460146002C95
:10A8800001D0A06900E00020009033462BA003F027
:10A890000FFC02F091FA014632A003F009FC3548A2
:10A8A000854203D134A003F069FC03E029463AA0B5
:10A8B00003F0FEFB09F00EFB7D21C900FDF762FCF1
:10A8C000014639A003F0F4FB08F00CFF01463AA062
:10A8D00003F0EEFBF8BD00001C00010056312E30E5
:10A8E000302E3238000000006669726D7761726543
:10A8F0003A202573202830782530386C58290D0AE5
:10A90000000000006375722062616E6B3A20415056
:10A910005025750D0A000000FF7F00006368697014
:10A920002074656D703A2041444320726561642053
:10A9300074696D656F75740D0A0000006368697055
:10A940002074656D703A2025642E256420432028EC
:10A950006164633D2575207472696D3D256C7529B0
:10A960000D0A00007664643A202575206D560D0AA4
:10A9700000000000FFFF000066616E2072706D3AFB
:10A98000206E2F6120286E6F20746163686F6D6583
:10A99000746572290D0A000066616E2072706D3A4E
:10A9A0002025750D0A000000757074696D653A20E8
:10A9B000256C7520730D0A006672656520686561F7
:10A9C000703A20257520420D0A00000002F03AFC82
:10A9D00000280DD007A003F0D1FBC82008F046FDE9
:10A9E000BFF34F8F11491048C860BFF34F8FFEE788
:10A9F0000FA0F0E7666163746F72793A20666C614C
:10AA00007368207772697465206661696C65642C6F
:10AA100020726573657474696E6720616E79776101
:10AA2000792E2E2E0D0A00000400FA0500ED00E03C
:10AA3000666163746F72792064656661756C7473A6
:10AA400020726573746F7265642C2072657365740F
:10AA500074696E672E2E2E0D0A00000003A003F00D
:10AA60008DFBC82008F002FDFEE7000068616E67FC
:10AA7000696E67206E6F77202D207761746368643C
:10AA80006F672073686F756C6420726573657420DE
:10AA9000696E207E3473202E2E2E0D0A00000000D9
:10AAA00070B5194D0E46022819DB00240C206043B6
:10AAB00029587068FDF703FC002807D0641C112C8E
:10AAC000F4D312A0716803F0F3FA70BD0C20444374
:10AAD00060194268295916A003F0EAFA70BD17A060
:10AAE00003F04CFB002420460C21484341194A68DE
:10AAF00029580FA003F0DCFA641C112CF3D312A028
:10AB000003F03CFB70BD0000304E0101756E6B6EB2
:10AB10006F776E20636F6D6D616E643A20257320D0
:10AB200028747279202768656C7027290D0A000047
:10AB30002020252D38732025730D0A00636F6D6D5D
:10AB4000616E64733A0D0A006B6579733A20544163
:10AB500042203D20636F6D706C6574652C205550EC
:10AB60002F444F574E203D20686973746F72790DE2
:10AB70000A00000070B50C46032823DB60680178EA
:10AB8000312902D0322906D01CE04078002819D1A2
:10AB9000184E012504E04078002813D1164E4025B8
:10ABA00016A1A068FDF78BFB00280FD014A1A068A8
:10ABB000FDF785FB00280ED012A1A068FDF77FFBF2
:10ABC00000280DD011A003F0D9FA70BD29463046F7
:10ABD00000F06CFB08E02946304600F063FB03E020
:10ABE0002946304600F034FB11A0A268616803F0EA
:10ABF0005FFA70BD000C0140000801406F6E00005C
:10AC00006F666600746F67676C65000075736167D7
:10AC1000653A206C6564203C317C323E203C6F6E8E
:10AC20007C6F66667C746F67676C653E0D0A00001A
:10AC30006C656420257320257320646F6E650D0A92
:10AC40000000000010B5034803F098FA01F010FF6F
:10AC500010BD0000D84F010106A003F08FFAC820F4
:10AC600008F004FCBFF34F8F07490648C860BFF3E4
:10AC70004F8FFEE7726573657474696E672E2E2EB2
:10AC80000D0A00000400FA0500ED00E010B509F01F
:10AC900021F97D210446C900FDF774FA02462146D8
:10ACA00010A003F005FA08F003FB014614A003F01E
:10ACB000FFF908F01DFD044608F014FD02460921C5
:10ACC0002346C90211A003F0F3F91DA003F056FAC0
:10ACD000274900200870084608F0E8FB244803F0E4
:10ACE0004DFA10BD757074696D653A20256C75203C
:10ACF0007469636B732028256C752073290D0A0015
:10AD00007461736B733A2025750D0A006865617074
:10AD10003A20746F74616C20257520422C20667275
:10AD2000656520257520422C206D696E206576654D
:10AD300072206672656520257520420D0A000000AC
:10AD40006E616D65202020202020202020202020E2
:10AD500020737461746520207072696F2020737491
:10AD600061636B28772920206E756D0D0A00000045
:10AD7000005B002010B506A003F000FAE121C90233
:10AD80000BA003F095F9164803F0F8F910BD000088
:10AD90007573617274313A2054583D5042362052D6
:10ADA000583D5042372028414634290D0A00000002
:10ADB000626175643A20256C752C203820646174BA
:10ADC0006120626974732C206E6F207061726974E7
:10ADD000792C20312073746F70206269740D0A0021
:10ADE000884F010110B5E124E402204602F084FE00
:10ADF000214602A003F05CF910BD0000757361727A
:10AE0000742072657365743A20256C7520384E3154
:10AE10002C20727820717565756520666C75736875
:10AE200065640D0A0000000010B506A108A003F03B
:10AE30003FF90DA003F0A2F91948016819A003F029
:10AE400037F910BD56312E30302E32380000000058
:10AE50006669726D776172652076657273696F6E6F
:10AE60003A2025730D0A00006D636D2D6464632D17
:10AE7000626C653A20424C452872647473732920D1
:10AE80002B204672656552544F53202B205541525A
:10AE90005428444D4129202B20434C490D0A0000E1
:10AEA0000040002053797374656D436F7265436C85
:10AEB0006F636B203D20256C7520487A0D0A0000D9
:10AEC000044A0029516801D0014300E081435160E8
:10AED00070470000401002404860704701681A4AFD
:10AEE000114001600021016041608160C160174A2A
:10AEF0001749904204D148680F22104348607047B8
:10AF0000144A904204D14868F022104348607047C8
:10AF1000114A904205D148680F221202104348603E
:10AF200070470E4A904205D148680F221203104321
:10AF3000486070470A4A9042FBD148680F221204C9
:10AF40001043486070470000FEFF00000800024008
:10AF5000000002401C000240300002404400024059
:10AF6000580002400029016802D00122114301E08B
:10AF7000014A114001607047FEFF0000406880B246
:10AF80007047024609680020114200D00120704736
:10AF900030B403680D4A0C6A13408A684D69224335
:10AFA0000C692C4322438C692243CC6922434C6AAE
:10AFB00022438C6A22431A430260CA6842600A68CC
:10AFC00082604968C16030BC704700000F80FFFF9D
:10AFD000002B01D010617047002010617047000005
:10AFE000014948617047000000040140054B002200
:10AFF00019685B690140034202D0002900D0012298
:10B00000104670470004014010B483791949026862
:10B01000002B28D00B6893430B604A6803689A435F
:10B020004A600279521813680468234313608A68DF
:10B0300003689A438A60CA6803689A43CA6042797F
:10B04000102A06D051180A68006802430A6010BC32
:10B0500070478A6803681A438A60CA6800680243B6
:10B06000CA6010BC704700794018016891430160C4
:10B0700010BC7047000401400B680022002B56D022
:10B08000F0B401240B68944023424AD04B68022B51
:10B0900001D0122B16D113070AD5456A5307DB0ED0
:10B0A0000F269E40B5434E699E402E43466209E0FE
:10B0B000056A5307DB0E0F269E40B5434E699E403E
:10B0C0002E4306624B68012B05D0112B03D0022BB7
:10B0D00001D0122B06D14568DB06DB0FA543934058
:10B0E0002B4343600568530003279F400E79BD43FF
:10B0F000B607B60F9E402E430660C5688E68BD43F6
:10B100009E402E43C66085680126A543CC689440C6
:10B110002C438460C46A9E400D69B4439D4025431E
:10B12000C5620B68521CD340ABD1F0BC704770476E
:10B1300005490160002242600F21826041610121C6
:10B140000261C16070470000FF3F000081627047EC
:10B150008161704742694A404261704782B0EFF3B3
:10B160000884FCF7C3FF400701D5EFF309840AA068
:10B1700000F0D6FBE06800900CA0A368626821682C
:10B1800000F0CEFBE069009014A0A3696269216918
:10B1900000F0C6FBFEE700000A2A2A2A2048617256
:10B1A000644661756C74202A2A2A0A0052302020D5
:10B1B0003D2530386C5820523120203D2530386CE8
:10B1C0005820523220203D2530386C5820523320F0
:10B1D000203D2530386C580A0000000052313220E2
:10B1E0003D2530386C58204C5220203D2530386C9D
:10B1F0005820504320203D2530386C58207850533B
:10B20000523D2530386C580A000000000149886022
:10B210007047000000300040024901480860704754
:10B22000CCCC000000300040024901480860704763
:10B23000AAAA0000003000400149486070470000A1
:10B2400000300040014908607047000000300040B5
:10B2500010B5FFF77FFF10BD30B505460E4887B02B
:10B260000C46854202D10121042004E00B488542AE
:10B2700010D10121082000F039F90948844209D889
:10B280006846FFF755FF0120019069460094284663
:10B29000FFF7F2FE07B030BD00080140000C01408E
:10B2A000FF3F000010B5FFF751FF10BD10B5FFF7CD
:10B2B0004FFF10BD10B400214156FF23CAB29207C0
:10B2C000D40E4278A3409207120EA24000290BDA56
:10B2D0000907090F08398C081049A4006118CC69C6
:10B2E0009C431443CC6107E08C080D49A40061180D
:10B2F0000C689C4314430C60827801210078002A7A
:10B3000004D0C006C00E8140064803E0C006C00E4F
:10B3100081400548016010BC7047000000ED00E06E
:10B3200000E400E000E100E080E100E0F7B5FFB0FC
:10B3300004460025A5B00520EFF31087FF210090FB
:10B34000453102A8FCF7A9FFEFF31086FF21453134
:10B3500053A8FCF7A2FF53A801300190982222497C
:10B3600053A8FCF781FF012080F3108801988047E3
:10B3700086F3108801221D49120303265300360369
:10B3800088420AD194421AD09C4201D1151116E08C
:10B39000B44210D101256D0211E0154988420AD14D
:10B3A000944201D115460AE09C4201D11D4606E0B7
:10B3B0003546AC4203D000987FB028B0F0BD06AC53
:10B3C000FF22013441320B4902A8FCF74DFF012056
:10B3D00080F310882846A69AA599A04787F310887D
:10B3E0007FB028B0F0BD000000430101C44013004D
:10B3F00085601300C041010110B5EFF310840121F5
:10B4000081F31088FF21090640180349096888471D
:10B4100084F3108810BD00000440002010B50848D7
:10B42000064901600749416007498160C9229200CD
:10B4300006490748FCF718FF10BD0000014900202D
:10B44000044000209549002069480020A4430101E0
:10B450006048002010B5EFF31084012383F31088B7
:10B46000FF231B06C018034B5B68984784F31088C2
:10B4700010BD0000044000200448416A012211432D
:10B480004162416A914341627047000000100240EE
:10B49000034AD16A102399430143D16270470000E7
:10B4A00000100240044A0029516901D0014300E024
:10B4B000814351617047000000100240044A002996
:10B4C000916A01D0014300E081439162704700001E
:10B4D00000100240044A0029D16901D0014300E074
:10B4E0008143D1617047000000100240044A0029E6
:10B4F000916901D0014300E08143916170470000F0
:10B50000001002400122054912060128086802D0F5
:10B510009043086070471043FBE7000000100240B2
:10B5200030B4164A516804231940154B01D0042940
:10B5300001D0036001E0134901605168124B890694
:10B54000890F5B5C0168D940416053680F4C5B0513
:10B550005B0FE35C0D46DD40856053689B045B0F29
:10B56000E35CD940C160D16AC90601D5084901E050
:10B570007D21C903016130BC70470000001002400A
:10B580000090D0030048E801984301019C43010169
:10B5900000093D0000224109094B01290BD0022975
:10B5A0000BD0596AC006C00E012383400B4200D065
:10B5B0000122104670471968F4E7196AF2E70000A3
:10B5C000001002407047000010B5FCF7A5FD0446CE
:10B5D00008F086FC002803D00120034900074860DA
:10B5E0002046FCF79DFD10BD00ED00E010B50A4CB3
:10B5F0002069411C01D000280AD1012006493422CB
:10B600000003FFF793FE2069411C03D0002801D0FE
:10B61000024810BD002010BD2C48002055480020D5
:10B62000F0B5564C85B0E06921040843E061812003
:10B63000534D0006286353486861534828625348B5
:10B64000032201689203914301605149342280141E
:10B65000FFF76CFE4E4B4F4E18694F4F411C29D0DF
:10B66000002827D0A9691A7849094901D206D20EC3
:10B670000A43AA612168EA139143216021687F226D
:10B68000120291430002084320606068304360600A
:10B690006068B84360606068211508436060206A94
:10B6A0003E4908402062206AD968090208432062A6
:10B6B00005B0F0BD61682046314361606168B943FF
:10B6C000616061680127BF02394361600021049114
:10B6D0007D21C9000391002100917F214024002594
:10B6E00002950191026861028A4302600E112349AA
:10B6F00008687F2212029043220202430A6005205A
:10B70000FCF7ECFC0120FCF7E9FC1C48406B8007CF
:10B7100004D4284603996D1C8842F3D91748C06B9E
:10B7200080B2B04201D9811B00E0311AB94202D285
:10B73000E2B28FB20292B04201D3019400E00094D1
:10B74000019A00988018C005000EA04203D004465C
:10B7500004988142CBD8094801687F2212029143A4
:10B76000029A12020A430260416849084900416096
:10B7700041684907FCD405B0F0BD0000001002404C
:10B78000007000400F080000180002000010014087
:10B790002C4800200000010000070000FF00F8FF17
:10B7A00010B50A4C2069411C01D000280AD10120A3
:10B7B000064934220003FFF7B9FD2069411C03D07C
:10B7C000002801D0014810BD002010BD2C480020E9
:10B7D00010B502F06DF910BD10B40B06CC065B0F6E
:10B7E000E40E0121A140012B07D0022B07D0143019
:10B7F000002A026805D00A4304E00C30F8E7103054
:10B80000F6E78A43026010BC704700000029818976
:10B8100003D001225203114301E0024A1140818109
:10B8200070470000FFDF0000002A828A01D00A432F
:10B8300000E08A43828270470246128800200A4252
:10B8400000D00120704770B40A06530FCE060125C0
:10B85000F60E2A460024B240012B0FD0022B10D046
:10B86000838A1340090A00888D402840002B02D0AB
:10B87000002800D00124204670BC70478389134003
:10B88000F0E7038AEDE7000070B50446008A86B051
:10B890000D461B490840E98801432182A0891949C6
:10B8A0002A890840A98811436A8902431143A1816A
:10B8B000A08A15490840A9890143A1826846FFF77B
:10B8C0002FFE1248844201D1039800E002982968B3
:10B8D000192289005043FCF755FC06466421FCF709
:10B8E00051FC0501280964214843301A0001323017
:10B8F000FCF748FC0007000F2843208106B070BD0C
:10B90000FFCF0000F3E90000FFFC00000038014019
:10B910008088C005C00D7047C905C90D818070477A
:10B920000FB410B503A9044B044A029800F066F95D
:10B9300010BC08BC04B0184771E60001C401002027
:10B940000FB410B504A9074B02AA039800F056F9EA
:10B95000044602A9002000F0F8FC204610BC08BCF8
:10B9600004B018474BC300017CB5154602460020C1
:10B970001C4600290BD0491E00920191044B6A46D7
:10B980002146284600F03AF9009A002111707CBD4A
:10B9900035C300012021020C01D010211046020AFB
:10B9A00001D010460839020901D01046091F82084B
:10B9B00001D01046891E420801D0881E7047081A1F
:10B9C00070470000004870472848002030B5002824
:10B9D00005D0164C021F20680023014605E00846EA
:10B9E00030BD904203D8034640680028F9D1002BAF
:10B9F00000D05968002B0AD01C68D51AA54204D182
:10BA00001268A4181A461C6002E05A6000E0226026
:10BA1000002807D01468851AA54203D10568641967
:10BA2000146040685060184630BD00002048002077
:10BA3000F1B50E4C0F480C4E001B0D4FC508ED0024
:10BA400000221146009804F0DBF8002803D130688A
:10BA5000002801D00020F8BD3C6000202560606017
:10BA600001203060ECE7000024480020ECB3002007
:10BA700020480020E8B50020F0B51FB486B0099832
:10BA8000089A030D0021024314D05148514A181856
:10BA9000504305141198012810981AD0281A401CF8
:10BAA00000264D4F4D49009601910490002812DA6E
:10BAB000444211E01198012449A3012801D11098B2
:10BAC000C1430698119A84600360C26041600BB064
:10BAD000F0BD4042E4E70446210500203F4A001C37
:10BAE00051410391029012E0E00707D032463B46F5
:10BAF00001990098FCF77CFF0191009032463B468B
:10BB000010461946FCF774FF06460F466410002CD9
:10BB1000EAD10498039B0028029A0999089806DA4A
:10BB2000FCF766FF019B009AFCF762FF05E0FCF75B
:10BB3000C7FF019B009AFCF7C3FF04460E46002294
:10BB4000284BFDF709F903D80020C043014607E060
:10BB50000022254B20463146FCF798FEFDF7B4F84D
:10BB6000102409E0002C0ADB0A220023FCF734FB36
:10BB7000079B30321A55641E02460A43F2D1112245
:10BB8000641C079B121B1C19119B012B03D0012362
:10BB900008430ED10AE0084304D011201090002081
:10BBA000119077E71098151A6D1E0BE010988242DD
:10BBB00002DD00236D1C03E0824201DA00236D1ECA
:10BBC000002BEED0069811998260C16030C07EE7EC
:10BBD00001FCFFFF104D0000000014400000F03F8A
:10BBE000300000000000F0430000E03F30380A2839
:10BBF00001D201207047002070470000FFB597B0C8
:10BC00000646002518E2252877D100242746FD495D
:10BC1000049400E00443761C32780120203A9040DE
:10BC20000842F7D130782A280ED002223078014617
:10BC30003039092916D804990A2359433039401854
:10BC40001443761C0490F1E7189802C804911890E8
:10BC5000002904DA012040030443484204900220F2
:10BC60000443761C30782E2814D1042004437078C5
:10BC7000761C2A2809D11898761C80C8189009E0EB
:10BC80000A214F43303FC719761C307801463039BE
:10BC90000929F5D930786C2810D006DC4C281AD048
:10BCA00068280ED06A2817D104E0742813D07A28A7
:10BCB00012D110E00120400504430CE001210905E8
:10BCC00001E0032109050C437178814203D1012071
:10BCD00000052418761C761C3078119066280BD04D
:10BCE00013DC58287DD009DC00287BD04528F6D00D
:10BCF0004628F4D047281AD1A5E118E0632835D0AA
:10BD0000642870D0652812D19DE170286CD008DCC1
:10BD10006728F1D069287BD06E280DD06F2806D116
:10BD2000BAE073282ED0752871D0782859D01A9A85
:10BD3000199990476D1C7EE16002400F022809D0DE
:10BD400003280DD00428189801680DD00D60001D3F
:10BD5000189070E11898EA1701680D604A60F6E7DC
:10BD6000189801680D80F2E70D70F0E718986A46A0
:10BD700001781172001D18900020507202A80090E6
:10BD8000012005E0189802C8189000200091C043D7
:10BD900061070DD5002101E00199491C0191B942CB
:10BDA00012DA8142F8DB009A515C0029F4D10BE0F1
:10BDB000002101E00199491C01918142FADB019ABD
:10BDC0000099895C0029F5D1019904981A9B471ABA
:10BDD00021463846199A00F097FA019940194518FA
:10BDE0000BE04FE02CE113E04EE000980099007862
:10BDF000491C00911A9A199990470198401E019088
:10BE0000401CF2D1214638461A9B199A10E137E0BE
:10BE10000A200021009001916002410F022907D001
:10BE2000189A01CA1892C2179446032908D00AE04A
:10BE30001898C01DC108C90005C91891944607E0AB
:10BE400000B2C2179446042902D140B2C1178C46F1
:10BE500000226146944506DA0A460021404291419B
:10BE60008C462D2102E0210504D52B216A46117351
:10BE7000012103E0E10701D02021F7E7029155E01D
:10BE80000A200AE0102008E0102000900021042081
:10BE900004430191082703E008200021019100904C
:10BEA0006002410F022907D0189A01CA1892002295
:10BEB0009446032908D008E01898C01DC108C9009D
:10BEC00005C91891944603E080B2042900D1C0B29C
:10BED00000210291210729D51199702906D0009AD5
:10BEE0001021019B4A401A4305D00EE040216A46CA
:10BEF0001173012108E06146014306D030216A46F2
:10BF000011731199517302210291009A0821019B2A
:10BF10004A401A430AD16146014301D1610705D560
:10BF200030216A46117301217F1E0291119958290F
:10BF300004D035A10E910DA90D910DE037A1F9E7BF
:10BF40006146019B009AFCF747F90E9B8C469B5C6F
:10BF50000D9A521E0D92137061460143F0D10D9857
:10BF600005A9081A20300190600703D501200004BC
:10BF7000844300E001270198874201DD381A00E080
:10BF80000020019900904118029809180498401A5D
:10BF90000490E00306D421461A9B199A049800F0F5
:10BFA000B3F94519002706E003A81A9AC05D19994C
:10BFB00090476D1C7F1C02988742F5DBE0030CD58F
:10BFC00021461A9B199A049800F09EF9451904E03D
:10BFD0001A9A3020199990476D1C0099481E0090BC
:10BFE0000029F5DC08E00D980D990078491C0D91A9
:10BFF0001A9A199990476D1C0199481E01900029C1
:10C00000F1DC63E109280100303132333435363751
:10C010003839616263646566000000003031323394
:10C020003435363738394142434445460000000034
:10C0300000F05AF94519761C3078002800D0E2E566
:10C0400028461BB0F0BD600700D406271898C01D15
:10C05000C108C90048680A680831C30FDB07189196
:10C06000190001D09CA108E0210501D59BA104E0A5
:10C07000E10701D09AA100E09AA1430011985B0862
:10C08000109165280CD006DC452809D046281DD023
:10C09000472841D141E0662818D067283CD13CE0D0
:10C0A0000021112F01DB112000E0781C019100908C
:10C0B00008A911A8FFF7E0FC139905910021119A36
:10C0C00015927F1C12980197009150E00120C00743
:10C0D00003900120019008A9009711A8FFF7CCFC5C
:10C0E000139A149905920022119B009212981593AD
:10C0F000059A0192002901D0104602E0791C4018EF
:10C100000190381A01D5019804E04042401E009089
:10C11000781C0190C01B029043E0012F00DA012738
:10C120000021112F01DD112000E03846019100901F
:10C1300008A911A8FFF7A0FC13990591119A0021F5
:10C14000129815920091019721070CD40599B942D4
:10C1500001DB019900E00191012904DD159A491ED6
:10C16000515C302906D0B84201DA011D05DA0121FF
:10C17000029115E00199491EEDE7002805DC0099C0
:10C18000411800910199091A03E0019A411C91425A
:10C1900000DD01910099401A401C02900120C00767
:10C1A0000390200706D402990198814202DB002007
:10C1B000C043029000206946C87707AF0121039869
:10C1C0000337C907884224D0022011902B201290F7
:10C1D000039800280CDA404203902D20129007E0CB
:10C1E0000A210398FBF7CEFF30317F1E0390397090
:10C1F0001199481E11900029F2DC03980028EFD114
:10C20000791E129808703078202108404530BF1EF2
:10C21000387006A8C01BC01D039010980078002835
:10C2200000D00120019941180298C01709180398FD
:10C2300009180498401A401E0490E00306D42146D1
:10C240001A9B199A049800F05FF845191098007825
:10C25000002803D01A9A199990476D1CE00324D541
:10C2600021461A9B199A049800F04EF845191CE0D3
:10C270000098002807DB00990598884203DD15988F
:10C28000405C199901E0199930201A9A904700985A
:10C290006D1C401C00900298401E0290002804D1A2
:10C2A0001A9A2E20199990476D1C0199481E0190E9
:10C2B0000029DDDC05E038781A9A7F1C199990472F
:10C2C0006D1C0399481E03900029F4DC21461A9B3B
:10C2D000199A0498ACE600002D0000002B00000025
:10C2E0002000000000000000F8B5044600251E46AE
:10C2F0001746880404D405E039462020B0476D1C59
:10C30000641EF9D52846F8BDFFB50446002581B066
:10C310001E46C80301D5302700E02027880404D535
:10C3200005E038460399B0476D1C641EF9D52846D0
:10C3300005B0F0BD4A68002A06D00A68531C0B609D
:10C3400010704868401E486070470A68531C0B60B4
:10C3500010707047002903D0002801D0884201D115
:10C36000002070478268002A08D05268002A03D053
:10C3700011604A60806841600120704781604960B7
:10C3800000200860F8E7FFB581B007000A9814465E
:10C390000D4605D0002D03D0002C01D0A74202D1BC
:10C3A000002005B0F0BD01267602002802D0E0682A
:10C3B000304307E02846049901F0CEFD051EF0D079
:10C3C000E068B0430646A089800505D4206A0028AD
:10C3D00002D0049949688847E660214638462562BC
:10C3E000FFF7B8FF05B0F0BD00B599B06021684611
:10C3F000FBF753FF042008AAD07012A00068019038
:10C400000B2010AAD070024610A109A8FBF72CFF40
:10C41000002010AA107101215171D0719171907397
:10C420001175D082A02010839176B42090831920BA
:10C43000C001D08308480090684603F0CBFE19B0D5
:10C4400000BD000003160A18000000000AFFFFFFED
:10C450004E6174696F6E73005DC400017047000027
:10C4600010B540210848FEF721FF08490020087058
:10C4700000F08EF9002802D005A0FFF751FAF7204E
:10C4800004F01CF810BD00000008014037470020F0
:10C490005B424C455D20636F6E6E65637465640D31
:10C4A0000A00000010B503F0B9FE00F07FF940214A
:10C4B0000648FEF7F7FE06490020087000F068F90C
:10C4C000002802D003A0FFF72BFA10BD000801409E
:10C4D000374700205B424C455D20646973636F6E93
:10C4E0006E65637465642C2061647665727469732B
:10C4F000696E67207265737461727465640D0A00F9
:10C5000010B58CB000240094019402940394049418
:10C51000059406940794089409940A94FFF766F822
:10C52000002804D0014601A8FDF72EF807E012A06C
:10C5300001886A4691804188D1808088108169464F
:10C54000CC704C810A20887012220A7303A80CA1B7
:10C550000130FBF789FE0C206946088418204884C6
:10C56000FF208C84F530C8840A480885684603F0AB
:10C57000F3FE0CB010BD000001020304050600002C
:10C5800043414949432D4D434D2D323032363039E8
:10C59000303200008813000000B583B00D490091CF
:10C5A0000D4900200191029069460872684603F027
:10C5B000D7FFFFF7A5FF00F033FAFFF715FF074895
:10C5C00003F074FD064803F071FD03F027FE03B08D
:10C5D00000BD0000E5C5000189D4000159CB000170
:10C5E00071D200010178012928D070B50025144EC0
:10C5F000144C022912D003290FD103F00FFE00F0D2
:10C60000D5F840213046FEF74DFE257000F0C0F809
:10C61000002802D00C48FFF783F970BD4021304656
:10C62000FEF744FE257000F0B3F8002802D007485A
:10C63000FFF776F9F72003F041FF70BD7047000067
:10C640000008014037470020D4C4000190C4000115
:10C65000F8B50646244F0020388178810124481E11
:10C660000D463E2814D80A4631462048FBF7FCFD0B
:10C670001E49002048551E4801F07AFD1B4801F074
:10C68000BDFC0446002001F073FD388900280CD160
:10C69000002C12D017A00090FBF70AFE84B22246AD
:10C6A00019480099FBF7E0FD3C81B878002819D0C3
:10C6B00016A0FFF735F900240CE019A0EBE7315D77
:10C6C000084620385F2800D32E2117A0FFF728F94D
:10C6D000641CA4B2AC4201D23F2CF0D3398913A020
:10C6E000FFF71EF9F8BD00005A4700202061002026
:10C6F00045E10001756E6B6E6F776E20636F6D6D37
:10C70000616E640D0A0000009B6400205B424C4592
:10C710005D20636C6920657865633A202200000023
:10C720006F6B0D0A000000002563000022202D3EE3
:10C7300020257542207273700D0A000030B40C4938
:10C74000098E182902D3891E8AB200E01422094CEE
:10C75000094D63892189ED18C91A89B2914200D91E
:10C7600011465A1862810180284630BC704700008B
:10C77000D04D00205A4700209B6400200348002130
:10C7800001708180C1804170704700005A470020CD
:10C7900001488078704700005A470020002800D0E8
:10C7A00001200149887070475A47002010B505499B
:10C7B000002008708880488100F058FF00F070FB6E
:10C7C00010BD00005A470020F3B583B00498002440
:10C7D00000287AD95B4802905B4A03981178005D83
:10C7E000002904D001290BD002291AD122E0CA283D
:10C7F0006CD156490870012090800521D18017E046
:10C80000524B91885854491C88B2908005285DD1BC
:10C810000298417803780802FF211843E1318842E9
:10C8200003D900201070908084E0C01DD0800220C9
:10C8300010707FE0444A454B91885854491C88B297
:10C840009080D188884275D1029800224178007882
:10C850000D0205433E488446281D86B23D48002E01
:10C8600014D93D4F6146895C090248400021030408
:10C8700002D54000784000E04000491CC9B280B2B7
:10C880000829F4D3521C92B2B242EBD32F4E711945
:10C890008A794B7911021943884247D17778B07869
:10C8A00001902948761D8078002806D033460095EF
:10C8B00039462AA0019A05F0C3FD112F2AD006DCC3
:10C8C000012F09D0102F31D124E039E032E0122FAE
:10C8D00020D0202F2AD124E001273F2D11D82A462D
:10C8E00031461F48FBF7C0FC1D49002048551D4834
:10C8F00001F03EFC1A4801F081FB0746002001F0E0
:10C9000037FC6846077001236A460320019900F04E
:10C910002BF80BE02B4632463846019900F090FB8D
:10C9200004E02A463146019800F004FA0648002146
:10C9300001708180641C0498A4B2844200D24BE749
:10C9400005B0F0BDA36100205A470020A06100207F
:10C95000A1610020FFFF00002110000052580000DC
:10C960006061002009240101FFB5D81D80B283B0A9
:10C970001D460190FB2803D90020C04307B0F0BD3D
:10C98000214CCA202070039860700498A070280A77
:10C99000E5702071002D04D02A46601D0599FBF733
:10C9A00063FC281D83B2194F19480024002B13D9AA
:10C9B000184E395D090248400021020402D54000AA
:10C9C000704000E04000491CC9B280B20829F4D38D
:10C9D000641CA4B29C42ECD30B4949194871000A6B
:10C9E00088710D488078002806D000950BA0059B23
:10C9F000049A039905F024FD0348019900F03EFED6
:10CA0000002007B0F0BD0000A0630020A16300205B
:10CA1000FFFF0000211000005A470020545800007A
:10CA200000B587B0002001900090039004906A4602
:10CA3000069010730C490291052191700323137025
:10CA40001023D37050701071012353719071507383
:10CA5000064805907D20917300011082104604F075
:10CA600045FA07B000BD000040E2010000B003013C
:10CA700001490120887070475047002010B50248D6
:10CA800003F0DCFF002010BD744E00202F48007919
:10CA900000285AD1F8B56D202C230322072140012C
:10CAA0000BF44AD0A0210446017029480027C17820
:10CAB000617027710321E180677201266671072189
:10CAC000244D2177A9796177687B002803D0E7801E
:10CAD000032060710EE0E87900280BD0A8790228C5
:10CAE00000D166772671E6802046A9792030417012
:10CAF0008670077015488079022804D0032815D065
:10CB000004281BD116E004F0E3F900280BD005201F
:10CB1000E0806771688A6061688AA06120460A3097
:10CB200004F004F80AE0094903208871288B606149
:10CB3000288B02E0E88B6061E88BA06103480671F6
:10CB4000467120460BF434D0F8BD7047D04D00201C
:10CB5000544E0020C04E002010B584B00A2303229A
:10CB6000072110480AF4E8D71B2101700021417009
:10CB70001424448003228280C1800B4A02810BF47A
:10CB800017D06846048009480190684603F0B0FC5D
:10CB9000684604810648039002A805F0A7F804B08F
:10CBA00010BD00001B0D0000FF010000D84C01016A
:10CBB0003DE30001FFB585B0054602A800901C4684
:10CBC0002846069904F0DCF96846007A002866D009
:10CBD00006980090280A334A019403900E2826D024
:10CBE000314800240178002951D92F48E100081864
:10CBF000828803998A4240D1009A81689646019AB8
:10CC0000284694460A791206120E36D00968254B3A
:10CC1000D700083FCE1937887668BFB2874201D067
:10CC20009F4226D1634603227146B04725E01F4943
:10CC3000681809282BD800981D49844608792E4683
:10CC400000062346000E1ED0C4000F68083C3C19A5
:10CC500027886468BFB2B74201D0974204D103224B
:10CC600061462846A0470EE0401E0006000EEBD1AC
:10CC700009E0521E1206120ECAD10B48641C00783D
:10CC8000E4B2A042B1D86846007A002807D009482B
:10CC9000426C002A02D0284606999047002009B02D
:10CCA000F0BD0000FFFF00007C4D0020EEF1FFFF13
:10CCB00028480101D04D002000487047FFFF0000C8
:10CCC00070B5124D01212846FCF7A4FD142006F092
:10CCD000CDFB702002F08CFE702002F089FE04462D
:10CCE00000212846FCF796FD094844800948844203
:10CCF00001D1401070BD2046FCF7C2FC0649FBF78D
:10CD000087FDFBF7A3FF00B270BD000000080240E2
:10CD1000A4470020FFFF00000000204110B500F0F4
:10CD20008BF90349884201D1022010BD012010BDBA
:10CD300000400201F0B5074600208DB015460E46B2
:10CD4000002A04D0012D04D13178FF2901D10B4EE6
:10CD500007250024002D08D90146325D684602F0FF
:10CD60007DFE641CA4B2AC42F6D303466A46394643
:10CD70002120FFF7F9FD0DB0F0BD0000FC4E0101D0
:10CD80000148408870470000A447002070B506465F
:10CD90000020074D044601462A5D064802F05EFE6B
:10CDA000641CA4B2072CF6D33080024870BD00008A
:10CDB000FC4E0101926A002010B5602002F018FEBE
:10CDC0000449884201D1002010BD6021FCF782FC9B
:10CDD00080B210BDFFFF000010B503F0F5FD044860
:10CDE0000169002901D004208847002010BD0000FF
:10CDF000E04E002070B5224C606B224DC00722D05F
:10CE0000A06B21497E2209685143401A2988491E96
:10CE100029804B21C90040181C49884213D30020A7
:10CE20002880206A400840002062194908680204EE
:10CE3000930F184A01D0904300E010430860164851
:10CE4000407F03F0F9FA298801200029216B07D0DF
:10CE5000014321630522032110480BF42FD10DE07B
:10CE6000FF22120291432163216B0522920211439A
:10CE70002163216B0143216304F078F8002070BD29
:10CE800000100240344700208C000020B104000054
:10CE90000010014000C00000304E0020010F0000D3
:10CEA00004480021017001624162816201630171E5
:10CEB000417170476847002002480021C17101811B
:10CEC0007047000068470020054A918901800029C9
:10CED00001D001209070002090810248704700002E
:10CEE00068470020826A0020F7B5414982B08A6312
:10CEF00003980024002879D93E483F4F00903C4ACF
:10CF00000298D179005D002904D001290CD00229B2
:10CF10001BD128E0CA2864D1384908700121118149
:10CF200005205081D1715CE0344B11895854491C63
:10CF300088B21081052854D10098417803780802FE
:10CF4000FF211843E131884203D90020D0711081BC
:10CF500047E0C01D80B25081052802D00220D07168
:10CF60003FE00020FBE7224A244D11896854491C08
:10CF700088B210815189884233D10098204D417880
:10CF80000278080210430346001D81B24A1E1D4864
:10CF900096B2002914D029780902484000216D1C5E
:10CFA000020402D54000784000E04000491CC9B2AC
:10CFB00080B20829F4D33146761EB6B20029EAD1F0
:10CFC0000E4AD1188D794E7929023143884204D115
:10CFD00091785078521D00F033F805480021C17156
:10CFE0000181641C0398A4B2844288D305B0F0BDCB
:10CFF000684700209E680020211000009B680020E8
:10D000009C680020FFFF000010B5024AFFF76CFF8C
:10D0100010BD00004910010101B5054A0121684613
:10D02000FFF762FF0349002288798A7108BD00007A
:10D030005D1401016847002000487047008000012E
:10D04000F0B51D464E4E83B013460C46102815D041
:10D0500011287AD0122879D013280DD1FFF720FF9C
:10D06000002213212046336A04F0A8F94548B16B29
:10D07000814201D10120B07103B0F0BD144600918E
:10D080000C2D09D0102D07D000230122102100986B
:10D0900004F094F903B0F0BD104604F07DF90746A2
:10D0A000201D04F079F902902046083004F074F94C
:10D0B0000190102D0BD00025307800280DD00222D1
:10D0C0001021336A009804F079F903B0F0BD2046CE
:10D0D0000C3004F061F90546EEE72B482B492C4C47
:10D0E000884202D0A0420CD10C462A49381F8842FF
:10D0F0000FD3002303221021009804F05FF903B03E
:10D10000F0BD002302221021009804F057F903B06B
:10D11000F0BD7078002803D1FEF780F9012070700F
:10D1200001203070776134610298B061019800216C
:10D1300031627162B1623163F061E80707D0114872
:10D14000B26B824203D1012002E00BE011E000202B
:10D150003071717100231A461021009804F02EF9E5
:10D1600003B0F0BD2A461946204603F07FFF03B006
:10D17000F0BD2A461946204604F036F803B0F0BD4B
:10D18000684700205D14010100800001008000015B
:10D1900000400201FDBF010010B50E4CE0780028F0
:10D1A00016D006F097FE616B401AA178002903D0D3
:10D1B000FF212D31884203D27D210901884207D306
:10D1C000BFF34F8F05490448C860BFF34F8FFEE798
:10D1D00010BD0000684700200400FA0500ED00E0E3
:10D1E00000487047C46A0020F8B53422114912483B
:10D1F000FBF73AF8104C114F20680125104EB84249
:10D200000BD16068012808D12046302100F0B8FE1B
:10D21000216B884201D13570F8BD34210648FBF7F7
:10D220003CF8FF202760F530656020810020E06039
:10D230003070F8BD00600001C46A00207ADA12CABA
:10D24000A847002010B534210748FBF726F8064808
:10D250000649016001214160FF21F5310181002172
:10D26000C16004F061F910BDC46A00207ADA12CA04
:10D2700010B584B014230322072112480AF45CD4A9
:10D280001B210170002141704724448003228280C9
:10D29000C1800D4AC2600D4A02610D2202720AF479
:10D2A00087D4684604800A480190684603F020F954
:10D2B000684604810748039002A804F017FD04B0F3
:10D2C00010BD00001B0D0000F84C0101E84C0101ED
:10D2D000E04C0101892B010100207047F8B5184D81
:10D2E000184FE879002801D02E7B00E0FE78032259
:10D2F000331D072114480AF41FD4A92104460170E4
:10D300001248C178617000216180E87910490028D5
:10D3100003D02A7B896C201D02E0FA78201D091DAC
:10D32000FAF7A2FF6088022180196080074802791D
:10D33000062A00D00171417120460AF439D4F8BDA3
:10D34000C04E0020A04E0020A60D0000D04D0020B1
:10D35000804E0020F8B51F262323032207212848EA
:10D360000AF4EAD30446AA20264F2070F878264D06
:10D370006070E8786080EA782449201DFAF774FF2D
:10D380006288B01AC1B2201D1018214A0326032951
:10D3900010D92B79002B0DD00670192343705389B7
:10D3A000091F1B0AC370937A83706388C9B21B1D5F
:10D3B0006380001D02291AD96B79002B17D0137BCB
:10D3C000891E8B4200D21946CDB2691C0170117BB7
:10D3D000A94201D1092100E0082141702A460D49E6
:10D3E000801CFAF741FF6088AD1C401960803879D5
:10D3F000062800D03E717E7120460AF4D9D3F8BDCC
:10D40000A60D0000D04D0020C04E0020A44E0020EC
:10D41000544E0020614E002070B53A2303220721AC
:10D4200016480AF489D3A421154D04460170E87802
:10D430006070A97913480022022910D0032913D063
:10D44000042916D062802271807902F023FC052025
:10D4500028710420687120460AF4AAD370BD018A9D
:10D46000642359436180EEE7C18A64235943618094
:10D47000E9E7818B642359436180E4E7A10D000053
:10D48000D04D0020C04E00207047000010B506F0BF
:10D4900011FD022803D106F01DFD0149086010BDF1
:10D4A0003847002010B58620FEF774F8002802D017
:10D4B0000FA0FEF735FAFDF7DFFF01210807FEF7A1
:10D4C00009F801210846FDF7FBFC1148FDF7BAFEFB
:10D4D0000520FDF7B1FE7D20C000FDF797FEFDF7AA
:10D4E000A3FEFDF799FE0B490020086010BD000067
:10D4F000204C6173742072657365743A20495744F7
:10D5000047207761746368646F67210A0000000038
:10D510005555000038470020FFB50F4683B0002165
:10D520000091019116466946FCF734F8040030D1A9
:10D530000521C9026846FCF733F8002828D12149A3
:10D540006846FCF72DF8002822D11F496846FCF7F1
:10D5500027F800281CD11D496846FCF721F800284F
:10D5600016D1292109026846FCF71AF800280FD1C4
:10D5700017496846FCF714F8002809D11549684690
:10D58000FCF70EF8002803D100988088C10B03D067
:10D590000624204607B0F0BD00050099000D0D18C7
:10D5A0006888B04200D207242988B819884201D976
:10D5B0000D24EEE7A8193A46001D0699FAF754FE25
:10D5C0006F80E6E701280000032800000228000021
:10D5D0000229000003290000084C06F06BFC022819
:10D5E00002D106F077FC20601DF4DAD600F012F8C4
:10D5F000FFF7D2FD012005F039FFEEE738470020A4
:10D6000010B503490020087000F004F810BD0000B8
:10D610005447002012480021007800281FD070B520
:10D62000104D86B02878002817D1A8886C88A042B1
:10D6300013D00D4E6A4680B2A04209D0335C5354D9
:10D64000401CC005491CC00D89B2A8801429F2D322
:10D6500001202870104605F09BFA06B070BD704797
:10D660003747002054470020205F00200249002057
:10D67000488088800870704754470020F0B4844682
:10D680000D480078002814D00022002911D90B4839
:10D690000B4D878843881C465B1CDB05DB0DBB42BA
:10D6A00007D06646B65C521C2E5592B243808A4221
:10D6B000F0D3F0BC704700003747002054470020EB
:10D6C000205F002070B5134D04462878002803D150
:10D6D000FDF7A4FE012028700F4820602821204675
:10D6E00000F04EFC0D4DA0622846FDF785FE002897
:10D6F0000DD12C2221462846FDF7ACFE002806D18C
:10D700002C2229462046FAF7F2FD002800D00120FD
:10D7100070BD0000AA47002011C011CA00400001DE
:10D7200010B5044600681949884208D120462821CE
:10D7300000F026FCA16A884201D115A200E016A2E1
:10D740001B491CA000F0B4FC21A0216800F0B0FC33
:10D7500026A0616800F0ACFC2AA02369E268A168F9
:10D7600000F0A6FC33A0616900F0A2FC37A0236A98
:10D77000E269A16900F09CFC2EA0616A00F098FCAF
:10D780003EA0A16A00F094FC10BD000011C011CAB7
:10D7900076616C6964000000494E56414C49442052
:10D7A00028626164206D616769632F637263290079
:10D7B00000400001626F6F7473657474696E672056
:10D7C000402030782530386C583A2025730D0A00F7
:10D7D00020206D61676963202020202020203D20CB
:10D7E00030782530386C580D0A0000002020616325
:10D7F000746976655F62616E6B203D20256C750DE6
:10D800000A000000202062616E6B313A206164647E
:10D81000723D30782530386C582073697A653D2523
:10D820006C75206372633D30782530386C580D0A72
:10D83000000000002020202020202020207665727B
:10D840003D30782530386C580D0A00002020626188
:10D850006E6B323A20616464723D30782530386CEA
:10D86000582073697A653D256C75206372633D307D
:10D87000782530386C580D0A0000000020206372B3
:10D88000633332202020202020203D203078253096
:10D89000386C580D0A00000030B58DB00121082009
:10D8A000FDF724FE01218803FDF720FE02A8FDF705
:10D8B0003FFC4020029002202C4D0424039002A93A
:10D8C00007942846FDF7D8FB80210794029102A90E
:10D8D0002846FDF7D1FBE120C002089000206946F0
:10D8E0008884C884088588850C204885204D08A92F
:10D8F0002846FDF7C9FF01210846FDF7D3FD1D4C61
:10D900002046FDF7EBFA012322461B490220FDF7D2
:10D910005FFB012280212846FDF786FF00220121BE
:10D92000402005F025FF154C0322606000210120F6
:10D9300005F01EFFA060012005F008FFE06000F088
:10D9400077F801220E492846FDF746FF1C2069465C
:10D95000087003204870012088706846FDF7AAFC13
:10D9600001212846FDF752FF0DB030BD000C0140EB
:10D970000038014008000240000002403C470020FF
:10D9800024040000F3B5274F81B00C4600257868C9
:10D9900000280AD006F08EFA022806D1002201994A
:10D9A000786806F03FF8012816D01F48FDF7E6FA20
:10D9B00003218902081A398880B281420ED01B489F
:10D9C0003988415C01980170032138888902401C24
:10D9D000FAF7D8FB3980012003B0F0BD002C0AD043
:10D9E000601C01D0A54206D2B868002803D006F01A
:10D9F00061FA022802D0002003B0F0BD1426601C9A
:10DA000003D0601B142800D206467D213046C90091
:10DA10004843FAF7B7FB0146B86806F0A4F8AD1919
:10DA2000B5E700003C4700201C000240004F0020EA
:10DA300030B5194D8BB000212846FDF793FA2846E2
:10DA4000FDF74CFA01232A4614490320FDF7C0FADA
:10DA50001348009013480190032080020390002493
:10DA600080200590202008900494000202940990E0
:10DA70000694079469460A942846FDF789FA0A48ED
:10DA8000048001212846FDF76DFA01224021074854
:10DA9000FDF7CAFE0BB030BD1C0002400000024082
:10DAA00004380140004F00203C470020003801406E
:10DAB00038B500200D4C00900B492046FDF7C3FE01
:10DAC000002810D02046FDF723FF09488068002871
:10DAD00002D0694605F06CFF0098002803D00120B1
:10DAE00004490007486038BD2404000000380140A4
:10DAF0003C47002000ED00E030B5194D85B00446EC
:10DB000040212846FDF798FE0028F9D0002128463C
:10DB1000FDF77CFE0020694600948880C88008815B
:10DB200088810C2048812846FDF7AEFEFFF780FF74
:10DB30000C4C6068002807D006F0BCF9022803D11D
:10DB40000021606805F036FE012207492846FDF7EE
:10DB500043FE01212846FDF759FE05B030BD000007
:10DB6000003801403C4700202404000010B5064C5A
:10DB7000E068002807D006F09DF9022803D1C11EF5
:10DB8000E06805F0F0FF10BD3C47002010B5074CE1
:10DB9000E068002809D006F08DF9022805D100239D
:10DBA0001A461946E06805F03CFE10BD3C470020CF
:10DBB00000283FD000293DD0F0B51F4E0C46054649
:10DBC0008BB000213046FDF7CDF91C4F02203946BD
:10DBD000FDF782F91A480090102002900020802161
:10DBE0000591049003210195039409030690079081
:10DBF000089009910A9069463046FDF7C9F901215C
:10DC00003046FDF7AFF939460220FDF7BAF9002892
:10DC1000F9D000213046FDF7A5F939460220FDF77D
:10DC20005BF9084C40212046FDF706FE0028F9D09C
:10DC30000BB0F0BD70470000080002400000024039
:10DC4000043801400038014010B4002807D00368B0
:10DC5000002B04D042688168914201D206E0002086
:10DC600010BC7047491C8160002804D0914202D248
:10DC70005C5C202CF6D99142F2D1491E816010BC27
:10DC800070470000F8B50C4605461046194600F0EE
:10DC900013F8064600200090064B324621462846DF
:10DCA000FEF771FB0028304602D100F043F8002057
:10DCB000F8BD0000B447002070B505460E46124876
:10DCC00000F0A2F804001CD0E6610820A561E06025
:10DCD0000E4A0F4B28463146FBF73EF802D80D4856
:10DCE00060610EE000220C4B28463146FBF720F81D
:10DCF00002D80120C00703E028463146FAF7C0FFEA
:10DD00006061204670BD0000B44700200000C0FFE5
:10DD1000FFFFDF41FFFFFF7F0000E0C110B50448B7
:10DD200000F072F8002801D04021C16010BD000051
:10DD3000B4470020002824D0F8B5124E044600272E
:10DD4000A0892568C0050DD4A068002804D0FFF77D
:10DD5000F1FFA089C00505D42069002802D07168B0
:10DD600088472761A089800505D4206A002802D051
:10DD70007168884727627168204688472C00DFD188
:10DD8000F8BD7047B447002010B5002201F088FDAF
:10DD900010BD000030B4124A0E4D0F4B0F4C00283E
:10DDA000136013D00168002900D0116054604068EE
:10DDB000002800D05060002090601068984203D185
:10DDC0005068A04200D1956030BC704795605460A7
:10DDD00030BC7047E52F010131BA0001CDB9000117
:10DDE000B4470020002803D0007B082801D0002081
:10DDF000704701207047002803D0007B402801D0E5
:10DE0000002070470120704710B50168282088471E
:10DE100000280AD00021016041608160C160016179
:10DE200041618161C1610162416210BD70B500262E
:10DE300004463546002808D0FAF73AFA411C2B462A
:10DE40003246204600F004F870BD002070BD00008E
:10DE5000FFB5002489B0064600940194344802942A
:10DE60000394049405940694046015464460002EBF
:10DE70005AD000293FD0024600960191D16890689F
:10DE800012690490069205912A48FFF7BDFF07909A
:10DE9000002830D000986F46002802D00298002851
:10DEA00001D000200DE00198042809D9032222A105
:10DEB0000098FAF732FA002802D10298C01C0290AA
:10DEC0003846FFF7C1FE0146079803F093FC00288F
:10DED0000ED00C98002814D06846FFF7B5FE0299C2
:10DEE0000198814204D202990098405C002808D031
:10DEF0000798FFF71FFF0199029888420AD204464B
:10DF00000BE0002D03D00299009840182860079874
:10DF10000DB0F0BD081E00D0441E002D01D03019F8
:10DF2000286003480660446000200DB0F0BD00008A
:10DF3000AC470020B4470020EFBBBF0010B5024A39
:10DF4000002103F075FF10BDB44700200149496866
:10DF500008470000B4470020002810D070B50E46D6
:10DF60000446FAF7A5F9401C336805469847061E93
:10DF700004D02A462146FAF777F9304670BD70473B
:10DF8000002230B4D243491E0FD3094C03785A40C3
:10DF90000023401C5508D20700D022465B1C6A4073
:10DFA000DBB2082BF6D3491EF0D230BCD043704709
:10DFB0002083B8ED02468B880020022B01D00D2073
:10DFC0007047C988002A05D00029F9D00129F7D067
:10DFD000812070470029FCD00229F9D17047112017
:10DFE00070470000112804D20C2148430249085808
:10DFF0007047002070470000304E010170B588B0B6
:10E0000000246A46234616E0401C01782029FBD0F4
:10E010000929F9D00906090E12D0A1005050641C3C
:10E0200000E0401C017800290AD0202901D00929EC
:10E03000F7D10370401C0178002901D0082CE4DBE3
:10E04000002C14D0104E002528460C21484331588E
:10E050000098FAF734F900280CD06D1C112DF3D379
:10E060000AA0009900F024F8012008B070BD00203B
:10E0700008B070BD0C204543A81982686946204647
:10E080009047002008B070BD304E0101756E6B6E78
:10E090006F776E20636F6D6D616E643A202573201B
:10E0A00028747279202768656C7027290D0A000092
:10E0B0000FB410B503AB60210648029AFDF754FC7B
:10E0C00005490020C877034800F058F810BC08BC88
:10E0D00004B01847805C0020C05C0020F3B581B01C
:10E0E0000D460198FAF7E4F8144C86B22046FAF788
:10E0F000DFF881B22046FFF75BFD0024002D0BD92D
:10E100000F4F3846FAF7D4F881B23846FFF750FD82
:10E11000641CA4B2AC42F3D3084C2046FAF7C8F80A
:10E1200081B22046FFF744FD002E03D0314601980E
:10E13000FFF73EFD304603B0F0BD00001CA7000114
:10E1400028A7000130B40125074B084CAD0203E0BD
:10E150006254491C1981401C0278002A02D0198996
:10E16000A942F5D330BC70475A4700209B64002079
:10E1700001490860704700004C47002010B507496E
:10E180000968002901D0884710BD0446FAF790F8C5
:10E1900081B22046FFF70CFD10BD00004C47002067
:10E1A000F0B51FB40546039814464600019876085A
:10E1B00047007F08334628463946FAF7CDFD02D29C
:10E1C0002846394601E0204631463322D243FAF749
:10E1D000EFFC06460F4622462846039B0199FAF7B4
:10E1E000F9FB490049083B463246FAF7A1FD02D83F
:10E1F000012005B0F0BD002005B0F0BD02460020B2
:10E20000802901D98D207047062A06D0072A07D019
:10E21000082AF8D10729F5D170470829F2D17047AB
:10E220000629EFD370477047704770B5C46805463C
:10E230006068002803D00020002802D00CE00120F4
:10E24000FAE7201DFBF7B2F909F466D360680028ED
:10E2500008D000200028F4D00020E860204609F40F
:10E260005BD370BD0120F5E730B40446A2890920D4
:10E27000521C93B2E48900222546D540ED0707D011
:10E280005D1C8D4202D130BC104670479B1C9BB276
:10E29000521CD2B2092AEFD330BC7047FFB585B00B
:10E2A0000E9D04462F8801201E4600213A46CA4092
:10E2B000D20704D04B0003225B1C9A401043491C38
:10E2C000C9B20929F2D3049030461E210840218AA0
:10E2D000184A00230191009302920390132304AA89
:10E2E00015490698FBF768F9009000281FD1012115
:10E2F000142009F49BD30746E06006980188B98191
:10E300002988F981F00701D00120C003079908434B
:10E310003880208A788014206082204600F060F8DF
:10E32000381DFBF74FF9208A002109F4D5D4009855
:10E3300009B0F0BDE84601010A1800000048704726
:10E3400080470101FFB5087881B00C46092836D214
:10E35000142003F097FC0746217800F0EFF800281E
:10E360002BD061782078FFF749FF060028D17D681F
:10E37000002D0ED020782979814207D12946381DF9
:10E38000FBF726F9284609F4C7D202E02D68002DD4
:10E39000F1D160780121083009F448D3054620788E
:10E3A0002871607868716278A11CA81DF9F75CFF7C
:10E3B0002946381DFBF712F902E0822600E081268B
:10E3C00002230648039A049909F4B6D32178017010
:10E3D000467009F4EDD3002005B0F0BD0114000033
:10E3E00010B50446142003F04DFC044921600321BC
:10E3F0006181123060600120208110BD90470101D1
:10E40000F8B517460C46104609F454D4012831D10A
:10E41000142003F037FC0546017C00F08FF8064617
:10E42000297C22781448914214D1697C63780902CE
:10E430003A46891D9B1D09F47FD3054606800020BE
:10E440002871607868806278A11C681DF9F70CFF5C
:10E45000284609E0697C062309023A46891D09F429
:10E460006BD306808021017109F4A2D300213846C4
:10E4700009F432D40020F8BD140C0000F8B50F46A2
:10E48000002409781846254609291DD20B007B4433
:10E490001B79DB189F440407101313130A160D0091
:10E4A000052414A510E00A2414A50DE0082416A5DF
:10E4B0000AE0072417A507E00A2418A504E00524AC
:10E4C00019A501E006241AA50146A31C1A4809F45F
:10E4D00033D30646387830707470002C04D022464E
:10E4E0002946B01CF9F7C0FE304609F461D300207C
:10E4F000F8BD00004E53494E470000004E532D42D8
:10E500004C452D312E300000123456FFFE9ABCDEF1
:10E5100000000000025E044000000300312E302E97
:10E52000302E302D4C450000312E302E30000000B2
:10E53000FFEEDDCCBBAA00000314000010B48289FA
:10E54000C489521C93B200222046D040C00706D096
:10E55000914202D15B1C9BB205E09B1C9BB2521CFA
:10E5600052B2092AF0DB092A02D010BC18467047C3
:10E5700010BC00207047000070B5050005D0134E98
:10E580003068854203D1002070BD72B6FEE704F00A
:10E5900025FF6C6904F02EFF7068844202D0B068D9
:10E5A000844201D1022070BD0948844204D1A86A86
:10E5B0000028F7D1032070BD0648844203D0002C08
:10E5C00001D0012070BD042070BD0000C4470020B0
:10E5D000D46B0020C06B0020002802D00368002B01
:10E5E00001D100207047F8B50D4641680446002966
:10E5F00002D0A068884211D21B4EB5420ED8A26844
:10E600006D1C5019814201D39818F8BD2169002969
:10E6100004D11649884203D9B04202D90020F8BD7E
:10E620004600226A0027002A05D031461846904746
:10E63000050012D00CE0A1693046884705000CD0D7
:10E64000A2682168521CF9F70FFEE169206888472B
:10E6500066602560A0684019F8BDE16920688847B8
:10E66000676000202760F8BDFFFFFF7FFFFFFF3FCF
:10E6700070B50D4D04460A2809D10D212846FDF735
:10E680004BF980212846FDF7D7F80028F9D0E1B2F0
:10E690002846FDF741F980212846FDF7CDF80028EE
:10E6A000F9D0204670BD000000380140F0B5087870
:10E6B000324F334D334E801E83B00C46062859D25C
:10E6C00001007944097949188F4402255434543A99
:10E6D00001203070A0786876A078C00705D02A495C
:10E6E0002A48FAF751FF387AA874B28A002A06D06D
:10E6F000FF20F53070800321254809F4DFD4F1694B
:10E70000002937D000200090019005206A46107043
:10E71000684688472EE000246C7601F007FEF16918
:10E72000002927D0009406206A460194107068469C
:10E7300088471FE01722A11C1648F9F795FD19E03C
:10E74000B8780001C0194030807D002812D11C2209
:10E75000A11C1148F9F788FD0F48A18A0182E18ABE
:10E760004182218B8182618BC1820B49608A08833F
:10E77000207F6874002003B0F0BD0000D04D002061
:10E78000144D0020304D0020D94D0020274D002091
:10E79000040F00000E4D0020F44C0020F0B5184688
:10E7A0000D46014685B022230322744809F4C4D1E2
:10E7B00001210446417028780B286ED2010079446B
:10E7C000097949188F4405CDCDCD6F6ABB23CDCDD6
:10E7D0006C00012020706070694881792171017995
:10E7E000A170C17961714179E170017AA171417AB9
:10E7F000E171817A2172C16900294ED00020009018
:10E8000002206A461070684601948847A9E00720F4
:10E8100020700120607068461CF420D7019F009E84
:10E82000F9F710FD801960820025F9F70BFD8119B9
:10E83000601900908170F9F705FDC11900986D1CF1
:10E84000EDB20175082DF0D30825F9F7FBFCB919D5
:10E85000401861196D1CEDB28870102DF5D3102091
:10E86000207748488178090108184030807D0128C8
:10E8700077D11C22A11C4448F9F7F6FC4248A18A32
:10E880000182E18A4182218B8182618BC1823E4972
:10E89000608A08833D48217F417462E0052000E0E2
:10E8A0000A2020705DE0042222706878012804D0DC
:10E8B000002802D0022833D053E00120304D607090
:10E8C000287C002810D002A81CF4C8D6F9F7BAFC9E
:10E8D0002F49F9F757FC2F480818029940182E497C
:10E8E000F9F750FC009101E0E8680090E96900291F
:10E8F00007D00020029003206A46107202A80392FB
:10E9000088471021A01CF9F7C8FC0098A070009857
:10E91000000AE0700098010C2171000E607120E087
:10E920001748C169002905D0002000900190684671
:10E930000270884720460C3809F430D114E00620D4
:10E94000164D2070E878012811D01021A01CF9F78D
:10E95000A4FCA9886182E988A1822989E18200203A
:10E960002076204609F424D1002005B0F0BD102205
:10E970000B49A01CF9F778FCEBE70000140E00002F
:10E98000304D0020D04D0020F44C0020144D0020CC
:10E99000A0BB0D00A08601003F420F00544E002096
:10E9A000DF4D002000B5084883B0026C002A08D073
:10E9B00000200090029005206B4618706846019177
:10E9C0009047002003B000BDD04D002010B584B0AA
:10E9D000FF2B19D0144C226C002A08D00020009084
:10E9E000029006206B4618706846019190470320FC
:10E9F00009F460D1032814D1A26F002A11D0032199
:10EA00000A4809F45BD30CE009480123007F032284
:10EA100001020848083109F48FD00721017009F478
:10EA2000C7D0002004B010BDD04D0020090E00005A
:10EA3000304E0020050E0000FFB5180A4C4E83B082
:10EA40000C46B070FF287DD00102342303224948D0
:10EA5000083109F471D00546B07800270101891901
:10EA600040318872B07821880001801940300181DE
:10EA7000B078617A000180194030C172B078628943
:10EA80000001811940318A81A289CA81E089088206
:10EA9000207C012802D0002807D00BE0B1780120AB
:10EAA000090189194031887504E0B07800018019A6
:10EAB0004030877520883080607A307221460A3174
:10EAC0002D48FAF761FD02F003FA00281BD0607AA6
:10EAD000012804D103221146284809F47DD002F010
:10EAE000FFF905280FD201007944097949188F44AC
:10EAF00006060602060001202821485505E00521EA
:10EB00002820415501E0282047550321059809F4A4
:10EB1000E3D017203086B178090189194031488245
:10EB20001748C068002803D00321164809F426D2EC
:10EB30001548028D002A03D00321144809F4BED2DF
:10EB4000306C00E00EE0002808D0022069460097F3
:10EB5000087002950194316C68468847284609F48C
:10EB600027D001E001F05AFB002007B0F0BD000003
:10EB7000D04D0020020E0000D94D0020150D0000E0
:10EB8000E04E0020030F0000544E0020020F000052
:10EB900030B5180A144D00010C46401983B0FF210E
:10EBA0004030817201F00EFC002803D102210320C5
:10EBB00009F492D02A6C002A08D00020009002901C
:10EBC0000320694608706846019490471021074861
:10EBD000F9F763FB06480068002802D0092008F412
:10EBE00065D6002003B030BDD04D0020EF4D002091
:10EBF000100C002000B5084883B0C169002907D077
:10EC000000200090019009206A46107068468847ED
:10EC1000002003B000BD0000304D0020FFB591B0D2
:10EC20000D46122303224348149908F485D7002186
:10EC30000446017040480078002862D03E48407C7D
:10EC4000002833D03C216846F9F727FB01F032FF5A
:10EC5000002841D004A90F913749461EF0B23A224C
:10EC60008969504341186846091DF9F7FDFA68465D
:10EC7000008B2988884206D10822A91C0F98F9F731
:10EC800036FB00280BD0207800280BD008A8407C49
:10EC9000607410226946601CF9F7E6FA1CE0012056
:10ECA0002070F3E73006000ED6D12AE023482988E9
:10ECB000008B884225D10822A91C2148F9F717FBAF
:10ECC000002809D1012020701E481022407C607469
:10ECD0001A49601CF9F7C8FA2078002811D01648A4
:10ECE000C169002907D000200090019007206A46E2
:10ECF000107068468847204608F45AD7002015B09F
:10ED0000F0BD0D48C169002907D000200090019096
:10ED100008206A46107068468847022303220A4882
:10ED2000149908F409D7012101700621417008F4F3
:10ED30003FD7E0E7180E0000304D0020F44C0020D3
:10ED4000044D0020144D0020040E000070B50C4648
:10ED500009781B481B4D1E46002904D0012912D0FA
:10ED600002292BD11AE01C23314608F4E5D60646C9
:10ED700020783070287B70802A7B1349301DF9F78A
:10ED800073FA304607E00A23314608F4D5D62178D5
:10ED900001706989418008F40BD70FE00A233146DE
:10EDA00008F4CAD621780170298C4180698C818051
:10EDB000A98CC180E98C018108F4FAD6002070BDCD
:10EDC0000B0E0000544E0020614E002010B5087854
:10EDD00000F060FF002010BD05480A8842861A0A2C
:10EDE000120110180988403081820020704700000D
:10EDF000D04D002030B5180AC043000683B00D4640
:10EE0000000E21D0190A0902E12006230322000185
:10EE1000083108F491D60446012020700220608059
:10EE2000FF204130A0800B48026C002A08D000204F
:10EE30000090042069460870684601950294904746
:10EE4000204608F4B5D601E001F0E8F9002003B04F
:10EE500030BD0000D04D002000B5084883B0026CE2
:10EE6000002A08D000200090029008206B461870FD
:10EE7000684601919047002003B000BDD04D0020AE
:10EE800070B518460C46014602230A4808F454D6C9
:10EE900005460949A07808736288211D0748F9F7DB
:10EEA000E3F90020687020782870284608F480D69E
:10EEB000002070BD0D0E0000544E0020614E002059
:10EEC0004A780B48002A05D02030012A08D0022AAF
:10EED00009D00AE00279012A07D10978C17004E05B
:10EEE0000978017501E0097841750020704700003C
:10EEF000D04D002070B54878002806D0FF25124C70
:10EF000001280BD0022816D01BE0104801790629F1
:10EF100017D10721017101F0EFF812E0207DFF28E1
:10EF20000FD001F0E7F90A4825750169002908D0DA
:10EF30000020884705E0607DFF2802D001F0BCF981
:10EF40006575002070BD0000F04D0020D04D002000
:10EF5000E04E002010B5032B06D010220548891D75
:10EF6000F9F782F9002010BD0348017A034801F047
:10EF700057FEF7E7EF4D0020D04D0020D94D00207F
:10EF8000F0B50D460878E34EE1493446497800274C
:10EF900020348DB0A1287AD012DCDF490C911B28D7
:10EFA00076D006DC012819D003287CD017286DD133
:10EFB0004FE128286ED091286DD0A02866D152E16B
:10EFC0000246A23A092A61D213007B441B79DB185E
:10EFD0009F44FE5CFDFD5CFDFCFDFD0068780028A3
:10EFE00054D1012002F0B2FE01F058FE3423032276
:10EFF0000721CA4808F4A0D503210170C849044676
:10F000008A7842700122C276FB224284C54AC284B9
:10F01000C54A82840A88028487768A888280CA8860
:10F02000C2800A892281487A8009032805D188781C
:10F030000522104201D10120A076A07E04221043B7
:10F04000A076BA486080C878012825D020461021D3
:10F050000A30F9F722F9316C002907D001206A46FD
:10F06000009710706846019502948847012000F0CF
:10F0700011FE204608F49CD5012303220721AC4849
:10F0800008F45AD51A21017008F492D533E11EE133
:10F09000CAE008E069E049E0204610220A300C99F5
:10F0A000F9F7E2F8D7E700970197029703970497DB
:10F0B000059706970797089709970A970B9701F006
:10F0C00007FF002805D0684601F048FD0AA801F0B6
:10F0D00015FD01F0FDFE00280CD06846807900285F
:10F0E00008D108A8807B002804D00121684601F0DF
:10F0F0007BF900E18A4C6946A0880880E088488056
:10F10000208988808F71102202A80C99F9F7ACF839
:10F11000E078012804D00697079708970997E4E755
:10F12000102206A80C99F9F79FF8DEE7E07B00288B
:10F1300013D11123032207217E4808F4FDD405468C
:10F14000282028707648C078012808D01021681C33
:10F15000F9F7A3F8284608F42BD5E773CBE0102283
:10F16000681C0C99F9F780F8F4E7012002F0EEFD35
:10F170000121032008F4B0D56F48012444841F20E6
:10F18000049067480178490601D57F210491817870
:10F190000522114204D0FF220499813211430491C7
:10F1A0000088C00504D5032104984902084304904F
:10F1B000082162480191029003210B2304AA0097C1
:10F1C0000394C9025E48FAF7F7F902E079E04AE0F1
:10F1D00089E0002846D15B4806218786FF200590FC
:10F1E000594801910290082305AA009703945749B2
:10F1F0005748FAF7E1F900287DD100F067FF0028B1
:10F2000079D10221032008F467D5B079012808D00C
:10F2100001F02CF83E484078C0076CD001F06EFB3E
:10F2200069E000F0FBFF66E001F052FEE77300F0DA
:10F230004DFF00285FD10221032008F44DD5B0799D
:10F240000128EED001F012F831484078C007E5D12E
:10F2500051E0687800284ED0F179481EF0713D48A1
:10F2600001F0AEFC47E07179491E052906D8A728B0
:10F2700002D13079002806D100F03EFF2878A4287A
:10F2800001D0A72837D17079042806D0062804D0E9
:10F29000082808D00C282ED10CE02F48016800293E
:10F2A00029D0B07904E01A480169002923D001204F
:10F2B000884720E01648016900291CD003208847B0
:10F2C00019E03771FF20F0702075607513E0207D24
:10F2D000FF2802D06878002802D001F00BF80AE07D
:10F2E000C8079BD107E0607DFF2802D0687800281E
:10F2F00004D000F0E1FF00200DB0F0BDA07D00289B
:10F30000F9D08807F7D5E17D144801F065FAF2E7F6
:10F31000E04E0020D04D0020DF4D0020040D000005
:10F32000544E00200502000048080000A08C000098
:10F33000190D0000230D0000B00B0020644B0101EB
:10F34000D20B0020680B0020BC4B0101011800000B
:10F350009C0B0020D94D0020804E0020084E00203C
:10F3600070B500250C462846401C0628FCDB254EBF
:10F370002246307E31461A32C96906282AD2030055
:10F380007B441B79DB189F4424020910171E0622B8
:10F39000A01CF8F7ACFF00281BD01BE0237E09203F
:10F3A00001F0BAF8002814D114E0237E212001F0E6
:10F3B000B3F800280DD10DE0237E162001F0ACF843
:10F3C000002806D106E0237E192001F0A5F80028C8
:10F3D00000D001250C48807D002811D171690029D9
:10F3E00001D020468847002D0AD03169002901D07C
:10F3F0000220884701F004FB217AA01C01F0ECF9FF
:10F40000002070BDE04E0020F04D002010B50A78BD
:10F41000000A000210434A78FF231B02120298439D
:10F420001A4010438A781B02120498431A40104372
:10F43000C9780002000A09060843F8F70CFF00200B
:10F4400010BD10B5104608F435D4002010BD0020C2
:10F45000401C0628FCDB002070470000F8B51C4665
:10F4600017460D46104608F425D4002811D1472030
:10F4700002F008FC064604233A460321064808F435
:10F480005BD3210A01702988B288891A418008F467
:10F490008FD30020F8BD00000D470000F8B51746D7
:10F4A0000C46472002F0EEFB21780646122901D0D7
:10F4B00013291BD1B06805460C351229C288018971
:10F4C00016D006230F4808F437D369884180617845
:10F4D000017108F46DD3B068002803D008F41CD281
:10F4E0000020B0600021384608F4F6D30020F8BDB3
:10F4F0000423054808F420D369880180617881706D
:10F50000E7E70000094700000747000000B508488A
:10F5100083B0026C002A08D00020009002900920DD
:10F520006B461870684601919047002003B000BDFB
:10F53000D04D002030B5104D83B0088828861C0AB5
:10F54000200140190A88403042822A6C0025002A96
:10F5500007D0009507206B46029518706846019108
:10F5600090470648A1004058002801D04030C5749B
:10F57000002003B030BD0000D04D0020580B00200B
:10F58000FFB581B0002000900E46039808F492D396
:10F59000002802D001284CD04DE0142002F072FB6C
:10F5A00007463188FEF760FE05462448092D36D20D
:10F5B0007C68002C1ED02179A94203D02468002C3D
:10F5C000F9D117E0002C15D06379039A9B1D04999B
:10F5D00008F4B2D20546308828800020287160796E
:10F5E00068806279A11D681DF8F73EFE284608F480
:10F5F000DFD220E03D740498010A7974384602F0A5
:10F6000039FB014601230E48039A08F495D2057090
:10F6100008F4CED20121039808F45ED30BE0062350
:10F62000039A049908F488D23188018080210171FD
:10F63000DDE702200090009805B0F0BD140C00003A
:10F6400002140000FFB585B00E46079808F432D3C7
:10F65000002802D0022009B0F0BD472002F012FBC2
:10F6600002900020694608700898070A308803F065
:10F67000D8F90024694605468C8000281ED10298DE
:10F680001622016A6846007803465043024610324B
:10F690008A5A5204920F1FD10A5C401C085C1E4912
:10F6A00000021018884217D102AA03A9184603F0D5
:10F6B000CBF802986946C05D88800224A31D1748D4
:10F6C000079A089908F438D20746308838803D7187
:10F6D0007C80002D15D019E03946029802F0CAFA54
:10F6E000014604230E48079A08F426D2077069469B
:10F6F0000978418008F45CD20121079808F4ECD223
:10F7000007E0224601A9781DF8F7AEFD384608F457
:10F710004FD2002009B0F0BD02290000140C0000F7
:10F7200004470000FFB58BB00C46472002F0AAFA50
:10F730000025694605900D740E9804A9070A2088D3
:10F7400003F06FF9060061D105981622016A684638
:10F75000007C5043024610328A5A5204920F3AD12A
:10F760000A5C401C085C304900021018884232D103
:10F7700002950395208800F0DFF802A9002300918C
:10F780001A4608A9F9F730FF6846008C01210903E1
:10F790000840C043C004C0172146401CFEF70AFCC5
:10F7A0000606360E32D168460997007C0190A5798D
:10F7B00007AA694603F048F86846028806A8079930
:10F7C000F8F752FD06A909980A460D5468460188C3
:10F7D000019803F077F83946059802F04BFAA188B2
:10F7E0000D9A891D8BB20146104808F4A5D1054633
:10F7F000A288A11D801DF8F737FD2F706846007C98
:10F800006880A088A880284608F4D2D1042308483C
:10F810000D9A0E9908F490D121880180867008F421
:10F82000C7D100200FB0F0BD022900000A47000038
:10F83000160C0000F0B589B00446F9F7DBFE05466A
:10F840000026154F1BE006A92046F9F7A3FE00236A
:10F8500002AA01A906A80096F9F7D2FE6846008917
:10F86000B84203D169460979022911D00B4988426F
:10F8700003D168460079022807D0641CA4B2A88886
:10F88000A04202D8E888A042DDD2002009B0F0BD35
:10F89000204609B0F0BD0000022900000328000046
:10F8A000F7B5002845D00199002942D08668002A82
:10F8B00001D10CE03668002E3BD0316A002938D0E7
:10F8C0000198F8F7FCFC0028F4D12CE03668002EF3
:10F8D0002FD0019C356A002CF8D0002DF6D0AC4218
:10F8E00024D02078F8F7A8FC07462878F8F7A4FC7D
:10F8F00087420DD12078002813D06078641C6D1CDD
:10F90000F8F79AFC07462878F8F796FC8742F1D07A
:10F910002078F8F791FC04462878F8F78DFC8442AB
:10F92000D4D1002E05D0306A002802D0304603B072
:10F93000F0BD002003B0F0BDF0B589B00446F9F782
:10F9400059FE05460026104F14E006A92046F9F797
:10F9500021FE002302AA01A906A80096F9F750FE8D
:10F9600068460089B84203D1641CA0B209B0F0BD5A
:10F97000641EA4B2A888A04202D8E888A042E4D2BB
:10F98000002009B0F0BD00000328000070B5164C3F
:10F990002078002827D101210803FBF783FD0020F0
:10F9A000FBF776FD0120FBF7ADFD104D2846F9F77A
:10F9B000D5FE03212846F9F741FF01212846F9F732
:10F9C00001FF012121702846F9F724FF142003F0DC
:10F9D0004DFD702000F00CF8702000F009F80021B7
:10F9E0002846F9F717FF70BDA44700200008024021
:10F9F00070B50546164CFFF7C9FF2946154D284638
:10FA0000F9F737FE01212846F9F7D2FE01212846F1
:10FA1000F9F70CFF002807D1641E13D001212846F6
:10FA2000F9F704FF0028F7D001212846F9F71EFE58
:10FA30002846F9F7F8FE044600212846F9F7B8FEF3
:10FA4000204670BD00212846F9F7B2FE024870BD7D
:10FA5000A086010000080240FFFF0000F7B5042760
:10FA60000225494E86B01446082A74D21000784404
:10FA700000790018874484030D3A3D53637043486E
:10FA8000019001AB00970799069800F08BF809B038
:10FA9000F0BD3F4F01213846F9F7BCFE142003F0BA
:10FAA000E5FC7020FFF7A4FF7020FFF7A1FF0446DC
:10FAB00000213846F9F7AEFE3648B442448001D101
:10FAC000354808E02046F9F7DBFD3449F8F7A0FE99
:10FAD000F9F7BCF800B2694688812A4603AB009565
:10FAE0000799069800F05EF809B0F0BDFDF7E4F85C
:10FAF0000AE06020FFF77CFFB04201D1002003E064
:10FB00006021F9F7E7FD80B26946088102AB224621
:10FB100000950799069800F045F809B0F0BD04F08B
:10FB2000D9F97D21C900F8F72DFB019001AB2246E0
:10FB300000970799069800F035F809B0F0BD03F07A
:10FB4000D1FD019001AB224600970799069800F07D
:10FB500029F809B0F0BD13E0FDF76EFA10498842AC
:10FB600001D1022000E001206946087401200090C4
:10FB700004AB22460799069800F014F809B0F0BDCE
:10FB8000079809B0F0BD0000FFFF00001C00010055
:10FB900000080240A4470020FF7F00000000204131
:10FBA0000040020130B4029C42540546491C88B210
:10FBB0002C54401C002180B2002C07D95A5C2A54D6
:10FBC000401C491CC9B280B2A142F7D330BC704777
:10FBD00010B5084C82B02078002808D10648009063
:10FBE000064801906846FEF7D5F80120207002B063
:10FBF00010BD0000C0470020192701011134010188
:10FC0000F8B50B30C608F600104D19E02068B04278
:10FC100015D3B0420BD96368871B201D0093F8F7FA
:10FC200023FBA019009B07604360286004E0606824
:10FC30002860201DF8F718FB201D2660F8BD251D43
:10FC40002C68002CE2D10020F8BD000020480020E4
:10FC5000FF25F5350D4E0E4FFDF7C2FA0489322C03
:10FC600000D22C4604F026F9022802D104F032F921
:10FC7000306001213846FBF7EBFA7D212046C900B0
:10FC80004843F8F77FFA03F0F1FBE5E73847002037
:10FC9000000C014010B5A0230949022809D0002218
:10FCA00003280AD0042808D00B704A7000F0A2F88C
:10FCB00010BD0B7080204870F8E7E0200870F4E772
:10FCC00011400020F8B52A49202048602948012128
:10FCD000C163294905228A610021C16327490B209C
:10FCE000086100F087F82748254A026326494163E6
:10FCF000264B8363264CC4632748264D0560274E58
:10FD00004660274981602749C16027490161274929
:10FD1000416127498161274901632848264941609B
:10FD2000274FC760274F07610262274A42628362FA
:10FD3000C46205634663254A8263254AC263264836
:10FD4000244A0260184A4260244A826001632449BE
:10FD500081632448244A41688918244A914206D282
:10FD6000234982680A63C2684A6300698863F8BDF0
:10FD700000100140C02702404025024040270240B9
:10FD80000259F80040280240025B8500025A8000B8
:10FD9000025D8500025F80508028024002000878E2
:10FDA000020A0800026EAC500259FC000200C800B2
:10FDB0001270131402700314026E2800C02802404F
:10FDC000025D0500125B0500025B8400020A06006A
:10FDD000026E2C5002C3BF00002902401200AC008A
:10FDE000125D0500104000206F2895FFAF590F00ED
:10FDF000C026024030B415481549037D154AFF2B33
:10FE000006D1407DFF2803D113484078C0070CD0AD
:10FE10001248134B04789C604078D86111480861FF
:10FE2000114B8B62106030BC7047104B0B61104857
:10FE30004861104C8C61104D8D62C8620F48086398
:10FE400013600F485060946030BC7047F04D002044
:10FE50000028024040280240E04E002011400020CF
:10FE600000270240127E0200127E0300027E020082
:10FE700002C2A00012C70000027E030012C7800069
:10FE800002C2E00082B0234921480863FDF704FD67
:10FE900021A0FBF745FD2BA0FBF742FD32A135A0C9
:10FEA000FBF73EFD3948016839A0FBF739FD3FA15A
:10FEB00043A0FBF735FD4BA0FBF732FDFDF7F2FA4F
:10FEC000FCF76AFBFCF75AFC01215148FBF7C4F927
:10FED00040215048FBF7C0F9FDF786F901F03AF8E8
:10FEE000022000240202009023464BA101944B48BB
:10FEF00003F024FF012000900023802248A10194F8
:10FF0000484803F01BFFF9F7B3FF03F089FBFEE756
:10FF100000800081007000400A3D3D3D3D3D3D3D7B
:10FF20003D3D3D3D3D3D3D3D3D3D3D3D3D3D3D3D01
:10FF30003D3D3D3D3D3D3D3D3D3D3D3D3D3D3D3DF1
:10FF40003D0A0000206D636D2D6464632D626C6555
:10FF50003A20424C45202B204672656552544F533F
:10FF6000202B20434C490A0056312E30302E323897
:10FF700000000000204669726D7761726520766529
:10FF80007273696F6E2025730A0000000040002024
:10FF90002053797374656D436F7265436C6F636B47
:10FFA000203D20256C7520487A0A000043414949CC
:10FFB000432D4D434D2D3230323630393032000032
:10FFC00020424C4520656E61626C65642C20616442
:10FFD000766572746973696E672061732022257378
:10FFE000220A00003D3D3D3D3D3D3D3D3D3D3D3D09
:10FFF0003D3D3D3D3D3D3D3D3D3D3D3D3D3D3D3D31
:020000040101F8
:100000003D3D3D3D3D3D3D3D3D3D3D3D0A0000000A
:10001000000C014000080140424C4500D9D50001C8
:100020004C45440051FC000110B50124E402204677
:10003000FAF7DCFF002805D02046FAF7D1FF0D497A
:1000400002200870012424032046FAF7CFFF00287D
:100050000AD02046FAF7C4FFBFF34F8F074906487E
:10006000C860BFF34F8FFEE705484068002800D006
:10007000804710BD800000200400FA0500ED00E07C
:100080004040002006480068002800D08047BFF3A9
:100090004F8F05490348C860BFF34F8FFEE700004C
:1000A000404000200400FA0500ED00E0064A117807
:1000B0000A2907D28900891848601078401C1070FE
:1000C0000120704700207047504D002010B5084CAB
:1000D000084AE17913780020994207D288008018F5
:1000E00040688047E079401CE071012010BD0000AD
:1000F000D04D0020504D0020F8B5324D052629790D
:1001000028468079304C08290CD20A007A441279AA
:100110009218974403080D1313191C2A052801D0BF
:10012000FCF7B4FCF8BD022808D0FDF7D7F8F8BDFD
:10013000607B002802D1E079002802D0FDF76CF93D
:10014000F8BDFDF707F9F8BD06202871F8BD0223B8
:10015000032207211D4807F4EFD4A5210170E97897
:100160004170072129716E7128E0022303220721C3
:10017000174807F4E1D40746A7203870E97879706A
:100180000620687100202871032007F493D5032806
:1001900012D0A879012804D0022802D003280BD15C
:1001A00004E0207D002801D0032003E0A07E002889
:1001B00002D00420A87100E0AE71384607F4F8D4EC
:1001C000F8BD0000D04D0020C04E0020A20D000060
:1001D000A30D000010B5002804D0014660220C4891
:1001E000F8F742F80B490C48CA781C2A04D9427B1C
:1001F000002A01D11C22CA70C1781F2901D91F21F0
:10020000C170017BE22901D9E221017310BD000018
:10021000804E0020A04E0020C04E00201149012237
:10022000087907280CD08879002809D0012801D046
:10023000052806D10C48827B002A03D002200CE05E
:100240008A717047027D002A01D0032005E0807E7C
:10025000002801D0042000E00520887110B5FCF7CB
:1002600015FC10BDD04D0020C04E002070B5104CC4
:100270000525A079062809D2010079440979491891
:100280008F44020204040403A57170BDA57102230A
:1002900003220721074807F44FD4A5210170E17814
:1002A000417007212171657107F482D470BD00008F
:1002B000D04D0020A20D000010B50B4C607DFF2832
:1002C00010D0022303220721084807F435D4A721C0
:1002D0000170617D4170064A00215171FF216175F5
:1002E00007F466D410BD0000F04D0020A30D0000FF
:1002F000D04D002010B50A4C207DFF280ED00223DF
:1003000003220721074807F417D4A7210170217D94
:100310004170054A0021517107F44AD410BD000014
:10032000F04D0020A30D0000D04D002010B508486E
:1003300002238078032201020648083107F4FCD327
:10034000012101701321417007F432D410BD000067
:10035000D04D0020040E000010B584B0002804D059
:1003600001462A220E48F7F77FFF0EA00FC86C4601
:100370000FC40B4B002069461C180A5C24792243E9
:100380000A54401CC0B20628F6D310220A48F7F7D8
:100390006BFF0A490A48F9F7F7F804B010BD0000EE
:1003A000544E0020501921901F04D5624FA489ABF0
:1003B00090D0CF2300000000DF4D0020584E0020D9
:1003C000FC0000200020074B01460A01D2184032F1
:1003D000927AFF2A01D0401CC0B2491CC9B203293D
:1003E000F3D37047D04D0020F8B507460B462820C0
:1003F00043430D46032207210E489B1C07F49CD360
:1004000091210170002406464570002D0ED920462A
:1004100028214843C1190022CA7180192822801C52
:10042000F7F722FF641CE4B2AC42F0D3304607F485
:10043000BFD3F8BD910D0000F8B57D262025F6004C
:10044000184B194C1949032812D00A6A01273A435C
:100450000A620A6A9207FCD50A6AAA430A6201285C
:100460001AD002281AD01E60F9F7D0F82060F8BD23
:100470000F480F2782683F023A438260086A0422CD
:1004800010430862086A0007FCD5086A284308621E
:100490003D2000011E60E9E7064800E006481860BC
:1004A000E2E700008C0000209000002000100240D5
:1004B00000100140D10300005704000010B50446AD
:1004C000084804238078032201020748891D07F4A5
:1004D00033D306494C80012101700021418007F48B
:1004E00067D310BDD04D0020010C0000F00B0020A0
:1004F000084A11780A290AD2C90043688918006895
:100500008B6048601078401C1070012070470020FC
:10051000704700007C4D0020FFB581B01C000646EE
:1005200018D01078411CA14214D8032C12D3401EBD
:10053000C5B25078971CB04206D12A463846029977
:10054000F7F7D5FE002808D07A19601B801E040634
:10055000240EE6D1002005B0F0BD012005B0F0BDAD
:10056000F0B504466F4E704883B06D4FB168C162FC
:100570006E490163F16A8162F16B4163B16B816322
:1005800031467C2240313846F7F76EFE00257D600B
:10059000FD607D626648B8627D64BD64FD643D6651
:1005A0006448B86664483862644865490570032049
:1005B00008706448F914016009040160891401603D
:1005C000F06861490746401E0088604B884200D0B1
:1005D0001F60366E701E0088884200D05E60012069
:1005E00000030090694601950D71082048710127AC
:1005F0008F716846FAF708FD84215548F7F74DFEDC
:100600002A215448F7F749FE60215348F7F745FE81
:1006100052484F49056145618561C5610562456282
:100620008562C562FF264E48CE700675467500206D
:10063000020152184032401CC0B296720328F7D310
:10064000206808646068486446486189C187217AE7
:100650004548032901D8417700E045770121202052
:10066000FAF720FF414A4249042001F09DFA42492D
:10067000404808600A464149052001F095FA404A81
:100680004049072001F090FA40493F4808600A4677
:100690003F49082001F088FA3E4A3F49092001F00D
:1006A00083FA3E4805633E48414907703D4805705E
:1006B0003D4805703D48086001203E49C002088061
:1006C0003D494F2008703D49082008703C480721EB
:1006D000067046708670C170057145718571C5716F
:1006E00011483849C16138490162384941620020E6
:1006F00002F0B2FC3649032007F432D30021032074
:1007000007F4EAD2002001F021FB01230322072194
:10071000304807F411D2077007F44AD203B0F0BD95
:10072000C009002000800001C000002085000101F8
:100730000D4700207131010129000101C600002090
:10074000D800002000E100E0FEE70000404000206B
:10075000D04D0020544E0020804E0020D04E00206E
:10076000F04D0020104E0020304E00208040002030
:100770008080010031480101C0400020C08001009C
:100780000041002000DB01008141002040410020A9
:1007900040DB0100C0460020C06102000070004044
:1007A00060000020C9000020610000200090D003FC
:1007B0006C0000206800002063000020640000201E
:1007C00008010020ED1B0101151D0101B51C0101EF
:1007D000C44C0101020D0000F8B5404D0646687D8D
:1007E0003F4C0F46FF281CD02046C268002A03D089
:1007F00003213C4807F462D43A23032207213A48F4
:1008000007F49AD1A4210170697D044641703748EC
:100810000022017800291ED00121A170A28002705F
:100820001BE06D20022303220721400107F484D13D
:10083000A22101702E49C978417007F4B9D1EF7532
:1008400031462C48F8F7A0FE0120A87560780221F7
:1008500008436070F8BDA270A2800120E0701921E9
:100860004901E18022482181038CE381438C23826A
:10087000838C6382C38CA382FF23E2824133184DB1
:1008800023836D786D070DD50525E5706181A18104
:10089000018CE184418C2185818C6185C08CA0858F
:1008A000E285238638200755204631463230F8F756
:1008B0006BFEE078810703D50220FFF7EBF906E035
:1008C000400701D5032000E00120FFF7E3F90A49C2
:1008D0000C204871204607F46BD1F8BDF04D002084
:1008E000E04E0020030F0000A10D0000504E00203C
:1008F000544E0020084E0020D04D0020F8B52C4E5C
:100900002C4D317D01276878FF2941D0C1073ED0A9
:10091000B84368702849002008703A230322072151
:10092000264807F409D10446A4202070307D607069
:100930002878A07068788006800F20716888E08031
:10094000A8882081E888E08128892082E77001203A
:10095000FFF7A0F9687840070AD5E078022108433C
:10096000E07068886081A888A0810320FFF792F971
:100970006878000703D5E0780C210843E07010493F
:10098000082048710020B075204607F411D1F8BD49
:10099000384368706D20022303220721400107F4C9
:1009A000CBD0A12101700749C9784170EDE7000063
:1009B000F04D0020E04E0020504E0020A10D000020
:1009C000D04D0020544E002010B50A4C607DFF2809
:1009D0000ED0022303220721074807F4ADD0A5213A
:1009E0000170617D4170054A0D21517107F4E0D01D
:1009F00010BD0000F04D0020A20D0000D04D0020E1
:100A000070B50B4C207DFF2811D00A4D687909285C
:100A10000DD0022303220721074807F48DD0A5211A
:100A20000170217D41700921697107F4C1D070BD49
:100A3000F04D0020D04D0020A20D000010B504465E
:100A40004088A1880246491C19234A43DB019A4287
:100A50000FDC06280DD3228890420AD3E2887D233A
:100A6000DB009A4205D84B00C9184843D1008842A0
:100A700001DD002010BD0D480E2380780322010205
:100A80000B48083107F458D00921017021884180B2
:100A900061888180A188C180E18801810021418134
:100AA000491E818107F484D0012010BDD04D002063
:100AB0000E0E000010B5084A084B90690188847832
:100AC000994206D1917CA14204D20024FAF794FC09
:100AD00000E00024204610BD304D002034120000FC
:100AE0000B4610B504493A2289695043411818460B
:100AF000091DF7F7B9FB10BD304D002010B590B0BF
:100B000004463C216846F7F7C8FBFFF7D3FF401EB9
:100B1000C0B26946FFF7E4FF08A8807CA0710CA969
:100B200020460331F8F730FD10B010BD10B590B07D
:100B300004463C216846F7F7B0FBFFF7BBFF401EB9
:100B4000C0B26946FFF7CCFF08A8007CA0710AA9D3
:100B500020460231F8F718FD10B010BD10B590B066
:100B600004463C216846F7F798FBFFF7A3FF401EB9
:100B7000C0B26946FFF7B4FF0AA920460231F8F770
:100B800003FD08A8007CA071204606A910220830A9
:100B90000231F7F769FB0848C1782046183001296F
:100BA00004D01021F7F779FB10B010BD10220349D3
:100BB000F7F75AFB10B010BD544E0020DF4D002057
:100BC00070B590B00D460646FFF774FF002D23D098
:100BD000854221D8182303220721104806F4ACD7F8
:100BE000044617202070012060703146A01CF8F7E1
:100BF000CBFC3C216846F7F750FB6D1EE8B2694616
:100C0000FFF76EFF204606A9102208300231F7F7E1
:100C10002BFB204606F4CCD710B070BD140D00009D
:100C2000F3B58FB00C463C216846F7F736FBFFF76B
:100C300041FF012C1AD0002816D0154D0AAE0236FD
:100C4000441EE0B23A22A969504341186846091D82
:100C5000F7F70AFB062231460F98F7F748FB002802
:100C60000DD02006000EEBD111B0F0BD0949421E97
:100C7000CA7101460F98FFF7A3FF11B0F0BD06A996
:100C8000102205480231F7F7EFFA11B0F0BD00006D
:100C9000304D0020D04D0020EF4D002070B5284C85
:100CA00082B020688003FCD5264D687FFFF7C4FB27
:100CB000606A606A012630436062606AB0436062C5
:100CC0002148C08F0A2811D9E16932071143E16137
:100CD0001E494A6832434A601E491D4A0A6003227F
:100CE0004A6088601C4808601C48086068461AF41E
:100CF000B5D41B4900980860687FFF252D020328A2
:100D000011D000F027F9206BA8432063206B3F210E
:100D1000490208432063206B3043206301220321F2
:100D2000104807F4CBD110480168A94301600F496E
:100D30000868FF2212049043086002B070BD0000F2
:100D400000100240304E0020104E002040100240A3
:100D50005555000000300040AAAA0000CCCC00008D
:100D600048400020010F000000E400E008E400E03B
:100D7000F0B5D7B054A81AF471D44A490024886A4F
:100D8000C96A54990122411A09010909D2069142FE
:100D900004D95499081A000100094142424E4029E1
:100DA0000CDC7088002809D0401E708014220321BA
:100DB0003E4807F483D1002057B0F0BD3C48FF21E6
:100DC000569029316846F7F768FA707CB5690028B3
:100DD00032D0FFF76FFE69468870B17C6F4688425B
:100DE0000BD23A2148430246291D381DF7F73CFA39
:100DF00069468878401C887008E03A21401E4843C4
:100E0000024629463E31381DF7F72EFA69468878A2
:100E10003A214843C0190A4636385699F7F724FA5A
:100E2000244869460880B069FAF7E6FAFF222732BB
:100E30006946B069FAF70EFBFF20F53070804A94DE
:100E40004B944C944D944E944F945094519452948E
:100E500017485394418D40AA1185818D5185C08DCD
:100E60009085154C48AA257C9573102213494CA8EF
:100E7000F7F7FAF91248C078012804D11022114975
:100E800050A8F7F7F1F901260F48002DC67306D1D7
:100E9000A07C002803D001214AA8FFF7A5FA0B483F
:100EA000067088E7C0800240304D0020040F00002B
:100EB000F44C002034120000144D00200E4D002090
:100EC000544E0020DF4D0020F04D0020504E0020F9
:100ED00002480078002800D001207047304D0020E3
:100EE0000148007970470000304D002070B5174967
:100EF0003CC80E4684B040363CC6436802688068F1
:100F00004B65134C0A658865607C002818D0002565
:100F100069460D72FAF782FAFFF7CCFD694608724E
:100F2000E1690126002906D068460095067002A8EE
:100F30000190684688476846007A002802D02670EB
:100F400004B070BD257004B070BD0000F44C0020EA
:100F5000304D002004490868401C0860012801D079
:100F60000120704700207047244000200349086892
:100F7000002802D0401E0860012070472440002055
:100F8000F8B50C462849294B4118294F294A002613
:100F9000069D002908D0012922D0274940180A2897
:100FA0002FD301202870F8BD20780A2838D2214993
:100FB00080000958214A914203D11E490E501E500B
:100FC0002EE0B9422CD10322082311461C4806F416
:100FD000B3D5217801706168416006F4E9D51FE05E
:100FE00020780A281CD280001158B94218D119580B
:100FF00011502078134962684018032107F45ED02D
:101000000EE0C0B20A280BD284001159002907D083
:10101000B94205D0094FB94202D016511E51884736
:101020002E700020F8BD0000FBF0FFFFCC4C00202C
:1010300087320101A44C0020F9F0FFFF8532010145
:10104000060F0000070F0000102909D810B50C4644
:101050000A4601460348F7F707F90348848110BDA3
:1010600070470000826A002068470020F7B55C4F97
:1010700082B0387814460D46002809D0042C0FD2CF
:10108000012211213B6A029800F098F905B0F0BDE9
:10109000002302221121029800F090F905B0F0BD62
:1010A000084600F079F9241F00943B6A2D1D9842F0
:1010B0000ED03879002802D078790028EED10222AB
:1010C0001121029800F07AF90120787105B0F0BD85
:1010D00078691E19864206D903221121029800F070
:1010E0006DF905B0F0BD3E62B86AB0420FD2B96A80
:1010F00038694018FAF780F9002801D0052207E086
:101100000120B96A00030818B862B042EFD3002288
:10111000002A3CD1386B002822D03249042808D25A
:10112000002C1BD02B780B54401C641E6D1C3863A4
:10113000F4E73E46042811D1716A3069294B401802
:1011400004221946FAF786F9002801D0052203E0A7
:10115000706A001D0022706200203063002A16D1E0
:10116000042C1DD37A6A3869A608B600801829466F
:101170003246FAF76FF9002801D0052203E0786AB9
:10118000801900227862AD19A41B002A08D0112111
:101190003B6A029800F012F9FBF782FE05B0F0BD41
:1011A000002C05D0224629460E48F7F75DF83C632F
:1011B0000020787138793B6A00280AD00098190B12
:1011C000181A000B00030903884202D17869834290
:1011D000E4D100221121029800F0F0F805B0F0BD32
:1011E0006847002094470020F7B5664C8CB0237800
:1011F000002B11D0042A07D001221221236A0C9857
:1012000000F0DCF80FB0F0BD084600F0C5F8064667
:10121000236A6069834206D0022212210C9800F0F2
:10122000CDF80FB0F0BD206B0025002815D00428A4
:1012300006D25549FF220A54401C20630428FAD3E1
:10124000636A206950490422C018FAF703F900289C
:101250007ED1606A2563001D606261692069FCF7C8
:101260008FFEB04202D1A169884209D00422122126
:10127000236A0C9800F0A2F8FBF712FE0FB0F0BD45
:101280002069001D00F088F821690A460832904262
:1012900003D362698918814209D806221221236A80
:1012A0000C9800F08BF8FBF7FBFD0FB0F0BD374E4C
:1012B0006F460FCE0FC70FCE0FC7B2687168306888
:1012C0000A920890324F0098203E0991B84206D108
:1012D00028213046FCF754FE0A9988420AD000952E
:1012E0000195029503950495059506950795089532
:1012F00009950A950097274A2169914201D1012059
:1013000000E0022001909142684601D1083000E0DF
:101310001830016061694160A1698160E169C16063
:1013200028216846FCF72CFE0A903046FAF764F84C
:1013300000280FD12C2269463046FAF78BF8002896
:1013400008D12C2231466846F6F7D1FF002800E08C
:1013500000E009D005221221236A0C9800F02EF833
:10136000FBF79EFD0FB0F0BDA5700022122163694E
:101370000C9800F023F802F0ADFD60630120E070EE
:101380000FB0F0BD684700209447002000400001E6
:1013900011C011CA008000010378C2781946437851
:1013A00012061B0219438378C0781B0419431143AA
:1013B0000902090A000608437047000070B586B0AC
:1013C0006C4621746274A374190AE174190C2175B6
:1013D000190E61751E498C6B002C30D0CA216A46EB
:1013E00011701F21517090700620D0700020107174
:1013F00004A9501DF8F7C8F816480923164D00AA8D
:1014000001321178090248400021521C060402D51D
:101410004000684000E04000491CC9B280B2082981
:10142000F4D319465B1E9BB20029EAD16946C87203
:10143000000A08730D216846A04706B070BD01463A
:10144000062304AA1F20FBF78FFA06B070BD000028
:1014500068470020FFFF00002110000070B50C4617
:101460000546FCF783FB21462846FCF7A1FBFCF769
:101470008DFB02490120887070BD00006847002084
:1014800070B5FEF7A5FBFCF749FC04002FD01A4D00
:101490002889F7F7BFFB02460B4618A12046FCF748
:1014A000F1FBE868F7F7B6FB02460B4614A12046AD
:1014B000FCF7E8FB13480078F7F7ACFB02460B4655
:1014C00011A12046FCF7DEFB2046FCF737FD054660
:1014D0002046FCF72FFC002D09D02846FCF74EFED5
:1014E0000BA0FCF74BFE2846FCF730FD70BD09A0B1
:1014F000FCF744FE70BD0000C46A00206C65640007
:1015000070776D00A847002076616C696400000068
:101510000D0A00006A736F6E3A20616C6C6F632075
:101520006661696C0D0A000070B5134C0125607886
:10153000002802D1F9F772FF657010483021FCF7DE
:101540001FFD0E490E4E08633046F9F755FF00287F
:101550000DD1342209493046F9F77CFF002806D125
:10156000342231460548F6F7C2FE002801D001209A
:1015700070BD2570002070BDA8470020C46A0020FF
:1015800000600001F3B583B004980021066880680C
:10159000009137187D1C305C2C4622287ED104989F
:1015A000406807E05C2A04D15B1C834277D2491C67
:1015B000641C641CA31B834202D22278222AF1D12C
:1015C000A21B82426BD22078222868D1E01B401AED
:1015D0000499401C09698847009000285ED0A54204
:1015E00070D229785C2903D00170401C6D1CD8E0B2
:1015F0000223611B012952DB6A78662A15D008DCB8
:10160000222A22D02F2A20D05C2A1ED0622A46D13C
:1016100008E06E2A0DD0722A0FD0742A11D0752AD4
:101620003DD115E00821017010E00C210170401C33
:10163000B6E00A210170401CB2E00D210170401C8F
:10164000AEE009210170401CAAE00270401CA7E036
:101650000022944606296FDBAF1C1346F95C0E4648
:10166000303E092E02D8303A8A180BE00E46413E31
:10167000052E01D8373A04E00E46613E052E1FD8EC
:10168000573A8A18032B00D212015B1C042BE5D3B6
:1016900037218902531A55498B4201E09CE094E0BE
:1016A0007BD91B23DB02D31A8B423FD80C23A91D05
:1016B0009E46631A062B70DB0B785C2B6DD102E023
:1016C0000022E5E770E04B78752B66D1891C01910B
:1016D00000210E46019B9B5D1F46303F092F02D81B
:1016E000303959180BE01F46413F052F01D83739D3
:1016F00004E01F46613F052F16D857395918032EAD
:1017000000D20901761C042EE4D337239B02CE1AA3
:1017100001239B029E4240D292058905120B890D3E
:101720000A439901521803E00021EEE706218E4694
:10173000802A02D2012315E02FE00121C9028A424A
:1017400003D20223C0218C460CE0012109048A4205
:1017500002D20323E02104E025498A421DD8042354
:10176000F0218C46591E0906090E0AD0164680271C
:101770003E43BF273E404654491E92090906090EC2
:10178000F4D1012B03D961460A43027002E05106ED
:10179000490E0170C018734600E00023002B14D0DE
:1017A000ED18A54200D21CE700210170039810211A
:1017B000C160039900980861049804990068201A90
:1017C000401C8860012005B0F0BD0098002803D0BF
:1017D0000498416900988847002D04D00498006857
:1017E000291A04988160002005B0F0BDFF030000B5
:1017F000FFFF1000F0B591B00C0006467ED02168C6
:1018000000297BD0A0686368021D9A4206D8081898
:101810000422DBA1F6F781FD002833D0A0686268BE
:10182000411D914207D8216805220818D6A1F6F774
:1018300074FD00282ED0A0686268011D914207D86F
:10184000216804220818D2A1F6F767FD002829D0E4
:101850006268A168914203D22068405C22282BD0A4
:1018600091427AD22068405C2D2802D03038092875
:1018700073D800200146109020682E22002807D03F
:101880006B464DE00420F060A068001DA0600120C0
:1018900011B0F0BD0120F060A068401DA0600120E3
:1018A00011B0F0BD0220F06001207061A068001D41
:1018B000A060012011B0F0BD21463046FFF762FE66
:1018C00011B0F0BD25682818085C342820D00DDC44
:1018D00005462B3D092D28D22F007F443F79FF1963
:1018E000BF441623161823161616160038280FD0D4
:1018F00008DC35280CD036280AD000E074E0372800
:1019000013D105E0392803D0452801D065280CD132
:10191000585400E05A54491C3F2906D2002C04D0E8
:10192000A06867684518BD42CCD30020585410A960
:10193000184601F099FC0F46054610996846884202
:1019400052D0F761944A954B28463946B561F7F76E
:1019500003FA03D8924870610FE019E00022914B1E
:1019600028463946F7F7E4F902D80120C00703E01A
:1019700028463946F7F784F970610820F060109A1C
:10198000A1686846101A0818A060012011B0F0BDC7
:101990007D20C000914203D223685B5C5B2B06D0A4
:1019A000914279D22268515C7B2967D074E000278C
:1019B000E1683D4681426FD2491CE1602168A06820
:1019C000095C5B2968D1401CA0602046FCF73CF90B
:1019D0006168A068884203D22268125C5D2A38D010
:1019E000884202D3401EA06056E0401EA060204600
:1019F00010300090FCF708FA002839D0002F23D0CF
:101A0000286045600546A068401CA0602046FCF7A1
:101A10001BF921462846FFF7EDFE00282AD0204674
:101A2000FCF712F9002C25D06168A068884203D227
:101A30002168095C2C290AD0626890421AD2216878
:101A4000085C5D2816D104E007463D46DBE70098B8
:101A5000D0E7E068401EE060002F00D07D602020CD
:101A6000B760F060A068401CA060012011B0F0BD1C
:101A7000002F11D03846FCF75DF90DE00027E16832
:101A80003D46814208D2491CE1606168A0688842F5
:101A900002D2115C7B2902D0002011B0F0BD401CA5
:101AA000A0602046FCF7D0F86168A068884203D2A5
:101AB0002268125C7D2A4CD0884293D2401EA060DE
:101AC000204610300090FCF79FF9002855D0002FD9
:101AD0004ED0286045600546002CCBD0A0686168D8
:101AE000401C8842C6D2A0602046FCF7ADF82146D3
:101AF0002846FFF747FD0028BCD02046FCF7A4F895
:101B000028692862002028616168A0688842B1D2F3
:101B10002168095C3A29ADD1401CA0602046FCF741
:101B200093F821462846FFF765FE0028A2D02046FC
:101B3000FCF78AF86168A068884203D22168095CD2
:101B40002C2918D06268904294D22168085C7D28C4
:101B500090D1E068401EE060002F00D07D60402002
:101B6000B760F060A068401CA060012011B0F0BD1B
:101B700007463D46B0E70098A5E7002F8CD079E7EF
:101B80006E756C6C0000000066616C73650000008F
:101B900074727565000000000000C0FFFFFFDF41A8
:101BA000FFFFFF7F0000E0C1102819D230B40D4CB8
:101BB00083001B199D6989032D0B2D03090D0D430E
:101BC0009D619969084D920992052940920A114335
:101BD00099610122616982401143616130BC7047A3
:101BE0007047000000200240FF0FC0FFF3B505461C
:101BF00081B00026408800F003F901000AD01C4F94
:101C00006A88002014234343DB195B8A934203D183
:101C100042262AE0402628E0401CC0B20A28F1D320
:101C2000002E22D1002414206043C019408AFF28CE
:101C300006D0641CE4B20A2CF5D30A2C14D014E0AC
:101C400028460830009014206043C0190E686B7855
:101C5000AA880746A91DB0470600EED16888788299
:101C60000298398A0180E8E74B26304603B0F0BD80
:101C7000884B002002885004400CD20B01D009028E
:101C80000843704710B40024094A214614234B43EB
:101C90009B185B8A834204D1142041438818C4688E
:101CA00003E0491CC9B20A29F0D3204610BC704792
:101CB000884B002030B4FF23040AC5B20A49002033
:101CC000142242435218128AAA4204D114225043C9
:101CD0004018438A03E0401CC0B20A28F0D3200217
:101CE00030BC184370470000884B0020084A117828
:101CF0000A290AD2C9004368891800688B604860C5
:101D00001078401C107001207047002070470000C0
:101D1000504C002030B4FF23040AC5B20A49002009
:101D2000142242435218528AAA4204D11422504328
:101D30004018038A03E0401CC0B20A28F0D32002F6
:101D400030BC184370470000884B0020F1B582B0CA
:101D50000299294E0020002900D1307000250298F8
:101D6000002804D0012834D002283ED10FE02946B3
:101D700014225143214A284609308C182082C0B2CF
:101D800006F408D0207C214605F4EAD72DE0284649
:101D900014214843194900234718B87C0090307833
:101DA0001C4600280DD9E0008019828800998A42DB
:101DB00002D1806880470346641C3078E4B2A042B8
:101DC000F1D8002B02D0596838468847387C06F491
:101DD00005D01422094B6A430021D018FF24C160AA
:101DE000448299504160018141816D1CEDB20A2D00
:101DF000B5D303B0F0BD0000504C0020884B00204C
:101E000070B50146094DCEB200202978044600295C
:101E10000BD9E10049198A88B24201D1886880470C
:101E2000641C2978E4B2A142F3D870BD504C002064
:101E3000F7B500248AB000940194029403940E46EE
:101E400004940594069407940894FF2701371168B9
:101E5000154638468847059601970090AA68696834
:101E60002868069000980892079100283CD069469F
:101E70000A9800F0CDF8002830D00098002806D04D
:101E800002994018F6F714FA029940180290AA68CD
:101E9000002A07D002990098491C904706001DD0DF
:101EA000009418E002982968401C8847060015D065
:101EB00002980199401C814201D20A4601E0029A2F
:101EC000521C30460099F6F7CFF9029834546968ED
:101ED00000988847009430460DB0F0BD0098002867
:101EE00002D069688847009400200DB0F0BD000062
:101EF000F8B500240A460546002910D0002D10D060
:101F000001460078002826D008780C283BD015DC44
:101F1000082838D0092836D00A2815D133E0002007
:101F2000F8BD03211046FCF757FB0028F8D022210A
:101F300001704170002181700120F8BD0D2822D070
:101F4000222820D05C281ED0202800D2641D48788A
:101F5000491C0028D8D1481B0719F91C1046FCF76A
:101F60003BFB061EE9D0002C0FD0222030702878D1
:101F7000741C002834D0C0B21F2813D9222811D0D5
:101F80005C2837D10EE0641CE1E7222434703A4625
:101F90002946701CF6F768F9F01944700021817029
:101FA0000120F8BD5C2020702A78641C0C2A23D004
:101FB00006DC082A1DD0092A24D00A2A06D11DE0F1
:101FC0000D2A1DD0222A12D05C2A13D00EA1204641
:101FD000F9F7B6FC241D6878641C6D1C0028CAD172
:101FE0002221F0194170002181700120F8BD2220CA
:101FF00000E062202070EEE76620FBE76E20F9E744
:102000007220F7E77420F5E775253034780000007A
:10201000002801D0002901D100207047F0B5054605
:10202000007B8BB00C4610287ED008DC012819D02C
:10203000022821D0042809D0082876D128E02028B9
:1020400074D0402873D080287DD19BE005212046A4
:10205000FCF7C2FA002803D0DCA1F7F7DDFA012073
:102060000BB0F0BD06212046FCF7B6FA0028F7D0E9
:10207000D8A1F7F789FA08E005212046FCF7ACFA69
:102080000028EDD0D5A1F7F7C7FA01200BB0F0BDBD
:1020900007910024AF69EE6900942E200194039407
:1020A00004940594029406940894314609940A9085
:1020B000002F01D0012000E0002001434800C94961
:1020C0004008081AC00F14D1012170004905C84208
:1020D00001D1002F0DD06869F6F788FD3A463346E6
:1020E000F6F726FE0BD1C0A168466A69F9F728FC0D
:1020F00026E0BEA16846F9F723FC054621E03A46F2
:102100003346BCA16846F9F71BFC054608AABBA1EB
:102110006846F6F711F901280CD13A463346099979
:102120000898FCF73DF803E03EE00CE041E094E065
:10213000002806D13A463346B1A16846F9F700FCBB
:1021400005461A2D02D300200BB0F0BD691C07987C
:10215000FCF742FA0028F7D0002D0BD92E236A464F
:10216000115D0A9EB14201D1035500E00155641C86
:10217000AC42F5D3002101550798806841190798B2
:10218000816082E728690028DED0F6F791F8401CCC
:10219000064601462046FCF71FFA0028D4D03246F6
:1021A0002969F6F761F870E72869FFF7A1FE0BB01F
:1021B000F0BDAD6801212046FCF70EFA0028F6D0EC
:1021C0005B210170A068401CA060E068401CE060DA
:1021D000002D34D0002621462846FFF719FF00289D
:1021E00013D0002C09D02068002806D0A168401820
:1021F000F6F75EF8A1684118A160286800281BD096
:102200006069002804D0022703E030460BB0F0BD1F
:102210000127791C2046FCF7DFF90028F5D02C2196
:1022200001706169401C002902D020210170401C0E
:102230000670A068C019A0602D68002DCBD10221C6
:102240002046FCF7C9F90028E0D05D21017000218B
:102250004170E068401EE06017E76069AD680028E3
:1022600001D0022700E00127791C2046FCF7B4F9D1
:102270000028CBD07B210170E168401C491CE16043
:1022800062690A21002A00D00170A068C019A0600C
:10229000002D78D000276069002814D02046E1681E
:1022A000FCF79AF9002825D0E2680021002A06D917
:1022B00009220270E368401C491C8B42F9D8E1688E
:1022C000A0684018A0602146286AFFF711FE002888
:1022D00010D0002C09D02068002806D0A168401832
:1022E000F5F7E6FFA1684118A1606069002804D0F5
:1022F000022603E038460BB0F0BD012631462046E9
:10230000FCF76AF90028F5D03A2101706169401C98
:10231000002901D009210170A06821468019A06020
:102320002846FFF775FE0028E4D0002C09D020686D
:10233000002806D0A1684018F5F7BAFFA168411837
:10234000A1606069002800D001202968002900D020
:1023500001214618711C2046FCF73EF90028C9D01F
:102360002968002902D02C210170401C61690029D4
:1023700002D00A210170401C0770A0688019A0607B
:102380002D68002D87D16069002802D0E168491CC2
:1023900000E002212046FCF71FF90028ABD061695C
:1023A00000290BD0E2680021012A07D0092202701F
:1023B000E368401C491C5B1E8B42F8D87D210170EC
:1023C00000214170E068401EE0605EE66E756C6C56
:1023D0000000000066616C73650000007472756532
:1023E000000000000000F07F256400006E756C6C3A
:1023F0000000000025312E3135670000256C670094
:1024000025312E313767000070B505460078002869
:1024100013D00A4E2846F5F74BFF84B20D2C00D995
:102420000D2471782346481C70702A460220FAF762
:102430009BFA2D1928780028ECD170BD5A4700204E
:10244000F8B5069E1F46182E01D9182500E035461E
:1024500013460A4601460CA00096F9F761FA0024DB
:10246000002D07D9395D11A0F9F75AFA641CA4B2FE
:10247000AC42F7D3AE4202D90EA0F9F751FA0FA041
:10248000F9F74EFAF8BD00005B424C452025735D1C
:1024900020747970653D307825303258207365712D
:1024A0003D2575206C656E3D257500002025303278
:1024B00058000000202E2E2E000000000D0A000003
:1024C000F8B5134E0F46756904463068001D00F0DC
:1024D000DBFE601C07D1002F05D031680D48091DB7
:1024E00000F06FFFF8BD30682C1944603168AC42D1
:1024F00004D2B068091D00F04BFFF8BD7068091DDB
:1025000000F046FF306B8442F7D23463F8BD000020
:10251000C4470020D46B0020124D134E134FE868BF
:10252000002817D000F05AFFF068C468201D00F0A2
:10253000ABFE2869401E2861E868401EE86000F094
:1025400059FF206B00F064FF204600F061FFE8684F
:102550000028E7D13868012801D900F07BFF00F09E
:10256000F9FEDCE7C4470020C06B0020F86A0020B9
:1025700030B4124900E011460A688242FBD34B682E
:102580005C18844203D140681818486008464368C4
:102590001C1894420CD10A4C2468A24206D05268FE
:1025A0009A1842600A681268026002E0046000E063
:1025B0000260814200D0086030BC704710480020A3
:1025C00000480020F7B582B0039800260068002874
:1025D00059D0039841680246496808324160009228
:1025E000914201D1496841604068C06801900398F8
:1025F000416849684160009A914201D1496841604F
:10260000CF68242002997043441804983D46002F57
:1026100001D11E490D682560294634316160E96A9F
:102620002161296BE161696CA1600023E96CA36100
:102630006161052813D015490A68954201D12373B9
:1026400011E0207303280ED1886B401C8863A86AB0
:10265000002801D00220207301F04EFD03E028463F
:10266000FBF78AFF2073286B00210278A52A04D18A
:102670004278401C491CA52AFAD088082084019879
:10268000761C8742B3D1304605B0F0BDC447002068
:1026900003480068401C72B600D0FEE7FEE7000069
:1026A00018480020F8B5054600F098FE2E46403642
:1026B00005243457002C0FDD2F462437686A002884
:1026C0000AD0384601F0E6FC002801D000F056FFA1
:1026D000641E64B2002CF1DC0027FF43777100F028
:1026E00089FE00F07BFE04243457002C10DD2846C0
:1026F00010300090286900280AD0009801F0CAFC28
:10270000002801D000F03AFF641E64B2002CF1DC16
:10271000377100F06FFEF8BDF8B50446002500F0F3
:10272000A7FF374E00273068364A002801D0F068EE
:102730001BE009213448C902430705D0C01DC00869
:10274000314BC000C31AC91A41180839C908C90059
:102750005760106031604F600B1A0F60436001607A
:10276000B3600120C0077360F06004423FD1002CC9
:102770003DD020460830410708D04107490F0823C3
:10278000591A0818410701D072B6FEE700282ED06A
:10279000716888422BD81B49146801E02146144611
:1027A0006268824202D22268002AF7D132689442DB
:1027B0001DD00D6822680A60616808350A1A102A5F
:1027C00009D921184B0701D072B6FEE74A60606054
:1027D0000846FFF7CDFE61687068401A7060B26805
:1027E000904200D2B060F06827600143616001F060
:1027F00083FC680701D072B6FEE72846F8BD0000EA
:102800000048002010480020E86B002004490868B8
:10281000002803D00868026D521C026508687047E2
:10282000C447002010B40124031F24061C601B1F92
:102830001960191F034B0B6014390A6010BC403833
:10284000704700009126010170B5064614460D46FA
:102850004720FFF717FA0369002B0DD01879B04213
:1028600007D158792880981D2060002B04D00020C3
:1028700070BD1B68002BF1D10020288020600A2049
:1028800070BD000070B516460C46104605F412D215
:10289000002813D14720FFF7F5F9054606233246F5
:1028A0001946074805F448D1A9886288891801802B
:1028B000A1884180A179017105F47AD1002070BD11
:1028C000180C0000F7B506460D464720FFF7DAF969
:1028D00004690746002C14D02079B0420BD16079EE
:1028E000A8420CD0384621461030F6F771FE20463B
:1028F00005F412D005E02468002CEDD101E0002C95
:102900000AD128460121083005F490D0044601463A
:1029100038461030F6F762FE267165712A46A01D12
:102920000299F5F7A1FC002003B0F0BDF8B5C56829
:102930000124287F0F4601281ADD0E4E204616225C
:1029400050430246296A10328A5A5204920F0BD120
:102950000A5C401C085C00021018B04204D1E1B2CD
:102960000022384600F03EF9287F641CA042E5DCD6
:10297000F8BD000002290000F8B5C5680124287FD1
:102980000F4601281ADD0E4E2046162250430246FD
:10299000296A10328A5A5204920F0BD10A5C401CE9
:1029A000085C00021018B04204D1E1B2002238469F
:1029B00000F018F9287F641CA042E5DCF8BD000097
:1029C0000229000070B5C46805462069002803D0BC
:1029D0000020002802D00EE00120FAE7264610363B
:1029E0003046F6F7E3FD04F497D72069002808D0B5
:1029F00000210029F4D00020E860204604F48CD7A0
:102A000070BD0121F5E710B504464720FFF73AF9FC
:102A100082790021A24202D98088001981B2084639
:102A200010BD70B504460D464720FFF72BF901464F
:102A300080888022A04206D889794118A14202D913
:102A4000201A28700022104670BDFFB585B00E9D7B
:102A50000646297801208840401E049018460E2121
:102A60000840328A69681F46403001920023039073
:102A7000009302912B7804AAA9680698F6F7D2FD74
:102A8000009000282AD10121282004F4CFD7044641
:102A9000AA686968286862622162E061F460069849
:102AA0000188A180217FA171F80701D00120C00316
:102AB000079908432080308A608047207082304622
:102AC00000F0AAF820461030F6F77CFD217F206A3E
:102AD00000F008F8308A002105F4FED0009809B013
:102AE000F0BD0000F3B583B00020019004980125EB
:102AF000012845DD1621039A69438818028A520489
:102B0000920F39D1039A4078515C000209181D4890
:102B1000814231D101A80290EFB204264720FFF78D
:102B2000B1F800900469002C14D02079B8420BD180
:102B30006079B0420CD0009821461030F6F748FD7D
:102B4000204604F4E9D605E02468002CEDD101E02C
:102B5000002C0AD130460121083004F467D704461E
:102B6000014600981030F6F739FD2771667132463C
:102B7000A01D0299F5F778FB04986D1C8542B9DB1E
:102B800005B0F0BD0229000000487047A8470101C8
:102B900070B5064610480D46007800281AD0472028
:102BA000FFF7B8F8A91D8BB2014603220B4804F4C5
:102BB000C3D704460A482A468078207001206070F6
:102BC00005206080A5803146A01DF5F74DFB20460D
:102BD00004F4EED770BD0000374700200647000020
:102BE000D04D002070B584B00E461446054601AAAB
:102BF00069463046FFF728FE6846028802A8019918
:102C0000F5F732FB02A84455024668460188304673
:102C1000FFF758FE04B070BD10B504464720FFF71B
:102C200031F8044921600921618118306060012078
:102C3000208110BDB8470101FFB583B00C46472085
:102C4000FFF720F80546808861882678401887B20B
:102C5000059805F42FD0012807D03846FCF7EAFD87
:102C60006946FFF7DEFE002802D0022007B0F0BD63
:102C70000121059805F430D00C3C0020AC6028738D
:102C800068460078687301AA02A9FFF7DDFDA8680D
:102C900001990446895D0C34890720D5A188C28832
:102CA00008318BB23102C1200001891D04F444D7E0
:102CB000064613203070A88861884018B080A0882C
:102CC000F0803046A288A11D0830F5F7CDFA3046D5
:102CD00004F46ED70121059804F4FED701E004F452
:102CE0001BD6012007B0F0BD10B5FAF789FC002013
:102CF00010BDFFB583B00C464720FEF7C3FF054665
:102D0000808861882678401887B2059804F4D2D765
:102D1000012807D03846FCF78DFD6946FFF781FE94
:102D2000002802D0022007B0F0BD0C3CAC602E732E
:102D300068460078687301AA02A9FFF785FDA868B4
:102D400001990446895D0C34890720D0A188C28886
:102D500008318BB23102C1200001891D04F4ECD688
:102D6000064612203070A88861884018B080A0887C
:102D7000F0803046A288A11D0830F5F775FA30467C
:102D800004F416D70121059804F4A6D701E004F451
:102D9000C3D5012007B0F0BD10B50C464720FEF7A3
:102DA00071FF80886188A31D401880B2A18800222D
:102DB000FAF7B2FB002010BDF8B5488800900C4629
:102DC0008E88F9F7E5FC00281DD0182E01D91827A8
:102DD00000E03746324626A00099F8F7A1FD00250D
:102DE000002F08D9601981792AA0F8F799FD6D1C88
:102DF000ADB2BD42F6D3BE4202D928A0F8F790FD8D
:102E000028A0F8F78DFD0098022821D0062804D0CC
:102E1000082822D00C2829D124E0022E26D1E088CF
:102E20002149012802D0002808D01FE001200870A5
:102E3000F9F7AEFC002819D01CA006E000200870AD
:102E4000F9F7A6FC002811D01EA0F8F769FD0DE0E7
:102E5000A188A01DF9F7B8FC08E0A188A01DF9F72A
:102E6000F7FB03E0A188A01DFAF7CEF80020F8BD1B
:102E70005B424C455D20777269746520696E643AE7
:102E8000206174745F6964783D2575206C656E3DC2
:102E9000257500002025303258000000202E2E2EEF
:102EA000000000000D0A0000374700205B424C453F
:102EB0005D206E6F7469667920656E61626C656411
:102EC0000D0A00005B424C455D206E6F74696679A7
:102ED0002064697361626C65640D0A00FFB581B09E
:102EE00000276846078048881C460D46082825D0DC
:102EF0000C2828D00A282AD005206946088016A662
:102F0000684600882146083083B21548039A04F4C5
:102F100013D6877129780446017068460288A2801A
:102F200069886180002A03D03146E01DF5F79CF9DD
:102F3000204604F43DD6002005B0F0BD6846F9F700
:102F4000FDFB0646DCE76846F9F7BEFF02E068468F
:102F5000F9F71CFF0646D3E74E53494E47000000E1
:102F60000547000070B516460C46104604F4A2D67C
:102F7000012818D1A1791A48002916D021780623F2
:102F800009023246891D04F4D7D50546A078FFF71B
:102F90003AFD288080202871284604F409D60021B3
:102FA000304604F499D6002070BDA1883246891DB0
:102FB0008BB221780902891D04F4BED50546A0789C
:102FC000FFF721FD288000202871A0886880A28852
:102FD000E11D681DF5F748F9284604F4E9D5DEE758
:102FE000140C0000F3B583B005001AD028680190D6
:102FF000284680380290C76F04983E1F864200D949
:1030000006462846F8F7E2FC044600913246294677
:103010000498FCF7F5FD0199002806D0016005B081
:10302000F0BD0498F8F704FDF9E729600299002C37
:10303000CF670AD021686218291F8A4202D9291B4A
:10304000091F216000996160E9E7024A0099116057
:10305000E5E700002048002010B5012400206407A7
:10306000206004F4BFD42E4802882E480168002056
:1030700004F444D52C4802882C480168012004F44B
:103080003DD52B48008882B22A480168022004F40A
:1030900035D52948008882B228480168032004F405
:1030A0002DD52748416AF02211434162254817F483
:1030B00017D5264824490160254941612549816089
:1030C0002549C160254981612549C16126492548B5
:1030D0008863FCF7F7FD2068C0B2F6F7A9FA234829
:1030E0000078002806D0002018F440D001460020C7
:1030F000F6F7A4FA2068C0B2F6F7A6FAF6F7AAFA2D
:103100002068C0B217F4BED52068C0B217F4C8D585
:103110002068C0B217F486D70120206010BD0000DF
:103120001C010020180100202401002020010020A3
:1031300034010020300100202C0100202801002053
:10314000402502407402002050025000808002405E
:1031500000080F0058086A00420500000F05050628
:103160000F000F034000D0004080024062000020AA
:10317000F0B5314C83B0E06980075AD50220206257
:10318000A56B082018F496D0012018F4A1D02B4983
:103190000027086940194608B219801A08612848B2
:1031A0000068F5F737FD0022264BF5F789FC019101
:1031B00000903E212846F6F753FA80197941F5F739
:1031C00037FD019B009AF5F713FCF5F77DFD0546E9
:1031D0001D4A0023F5F700F806461B49F6F740FAAA
:1031E0001A49281A081A81B2220419483243426047
:1031F0000160206B0821884308432063A0690721F0
:1032000009078843A061A169012081430143A161AD
:103210002062FCF757FD0F48104A00784100411822
:103220000D4808184178D1610D498078C8600D4873
:10323000077003B0F0BD000000800240A80200202B
:103240009000002000408F407102000070020000DA
:103250004080024010400020C84601014025024045
:10326000802502408000002000B50A4683B000217E
:103270000091019101466846F5F7C5FE0199009855
:1032800003B000BD704770474368826801699A6067
:10329000836842685A604A68824201D182684A6003
:1032A000002202610868401E08600868704700003C
:1032B0000148006970470000C4470020F8B5174670
:1032C000204A06460024906B0725401C9063106935
:1032D000814232D314206D1E1B49684341182420BB
:1032E000604380190122FFF76DF90419002DF1D117
:1032F0002420144D6043801902226968FFF762F9A7
:1033000004192420604380190222A968FFF75AF9A2
:10331000041924206043801904220C49FFF752F954
:10332000041924206043801903220949FFF74AF950
:103330000419002F01D00020386000F0DDFE204687
:10334000F8BD0000C4470020F86A0020C06B0020D0
:10335000D46B002010B500F0BDFD04490968401A87
:103360000349884201D2F7F75FFF10BD38470020BC
:10337000B80B00000146083100224160D243C16011
:103380008260016100210160704700210161704786
:1033900030B40C68621C02D00246083202E00269B6
:1033A00004E01A4653681D68A542FAD953684B6079
:1033B00099608A60516008610168491C016030BCF5
:1033C000704742684A6093688B6093685960916067
:1033D00008610168491C01607047000072B604482A
:1033E0000168491C0160BFF34F8FBFF36F8F7047B7
:1033F0001848002005490868002804D0401E0860CD
:1034000000D162B6704772B6FEE70000184800208F
:1034100000281CD070B504460D4D083C6068E96872
:10342000084201D172B6FEE72268002A01D072B6C6
:10343000FEE78843606000F01BF960686968401827
:1034400068602046FFF794F800F056FE70BD7047A4
:10345000004800200120044900074860BFF34F8F57
:10346000BFF36F8F7047000000ED00E010B500283B
:103470000FD009498A6B002A01D072B6FEE78A6B29
:10348000521C8A630021FFF71BF800F035FE00286C
:1034900001D1FFF7DFFF10BDC447002002498A6A4F
:1034A0000260496941607047C4470020F0B585B0AB
:1034B0000027054607702C48016902910069242104
:1034C0004843FFF729F906004CD000220299FFF784
:1034D000F5FE03970290002841D903982421484320
:1034E0008019017B052911D20A007A4412799218B9
:1034F0009744020406080A00582408E0522406E013
:10350000422404E0532402E0442400E00024416803
:103510002846F4F7F9FE2846F4F7CAFE0F2804D22D
:1035200020212954401C0F28FBD32F542D18039819
:10353000242148438019018C82680192009103691B
:1035400022460AA12846F8F7FBF92846F4F7B0FE10
:10355000451903980299401C03908842BDD3304618
:10356000FFF756FF05B0F0BDC447002009256309E9
:1035700025750925750925750D0A000001490120E9
:1035800048627047C447002010B50C46002809D097
:10359000054909681831FFF7FBFE01212046FEF7B7
:1035A0008FFF10BD72B6FEE7C447002070B50B4612
:1035B00004002FD0226D002A0ED0E16C994200D277
:1035C0001946E06A884225D0012A23D1124D2A6883
:1035D000944203D172B6FEE772B6FEE7E162A269D9
:1035E000002A02DB0722511AA16114220B4E50431C
:1035F0006169801981420DD1201DFFF745FEE06A07
:10360000A969884200D9A861142148438019211D65
:10361000FFF7D7FE70BD0000C4470020F86A002005
:1036200010B582B00D4800240190234680220CA1E1
:1036300000940D4800F082FB012803D0401C0BD100
:1036400072B6FEE772B600210848C9430163012142
:10365000C161446100F052F802B010BDF84700208B
:1036600049444C450000000019250101C4470020D1
:103670000248816B491C816370470000C4470020E9
:10368000164B986B002802D001205862704700202A
:1036900058629869142102464A4311498A58002AFF
:1036A0000AD1002806D01422401E42438A58002A1C
:1036B000F7D001E072B6FEE7142210B4424351186D
:1036C0004A680C46526808344A60A24201D15268E6
:1036D0004A60D1681960986110BC7047C4470020E7
:1036E000F86A002001484068704700000048002048
:1036F00001488068704700000048002070B50F48FE
:10370000016AFF22120411430162016A120211438D
:1037100001620B4C00252561A5610A487D21C90085
:103720000068F4F72FFD401E606107202061064805
:103730000560F4F7DDFC002070BD000000ED00E046
:1037400000E000E0004000201848002010B50246CC
:103750000021012000F00CF8041E07D00021416078
:1037600001600B460A46C16000F05BF8204610BDC0
:10377000F8B517460E46050016D0002E16D0704339
:103780005030FEF7C9FF04000CD020465030002E08
:103790000ED02060266420460121E56300F00AF87F
:1037A0004C2007552046F8BD72B6FEE70020E7E73B
:1037B0002460EFE770B50D46040026D0FFF70EFE3B
:1037C000216CE06B48432168411861600021A163CE
:1037D0002168A160E06B216C401E484321682246AD
:1037E00041180020C0434032E16010715071204602
:1037F0001030002D0BD0FFF7BDFD20462430FFF721
:10380000B9FDFFF7F7FD012070BD72B6FEE7216933
:103810000029F6D000F03EFC0028F2D0FFF71AFE97
:10382000EFE7FFB5002783B00446002803D00498D3
:10383000002802D006E072B6FEE7206C002801D016
:1038400072B6FEE70698022804D1E06B012801D089
:1038500072B6FEE700F02EFB002804D10598002880
:1038600001D072B6FEE72046254610304035029062
:10387000FFF7B4FDA06BE16B884208D306980228DD
:1038800005D0059800284AD0002F4BD04EE0069E68
:103890000499A56B0027226C002A11D0002E19D0A4
:1038A000E068F4F7E1FCE168206C091AE160226845
:1038B000914202D26168081AE060022E17D019E026
:1038C0002068002816D1606800F074FB07460020CD
:1038D00060600FE0A068F4F7C7FC216CA068401896
:1038E000A0606168884205D32068A06002E0002DD6
:1038F00000D06D1E6D1CA563606A002806D02046AE
:10390000243000F0C7FB002802D103E0002F01D0D3
:10391000FFF7A0FDFFF76EFD012007B0F0BDFFF738
:1039200069FD20E06846FFF7B9FD0127FFF762FD5A
:10393000FFF79EFEFFF752FD04202856401C00D1E1
:10394000287105202856401C00D16871FFF752FDF0
:1039500005A9684600F0C0F9002807D02046FEF708
:10396000A1FE00F0C9FB002007B0F0BDFFF736FD57
:10397000A06BE16B884201D1012600E00026FFF731
:1039800039FD002E0ED005990298FFF7FDFD204667
:10399000FEF788FE00F0B0FB002800D068E7FFF7D4
:1039A00059FD65E72046FEF77DFE00F0A5FB5FE7C9
:1039B00070B50D46040004D0206C002803D072B608
:1039C000FEE772B6FEE72068002804D16068002890
:1039D00001D072B6FEE7F4F79FFBA16B0646E06BE1
:1039E000884219D92246403205201056491CA1634D
:1039F000411C03D0401C507101240EE0606A002875
:103A0000FAD02046243000F045FB0028F4D0002DE9
:103A1000F2D001202860EFE700243046F4F780FB65
:103A2000204670BDF7B5002784B00446002803D0B7
:103A30000598002802D006E072B6FEE7206C002848
:103A400001D072B6FEE700F035FA002804D10698DE
:103A5000002801D072B6FEE72046254624304035C6
:103A60000290FFF7BBFCA66B002E21D0226C059BB9
:103A7000002A0BD0E0688018E0606168884201D3BA
:103A80002068E06001461846F4F7EEFB761EA66358
:103A90002069002807D02046103000F0FBFA0028EB
:103AA00001D0FFF7D7FCFFF7A5FC012007B0F0BD60
:103AB0000698002802D0002F05D008E0FFF79AFCF6
:103AC000002007B0F0BD6846FFF7E8FC0127FFF7CC
:103AD00091FCFFF7CDFDFFF781FC04202856401C28
:103AE00000D1287105202856401C00D16871FFF7CD
:103AF00081FC06A9684600F0EFF8002811D02046A6
:103B0000FEF7D0FD00F0F8FAFFF768FCA06B002884
:103B100027D00026FFF76EFC002EA2D0002007B0B1
:103B2000F0BDFFF75BFCA06B002812D00026FFF76A
:103B300061FC002E0FD006990298FFF725FD204664
:103B4000FEF7B0FD00F0D8FA00288AD1FFF782FC1A
:103B500087E70126EBE72046FEF7A4FD00F0CCFA4C
:103B60007FE70126D6E7F3B5002785B00446009726
:103B7000002804D0206C002803D072B6FEE772B68D
:103B8000FEE700F097F9002804D10698002801D03C
:103B900072B6FEE720462546243040350190FFF7F7
:103BA0001DFCA06B002817D0401EA06320680028D1
:103BB00002D1FEF72BFE60602069002807D0204666
:103BC000103000F067FA002801D0FFF743FCFFF740
:103BD00011FC012007B0F0BD0698002802D0002F8C
:103BE0000AD00DE00098002801D072B6FEE7FFF77A
:103BF00001FC002007B0F0BD02A8FFF74FFC012731
:103C0000FFF7F8FBFFF734FDFFF7E8FB0420285629
:103C1000401C00D1287105202856401C00D1687135
:103C2000FFF7E8FB06A902A800F056F800281BD011
:103C30002046FEF737FD00F05FFAFFF7CFFBA06BE1
:103C400000283ED00026FFF7D5FB002EA7D0009815
:103C500000283ED0FFF7C2FB606A002833D0206BFB
:103C600007210068091A2FE0FFF7B8FBA06B0028B6
:103C700008D00026FFF7BEFB002E1CD020680028CD
:103C800002D009E00126F5E7FFF7A8FB606800F025
:103C9000C5F90090FFF7AEFB06990198FFF774FC99
:103CA0002046FEF7FFFC00F027FA002800D076E758
:103CB000FFF7D0FB73E72046FEF7F4FC00F01CFA98
:103CC0006DE70126BFE700216068FFF76FFCFFF793
:103CD00091FB002007B0F0BDF8B50D46040012D0EE
:103CE000002D12D0FFF77AFB134E726963682868C3
:103CF000D11A471C0BD02768B66AB74209D0934245
:103D000007D8012413E072B6FEE772B6FEE700247E
:103D10000DE0884208D9401A28600748816A21606E
:103D200040696060002402E0002001242860FFF761
:103D300061FB2046F8BD0000C4470020FFB585B0F8
:103D400090000F9F0E9D0290FEF7E6FC06001ED02D
:103D50005C20FEF7E1FC040016D026630599019172
:103D60000899009130460299069EA5220391F4F726
:103D70008DFA0399206B091F4018C008C0000290FB
:103D8000400708D072B6FEE73046FFF741FB00203F
:103D9000C04309B0F0BD2118325C20310A75315C96
:103DA000002902D0401C1028F5D3264600204036BA
:103DB000F070072D00D30625E5620020E56420653C
:103DC000201DFFF7E2FA20461830FFF7DEFA2461E3
:103DD0000720411B6462A161002161653176009A70
:103DE00001990298FEF71EFD2060002F00D03C6074
:103DF0002546FFF7F3FA284E3069401C30613068E1
:103E0000264F002803D0F069002821D026E0356035
:103E10003069012822D1002414206043C019FFF723
:103E2000A9FA641C072CF7D31D48FFF7A3FA1D4815
:103E3000FFF7A0FA1C48FFF79DFA1C48FFF79AFA13
:103E40001B48FFF797FA164870601430B06005E021
:103E50003068E96AC06A884200D83560F06A401C60
:103E6000F0626864E86AB169884200D9B0611421DF
:103E70004843C019291DFFF7A4FAFFF7BBFAF06900
:103E8000002806D03068E96AC06A884201D2FFF78C
:103E9000E1FA012009B0F0BDC4470020F86A002013
:103EA000846B0020986B0020AC6B0020C06B00205E
:103EB000D46B00200648C169002904D0806B00281B
:103EC00003D0002070470120704702207047000097
:103ED000C44700200148406970470000C4470020E3
:103EE000F8B5324F0026B86B002808D0386A401C5D
:103EF0003862786A002800D001263046F8BD7D6916
:103F00006D1C7D6115D178680068002801D072B6FB
:103F1000FEE77868B9687960B860B86A401CB86232
:103F200078680068002813D07868C068C068406866
:103F30003863386B854211D37868006800280AD04E
:103F40007868C068C4686068854211D2386305E04B
:103F50000020C043ECE70020C043386338681421D8
:103F6000C06A4843124908580128C2D90126C0E74F
:103F7000201DFFF789F9A06A002803D020461830D9
:103F8000FFF782F9E06AB969884200D9B861142163
:103F9000484307494018211DFFF713FAE06A3968C2
:103FA000C96A8842C8D30126C6E70000C44700207A
:103FB000F86A002070B500210446002828D0154D6D
:103FC0002868844201D072B6FEE7206D002808D030
:103FD000401E2065E36CE26A9A4219D0002802D0A4
:103FE00016E072B6FEE7201DFFF74EF9E06C0721E0
:103FF000E062081AA061E06AA969884200D9A86154
:104000001421484304494018211DFFF7DAF9012122
:10401000084670BDC4470020F86A002070B5044609
:104020000020002C2AD0194DE16A2A68D26A9142F8
:1040300025D2A069002804DB28680721C06A081A75
:10404000A061E06A1422124E5043616980198142D6
:1040500010D1201DFFF718F92868C06AE062A9692D
:10406000884200D9A861142148438019211DFFF717
:10407000A8F902E02868C06AE062012070BDE16C26
:104080002A68D26A9142F8D370BD0000C44700206C
:10409000F86A002070B5C068C468002C0BD02046B8
:1040A00018300646FFF7F0F8104DA86B002804D032
:1040B00031460F480EE072B6FEE7201DFFF7E4F828
:1040C000E06AA969884200D9A861142148430949D6
:1040D0004018211DFFF775F9E06A2968C96A88420E
:1040E00002D90120686270BD002070BDC447002065
:1040F000AC6B0020F86A0020F8B52E4D0027A86BA5
:10410000002808D0FFF76AF9A86B401EA863A86BC7
:10411000002802D046E072B6FEE72869002841D0A8
:10412000254E306800282AD0F068C4682046183030
:10413000FFF7AAF8201DFFF7A7F8E06AA9698842EF
:1041400000D9A861142148431C494018211DFFF7DC
:1041500038F9E06A2968C96A884201D30120686297
:1041600030680028E0D1002C09D068682946006832
:1041700000281BD04868C068C068406808632C6A83
:10418000002C09D00126FFF7ABFE002800D06E629C
:10419000641EF8D100202862686A002802D0012736
:1041A000FFF758F9FFF726F93846F8BD0020C0435D
:1041B000E4E70000C4470020AC6B0020F86A002050
:1041C00040BA7047C0BA70470138FDD1704700004F
:1041D000F7B50325AD06286A82B016460C4640089E
:1041E00040002862286A022108432862286A800762
:1041F000FCD46620686001272F61A86AC005FCD541
:10420000992068602F61A86AC005FCD5FF20913015
:10421000FFF7DAFFFF230133AB626846EF60352119
:1042200069602F61A96AC905FCD5AB62A969EF6015
:10423000C9B205226A602F61AA6AD205FCD5AB62B9
:10424000AA690902D2B211430180C80702D0032033
:1042500005B0F0BDAB626869FF2108318843686131
:104260006869C91E084368610298000248306860A6
:104270000820A860EE602F61A86AC005FCD5FF2069
:104280000130A8620023F61CB0080ED0B208114815
:10429000006899006054060A09194E70060C000E59
:1042A0008E705B1CC8709A42F1D8FF200130A86262
:1042B0006869FF210831884368616869384368612B
:1042C000286A800880002862286A38432862002013
:1042D00005B0F0BD8000000C032080064169FF227C
:1042E000083291434161426901210A434261026AF5
:1042F000920892000262026A0A430262704700005A
:10430000002003218906096A490849000322920610
:1043100011621146096A02221143032292061162B8
:1043200000BF03218906096A022211400229F8D040
:10433000D1010322920691620321D1609F21516035
:104340000121116100BF03218906896AFF22013220
:1043500011409142F7D10322920691621146886979
:104360004969FF22083291430322920651611146A6
:104370004969012211430322920651611146096ADB
:104380008908890011621146096A0122114303223A
:104390009206116270470000000001020000000058
:1043A000010203040138FDD170470000F0B403247A
:1043B000A406236A5B085B002362236A02252B4361
:1043C0002362236A9B07FCD4FF230133A362656940
:1043D000DE1DB543656165691E1D354365610002DB
:1043E0006B3060600820A060E26001262661A06A50
:1043F000C005FCD5A3620023D21C90080ED09508FE
:104400000F4800689A008854070A52185770070C22
:10441000000E97705B1CD0709D42F1D86069FF213F
:10442000083188436061606930436061206A8008B8
:1044300080002062206A30432062F0BC0020704778
:104440008000000CF8B5064601200025C004864215
:1044500001D90520F8BD0324A406206A40084000C5
:104460002062206A022108432062206A8007FCD46F
:10447000FF270137A76200F0BBF8002801D0032511
:1044800015E00620606001212161A06AC005FCD50D
:10449000A7623002203060602161A06AC005FCD5AF
:1044A000A7620C4800F0C8F8002800D10225606916
:1044B000FF21083188436061606901210843606120
:1044C000206A800880002062206A08432062284613
:1044D000F8BD0000E6960100F7B506460120C004CD
:1044E00082B01546864202D9052005B0F0BD0320F2
:1044F0008006016A490849000162016A02221143EB
:104500000162016A8907FCD4FF2101318162F2B2A4
:104510008C1AA54200D8ACB20398009000F068F85D
:10452000002840D106214806416001210161816ACD
:10453000C905FCD5FF210131032080068162416954
:10454000FF220832914341614169042211434161D4
:10455000310232314160C4600022002C16D900982B
:1045600087183B78F87819467B7800061B021943B8
:10457000BB781B04194301430802F978000A0906B5
:10458000084319490860121DA242E8D30121032003
:1045900080060161816AC905FCD5FF210131816274
:1045A000124800F049F8A54209D0039836190019BD
:1045B0002D1BFF2401340390A542ADD8ABE70320A7
:1045C00080064169FF22083291434161416901221D
:1045D00011434161016A890889000162016A11433E
:1045E0000162002005B0F0BD8000000C1A0600003A
:1045F00038B40125032080066A46C5603521416034
:104600000561816AC905FCD5FF2401348462816992
:10461000C560CBB2052141600561816AC905FCD541
:10462000846280691902C0B2014388B21180C00758
:1046300000D0012038BC7047F8B4002101250322C6
:1046400092066B46D560352454601561946AE40582
:10465000FCD5FF27013797629469D560E4B205263F
:1046600056601561966AF605FCD597629669240234
:10467000F6B234431C80E30722D0814202D9F8BC51
:1046800000207047032292066B46D56035245460A3
:104690001561491C946AE405FCD597629469D5605C
:1046A000E4B2052656601561966AF605FCD5976258
:1046B00092692402D2B21443A2B21C80D207DCD188
:1046C000F8BC0120704700000017130017100017F6
:1046D0000E0017090017040017000017180117141F
:1046E0000117150117190000002800020000000042
:1046F0000328000200000000292A00020080800038
:104700000328000200000000242A0002008080002C
:104710000328000200000000252A0002008080001B
:104720000328000200000000272A00020080800009
:104730000328000200000000262A000200808000FA
:104740000328000200000000282A000200808000E8
:104750000328000200000000232A00020080080055
:1047600003280002000000002A2A0002008008003E
:104770000328000200000000502A00020080070009
:104780009DE200012BE2000129E2000127E2000185
:104790000014000045E30001130C000081F5000146
:1047A0000314000001E400014B2A0101C5290101A5
:1047B000792901012D290101130C000045F60001A2
:1047C000150C000025F70001170C00005DF4000136
:1047D000000C00009DF4000106470000F32C0101CD
:1047E00003470000992D010108470000392C010101
:1047F0000E4700008528010105470000652F0101D3
:10480000FFFF0000D9D20001130E00009DE7000158
:10481000150E0000ADE60001170E00001DEC0001B2
:10482000190E0000F5EB0001004801010500000031
:10483000F7B586B0002002905C48154604695C48D4
:104840000E46824201D9054602E0002D00D1012525
:10485000002C08D0A1880698814204D1E088B0429B
:1048600001D1012002905348039084460698010428
:1048700031430020002C1CD00A0CA7888BB2974231
:1048800007D1E7889F4204D1002807D02168016042
:1048900007E020462468002CEFD10AE06146226838
:1048A0000A602168002902D00020206001E06146F2
:1048B0004860002C07D10221102000F095F80699DD
:1048C00081800446C6802801052100F077F807465C
:1048D0007D200E464643EFF31085012080F31088BB
:1048E000684600F087F885F3108800980490C01996
:1048F0000501019927202D098E1900010591864295
:1049000003D96D1C2D012D09361AE660A5600398A8
:10491000294F86460020844670460068002813D040
:10492000A268E1680091C36881680193531A1B0172
:104930001B09BB420AD2914203D1019A00999142CC
:1049400004D984460068E9E77246546020606046F6
:10495000002801D0046001E071460C601348029900
:104960000069002901D1A04203D1C168806800F02C
:1049700047F8EFF31084012080F3108802A800F0BC
:1049800039F884F31088039902980191291A0901D2
:1049900009090090B94204D2A84205D10198864283
:1049A00002D8032000F032F809B0F0BDC8010020A1
:1049B000FFFF7F02D8010020FFFFFF0730B50B4645
:1049C000014600202022012409E00D46D5409D42E9
:1049D00005D31D469540491B25469540401915466F
:1049E000521E002DF1DC30BD03B40148019001BD21
:1049F0002D7A010003B40148019001BD5DB60200AB
:104A000003B40148019001BD9DB6020003B4014802
:104A1000019001BDAD78010030B4C3688268886838
:104A2000084D141A2401C9682409AC4203D29042EB
:104A300004D18B4202D830BC0120704730BC00202A
:104A400070470000FFFFFF070A0C838889B293427A
:104A500004D1C088884201D10120704700207047EE
:104A600070B4054600680022002810D00B0C868820
:104A70008CB29E4207D1C688A64204D10168002AA2
:104A800007D0116006E0024600680028EFD170BC34
:104A9000704729600168002903D00021016070BCC3
:104AA00070476A6070BC7047F0B5104F0268864668
:104AB0000025002A10D0C8688C6893688446E01AE4
:104AC00000010009D668B84208D2A34201D1B4451A
:104AD00004D915461268ECE7704641600A60002D63
:104AE00001D02960F0BD70460160F0BDFFFFFF07F7
:104AF00070B584B004460E46EFF31085012080F3B4
:104B0000108802A8FFF776FF85F3108802980399B2
:104B1000024600900191A01A00010749000988424D
:104B200004D2A24205D10198864202D8012004B0E5
:104B300070BD002004B070BDFFFFFF0730B583B02B
:104B40000446EFF31085012080F310886846FFF7D4
:104B500051FF85F31088019900986160206003B0CF
:104B600030BD000000280002000000000328000201
:104B700000000000002A000A008020000328000234
:104B800000000000012A0002008002000328000249
:104B900000000000042A0002008008000328000230
:104BA00000000000A62A0002008001000328000285
:104BB00000000000C92A0002008001000028000255
:104BC000000000000328000200000000052A002069
:104BD000008004000229000A0000020003280002ED
:104BE00000000000292B000A0080100003280002AA
:104BF000000000002A2B000200801000FFFF0000D0
:104C0000B5CB0001A40D0000C1EE0001A50D000010
:104C1000F5EE00011A0D00000DF40001150D000065
:104C200055EF0001000D000081EF00011C0D000098
:104C300043F40001A70D000061F30001A80D00007E
:104C40004FF40001020C000035F50001000C0000DB
:104C50000DF50001010E000039EA00010F0E000001
:104C6000F5ED0001110E000059EE00012C0E0000C0
:104C7000D9ED0001030E000091EB00010A0E0000C7
:104C80004DED0001300E0000CDED00010C0E0000D6
:104C900081EE0001000E0000A5E90001090E0000F0
:104CA000CDE90001010F0000F5CD0001020F000069
:104CB0007DCA0001030F0000D9CD0001040F0000E0
:104CC000710D0101FC4B0101364700200100190064
:104CD000021400007DE40001D04C0101010000003D
:104CE000184E01010300000001102EC78A0E7390B8
:104CF000E111C20860270000002800000000000049
:104D00000000000000000000000200000000032876
:104D10000000000000000000000000000000000A89
:104D20000000000001002EC78A0E7390E111C20836
:104D300060270000000400C00002012900000000FC
:104D400000000000000000000000000A00801400C5
:104D50000328000000000000000000000000000028
:104D6000000A0000000002002EC78A0E7390E111B5
:104D7000C20860270000001000C0000202290000E5
:104D8000000000000000000000000000000A008099
:104D900014000328000000000000000000000000D4
:104DA0000000000A0000000003002EC78A0E739066
:104DB000E111C20860270000000A00C000020328B9
:104DC0000000000000000000000000000000000AD9
:104DD0000000000004002EC78A0E7390E111C20883
:104DE00060270000000200C000020328000000004D
:104DF00000000000000000000000000A00000000A9
:104E000005002EC78A0E7390E111C20860270000CA
:104E1000000A00C00002000004470000DD2E01016E
:104E20000A470000B92D010107470000E92C0101E4
:104E300008530101D4520101A1AA0001B05201019D
:104E40009852010129AE0001B8520101B05101018F
:104E50008DAC0001CC520101B850010135A8000110
:104E60006452010120510101BDA70001205201013E
:104E7000EC51010175AB000140530101F4500101F7
:104E8000999E000150530101E0530101619F00010F
:104E9000105301016C520101419B00015853010163
:104EA00048500101759B0001D0530101605301017D
:104EB000559800011C5201018050010145AC0001D0
:104EC000485301015C51010159AC0001D853010163
:104ED00098530101CDA90001C853010124520101D9
:104EE000E5AD0001C05201011853010175AD00018B
:104EF0005C5201017C5101015DAA00010102030421
:104F0000050607004040404040404040404141418C
:104F1000414140404040404040404040404040408F
:104F20004040404005020202020202020202020266
:104F30000202020220202020202020202020020225
:104F400002020202029090909090901010101010A7
:104F5000101010101010101010101010101010025F
:104F600002020202028888888888880808080808DF
:104F700008080808080808080808080808080802B7
:104F800002020240044F0101666C6F7720636F6E6E
:104F900074726F6C3A206E6F6E653B2074783A20A5
:104FA000444D41204348312028706F6C6C65642962
:104FB0003B2072783A20444D4120434832207269A8
:104FC0006E672028334B422C2069646C652069721F
:104FD00071290D0A000000005B6F74615D20626939
:104FE0006E617279206D6F6465204F4E202D2073A5
:104FF000656E642030784341204F544120667261D1
:105000006D6573206E6F770D0A28626C655F707234
:105010006F746F636F6C2E6D642073656374696F5A
:105020006E20362E363B204F54415F41424F525442
:10503000206F722033732069646C65206578697411
:1050400073290D0A000000006273736574203C66CA
:1050500069656C643E203C76616C3E3A20777269EB
:10506000746520626F6F7473657474696E6720660F
:1050700069656C6420286361726566756C2129001E
:105080006F74613A205541525420656E7465727395
:10509000204F54412062696E617279206672616DA1
:1050A00065206D6F646520287365652068656C7088
:1050B000206F74612900000073686F772064657643
:1050C00069636520696E666F202874656D702F7640
:1050D00064642F66616E2C2073616D65206173209E
:1050E000424C4520494E464F5F515545525920612B
:1050F0006C6C2900617070676574205B6A736F6EF9
:105100005D3A2073686F7720617070207061726102
:105110006D7320286C65642F70776D290000000086
:10512000626C656C6F67205B6F6E7C6F66665D3A64
:1051300020424C452074726166666963206C6F671B
:1051400020286576656E7473202B206672616D650C
:10515000206865782064756D70290000726573653C
:10516000743A2073797374656D2072657365742069
:10517000287265626F6F74290000000068616E67B5
:105180003A2077656467652074686520434C492040
:105190007461736B202849574447207761746368B2
:1051A000646F6720666972652074657374290000F6
:1051B00073686F77204672656552544F532072753D
:1051C0006E74696D6520696E666F202875707469EC
:1051D0006D652F7461736B732F686561702F7461D7
:1051E000736B206C69737429000000006C65642087
:1051F0003C317C323E203C6F6E7C6F66667C746F07
:1052000067676C653E3A20636F6E74726F6C2062E4
:105210006F617264204C4544000000006F746100AF
:105220006C656400756172747273743A2072652DD6
:10523000696E6974205553415254312028343630F8
:1052400038303020384E31292C20666C7573682038
:1052500072782071756575650000000068616E6781
:1052600000000000626C656C6F670000627364751B
:105270006D703A2073686F7720626F6F7473657416
:1052800074696E67207265636F7264202B2063728D
:105290006320636865636B0073686F77206669726B
:1052A0006D776172652076657273696F6E000000BC
:1052B00076657273696F6E00737973696E666F00DD
:1052C00075617274696E666F0000000064657669CE
:1052D0006E666F0068656C70205B636D645D3A207C
:1052E0006C69737420636F6D6D616E6473202F2021
:1052F00073686F77206F6E6520636F6D6D616E648C
:1053000027732068656C700068656C700000000091
:10531000627364756D70000075617274696E666F9A
:105320003A2073686F772055534152543120706989
:105330006E732F626175642F666F726D6174000009
:1053400061707067657400007265736574000000B9
:10535000617070736574000062737365740000009F
:105360006170707377205B317C325D3A20737769AE
:1053700074636820626F6F742062616E6B202863B3
:10538000726320766572696669656429202B2072D4
:1053900065626F6F74000000666163746F72793AC2
:1053A00020726573746F726520706172616D732015
:1053B000746F2064656661756C747320616E64201F
:1053C0007265626F6F74000075617274727374003D
:1053D0006170707377000000666163746F727900AA
:1053E000617070736574203C6C65647C70776D3E91
:1053F000203C76616C3E207C206170707365742067
:105400006A736F6E207B226C6564223A3530307D82
:105410000000000075736167653A20617070736504
:1054200074203C6C65647C70776D3E203C76616CCA
:105430003E207C20617070736574206A736F6E20EB
:105440007B226C6564223A3530302C2270776D22D5
:105450003A35307D0D0A000061707073773A206232
:10546000616E6B256C7520696D6167652063726381
:10547000206D69736D6174636820287265636F7253
:10548000642030782530386C582C20616374756145
:105490006C2030782530386C58290D0A0000000047
:1054A0002020202020202020206231616464727C32
:1054B0006232616464727C623173697A657C6232E3
:1054C00073697A657C62316372637C623263726392
:1054D0007C62317665727C6232766572203C6865EA
:1054E000787C6465633E0D0A000000000C550101E4
:1054F000004000202C08000030950001245B0101D1
:105500002C480020BC750000F02A000011D490D077
:105510000322A01AFF01011013C202025420382BEB
:1055200011D80D490868496813F008FB0498EFF793
:105530008EFF0446C1888088FF22FFF79DFD20462C
:10554000FFF73AFCB3E705B0F0BD981407D8011B8C
:1055500020C8042430D702100E4B1847FBFD064626
:10556000052030707580281699B181301D3946E5C7
:10557000F773FD3046F9F70EFF0E222946422C45FF
:10558000FD074038112E0CD0534B0522032128462D
:10559000FDF733FE121E134B75162D05D0398F14EF
:1055A0002902D01499897912E01010211176FAF7A6
:1055B0004BF8044D2859F9F7FBFE4C202851801177
:1055C00012041B2007771538B5049C103294014C47
:1055D000A04738BD5143F84A26468F183946203631
:1055E000FD6D707D80311191C97FA0370E912246EB
:1055F000397815320F92F14A109203292BD0100CF2
:105600002873D0F17D0F980CF00DF81014286FD08E
:10561000688869460883F0B597B008780C460F9003
:1056200010182014900F9848214843FE4922464004
:1056300018064680361090F17F180991C56DA0308C
:105640001690014E180A274612922037F74A155233
:10565000100F2AD061783C2949D0432947D0787D62
:105660001008287DD0F97D129814F0FCF9100E284E
:1056700078D0698868468184687A297A102204097A
:10568000020843E97908430690A97A08A84172E91B
:105690007A8172297BC17229460D310E380E911024
:1056A0000AF02FFAA878400733D5100E2132E09087
:1056B0007E012806D0507E401E120610080E50763D
:1056C00003D006E03D21DB480106111012F0D2F9AB
:1056D000169A01211170A978D448C9075CD0100826
:1056E00099482359430818101822A0300270FF204F
:1056F000F07752E001220270A878CC49C0074CD064
:105700009F98482358434020181442E0E97C08A899
:105710000173297D4173697D8173A97DC108180DCD
:105720000174297E4174697E8174B189BC101E8127
:10573000F189C181318A0182109940318A8F828337
:10574000C98F0184B188C183F18841841C21C1843F
:1057500042101472B848817808A8C17401E04DE184
:105760001BE0022606752C2902D0CC100D02D4E8CD
:105770007A800705D5297B0E98380BF07EF908A9A9
:10578000087503A90F0C1110402801D11698067056
:1057900060783C2870D030E1628869460A82A2882D
:1057A0004A82A2790A75E2794A75207A8875E07E84
:1057B000C875A08B0883E08B4883208C8883608C1D
:1057C000C8832146243108A81018F0A4F9787A0873
:1057D000A94871B87A8871A08D69460885206B0B3D
:1057E000901E200C90012018103E75387D0875B869
:1057F0007D8875A878C006C017401CC8758E48699A
:1058000046028A0A87428A4A87827D08A90A77C2A5
:105810007D4A77027E8A77428B10A90A80828B4A62
:1058200080807F087104A919A41332F910109848D8
:105830002148437C49401803907C301299101AF09B
:105840005DF90398F97D8030817003990922A031B8
:105850000A700121C170039817218166E18B4910FC
:105860000F41660521C166016715996030C97E1830
:105870000E2904D072498161012102E02AE024143A
:105880006181751F998182F97D12601009F6F80215
:105890002802D201214CF003F912281B05F9062831
:1058A0000CD20A215F4A41438918FF318131497F77
:1058B000890703D5FA7D7C2BFCF8961DFFF8169915
:1058C000E0100C70FF20F077012014900920100ADE
:1058D000F0FBF821460F3105911008284ED0202307
:1058E0003E222C21564860100906460A20307014CA
:1058F00098142801D01220100AE03C20707001207A
:1059000030712C987080162D2CD0B01D5A1015F2C5
:10591000F8F87D7071E87A800706D521463046098F
:10592000310C302808F0E7F803E030460A1ADD2091
:10593000180A800705D53046123005303ADA1A1AAF
:10594000121A1015D0F8E08B3083208C7083608C95
:10595000B083B87AB07730461010F0BFF83AE0283C
:105960007B707129460D31B01D2CF0C2F8163EB483
:10597000F83DE0149E1A2E9E3808A7F8012106462D
:10598000019E1A0D9E3C70703198280BF87D82079D
:1059900009D57171B01D6A3CA5F80AB6180A3046DF
:1059A0001DE0C007C00F701829B21A9978180BB003
:1059B00081208CF081608C3082782A74623C83F87C
:1059C00006601A16601777F81421017010089941C3
:1059D00080B97D01713815F075F81598807E022820
:1059E00026D160781499084322D0082C1A0B2C1C5D
:1059F00061F8122C100D61784170297881700FE0E8
:105A000040041420C00624200A201A39041A400C2D
:105A100011190414B1A2013304111F998180397E38
:105A20008156134AF81E2017B0F0BD241DBA7047E6
:105A3000C004100C03B40148019001BD919B0269A0
:105A40000C8BE1980C8B7D9F0C7C49FA010C8B0927
:105A5000D30C8B6D5B249B3D99488A900C8B55072A
:105A6000308BD59C188B397B1824796D0118222135
:105A700001804180818070470A7802704B784370C2
:105A80008A788270CA78C2700B7903714A79427140
:105A90001A2C6802600E033670472017497B41704C
:105AA0000570F1F7F3FC2068F1F7A4FB256003B063
:105AB000F0BD22241220200A80024080C10240064C
:105AC000021017F8B54E784821F0B2484323492117
:105AD0004D41180C46AA7EA0346A27B014EDC302CB
:105AE0001710B5074CE069100A0408D5FFF7F3FF5B
:105AF00005481278180B2802D10120C0032062103B
:105B00005429501AC6581AF4DB016EC3FFFF133133
:105B1000BA1401CDB90D5701E52F018A1AAA010166
:045B20001000000071
:00000001FF
